:020000040800F2
:100000000000022005A500084BA500084DA500082A
:100010004FA5000851A5000853A5000800000000E6
:1000200000000000000000000000000055A50008CE
:1000300057A500080000000059A500080118000895
:100040005FA5000861A5000863A5000865A5000874
:1000500067A5000869A500086BA500086DA5000844
:100060006FA5000871A5000873A5000875A5000814
:1000700077A5000879A500087BA5000895AA0008C7
:100080007FA5000881A5000883A5000885A50008B4
:1000900087A5000889A500088BA500088DA5000884
:1000A0008FA5000891A5000893A5000895A5000854
:1000B000A584000899A500089BA500089DA5000837
:1000C0009FA50008A1A50008A3A50008A5A50008F4
:1000D000A7A50008A9A5000815830008ADA500087C
:1000E000AFA50008B1A50008B3A50008B5A5000894
:1000F000B7A50008B9A50008BBA50008BDA5000864
:10010000BFA50008C1A50008C3A50008C5A5000833
:10011000C7A50008C9A50008CBA50008CDA5000803
:10012000CFA50008D1A50008D3A50008D5A50008D3
:10013000D7A50008D9A50008DBA50008DDA50008A3
:10014000DFA50008E1A50008E3A50008E5A5000873
:10015000E7A50008E9A50008EBA50008FD46000892
:10016000EFA50008F1A50008F3A50008F5A5000813
:10017000F7A50008F9A50008FBA50008FDA50008E3
:10018000FFA5000801A6000810B5054C237833B977
:10019000044B13B10448AFF300800123237010BD5A
:1001A000A402002000000000F4FC000808B5064B83
:1001B0001BB106480649AFF300800648036813B137
:1001C000054B03B1984708BD00000000F4FC00088F
:1001D000A8020020A402002000000000154B002B04
:1001E00008BF134B9D46A3F5803A00218B460F466E
:1001F0001348144A121A0AF06CFE0F4B002B00D061
:1002000098470E4B002B00D0984700200021040097
:100210000D000D48002802D00C48AFF300800AF012
:100220000BFE2000290008F06DFA0AF0F1FD00BF76
:100230000000080000000220000000000000000094
:10024000A4020020F4620020000000000000000072
:1002500030B4C3787BB902784FF461435109CEF2D0
:10026000000302F01F022031012000FA02F243F8DD
:10027000212030BC70474FF46D43CEF20003457827
:10028000DA6884780378D243C2F30222C2F104010F
:10029000C9B205FA01F10F2545FA02F2C9B22240AE
:1002A0000A4303F1604303F561431201D2B283F8BC
:1002B000002302784FF461435109CEF2000302F0AB
:1002C0001F02012000FA02F243F82120D1E700BF0B
:1002D000F0B444680B680A7924F0407424F4807404
:1002E000234343EA02234360CD680C6987688A6828
:1002F0004E794FF2FD732C43CCF2FF0322433B4077
:10030000134343EA460383600B7DC26A013B22F438
:100310007002DBB242EA0353C362F0BC704700BF15
:1003200000230360037143718360C3600361012391
:100330000375704770B44FF40C5290E84200C4F259
:10034000010285685468C06843F2E0033143CFF688
:10035000FC732943234001430B43536070BC704737
:100360000023036043608360C3607047836819B9EA
:1003700023F001038360704743F0010383607047FB
:10038000092970B421D901EB41041E3CC668072538
:1003900005FA04F526EA050503FA04F445EA040320
:1003A000062AC36020D90C2A02EB82022BD9413ADB
:1003B000C46A1F2303FA02F324EA030301FA02F1D9
:1003C00043EA0102C26270BC7047066901EB410456
:1003D000072505FA04F526EA050503FA04F445EABB
:1003E0000403062A0361DED8013A02EB8202446B61
:1003F0001F2303FA02F324EA030301FA02F143EA9A
:1004000001024263DFE7233A046B1F2303FA02F37E
:1004100024EA030301FA02F143EA01020263D2E78C
:10042000836843F080438360704700BFC06C80B234
:10043000704700BF036819420CBF002001207047BD
:10044000016846F21002002321F00101C4F2020209
:100450000160036043608360C360036121239042B5
:1004600043616BD046F22803C4F2020398426CD079
:1004700046F24003C4F2020398426ED046F258039B
:10048000C4F20203984270D046F27003C4F2020331
:10049000984272D046F28803C4F20203984275D0A3
:1004A00046F2A003C4F2020398423ED046F2B803DB
:1004B000C4F20203984273D046F21043C4F202031E
:1004C000984275D046F22843C4F20203984276D08F
:1004D00046F24043C4F20203984278D046F25843B1
:1004E000C4F2020398427AD046F27043C4F2020387
:1004F00098427CD046F28843C4F2020398427FD0EF
:1005000046F2A043C4F20203984200F0838046F210
:10051000B843C4F20203984201BF4FF4C843C4F287
:1005200002034FF03D52DA6070474FF4C043C4F20B
:1005300002030022C2F23D02DA6070474FF4C0436A
:10054000C4F202033D229A6070474FF4C043C4F2E4
:1005500002034FF474629A6070474FF4C043C4F2D0
:1005600002034FF474129A6070474FF4C043C4F210
:1005700002034FF074629A6070474FF4C043C4F2B4
:1005800002033D22C2F20002DA6070474FF4C0431A
:10059000C4F202034FF47462C2F20002DA607047E0
:1005A0004FF4C043C4F202034FF03D52DA6070478B
:1005B0004FF4C843C4F202033D229A6070474FF4DF
:1005C000C843C4F202034FF474629A6070474FF458
:1005D000C843C4F202034FF474129A6070474FF498
:1005E000C843C4F202034FF074629A6070474FF43C
:1005F000C843C4F202033D22C2F20002DA6070472F
:100600004FF4C843C4F202034FF47462C2F2000212
:10061000DA6070474FF4C843C4F202030022C2F20A
:100620003D02DA60704700BFCA680B68D0F800C0AE
:100630002DE9F0014F698E69CD690C6A42EA030821
:1006400048EA07073E434B6A35432C4344EA03021A
:100650008C6A42EA04034A6B8C6B48F23F071343EF
:10066000CFF21C0723430CEA07071F4307604469C6
:100670000A6BCB6A24F007041343234343610B69DD
:1006800043604B6883608B68C360BDE8F0017047CE
:100690000023036043608360C3600361436183613F
:1006A000C361036243628362C36203634363836320
:1006B000704700BF036819B923F001030360704756
:1006C00043F0010303607047416070470B060CD58F
:1006D0004369AAB143F08003802943610FD00368C6
:1006E00001F01E01194301607047802907D0002ADC
:1006F000F5D1036801F01E0123EA01010160704792
:1007000023F0800380294361F3D1704770B44FF424
:10071000C04246F20F454FF4C84421F0F023C4F222
:100720000205C4F20204C4F2020223F0C316A84276
:1007300088BF224696B1046804F01E0404EAD1245E
:1007400089004CBF5268126823F0821313EA02003A
:1007500002D0201C18BF012070BC7047446904F00F
:100760008004EDE710B44FF4C84246F20F444FF452
:10077000C043C4F20204C4F20202C4F20203A04263
:100780008CBF1046184611F0005F21F0F02121F0D7
:10079000821114BFC160816010BC704700222DE936
:1007A000F00113460126032703E001330232102B28
:1007B0002CD00D6806FA03F42540A542F5D1D0F8F7
:1007C00000C007FA02F4E44304EA0C0CC0F800C0CD
:1007D00091F804C0D0F800800CFA02FC4CEA080C36
:1007E000C0F800C091F804C00CF1FF3CBCF1010F4F
:1007F0000FD9C5682C40C460CC79C56804FA02F4EE
:1008000001332C430232102BC460D2D1BDE8F00179
:100810007047D0F808C004EA0C0CC0F808C091F882
:1008200005C0D0F808800CFA02FC4CEA080CC0F8AD
:1008300008C0D0F804C02CEA0505456091F806C050
:1008400045680CFA03FC1FFA8CFC4CEA0505456070
:10085000CFE700BF00234FF6FF72026003714371C0
:100860008371C371704700BF036919420CBF002038
:10087000012070470AB9418370470183704700BF68
:10088000CB08083301F0070130B4890050F8235039
:100890000F2404FA01F425EA040440F8234050F838
:1008A000234002FA01F2144340F8234030BC704761
:1008B00008B54FF4A843C4F20003984218D04FF48F
:1008C000B043C4F2000398421ED04FF4B843C4F2C0
:1008D0000003984200D008BD01214FF4000000F051
:1008E00091F94FF400000021BDE8084000F08AB9FA
:1008F00001214FF4001000F085F94FF400100021A1
:10090000BDE8084000F07EB901214FF4800000F0FE
:1009100079F94FF480000021BDE8084000F072B979
:10092000F0B5044685B068460D46A68800F0E8F8A4
:10093000029A4DF68363C4F21B33A3FB021326F025
:100940003F06980C3604360C87B23E43A6802388B7
:1009500023F001031B041B0C238048F2A0612B68C9
:10096000C0F201018B4222D85B00B2FBF3F292B2DB
:1009700001372784032A98BF0422A28323889BB2CD
:1009800043F00103238023886989AA8823F48163C3
:1009900023F002031B040A431B0C13439BB2238066
:1009A0002A89AB8913439BB2238105B0F0BDEE8841
:1009B0004BF6FF718E421DBF03EB830303EB8303F2
:1009C000B2FBF3F203EB43030CBFB2FBF3F242F4CE
:1009D000804292B213051B0D0BB942F001024FF495
:1009E000967344F6D35103FB00F0C1F2620181FB20
:1009F00000318909013142F400422184BDE700BF82
:100A0000002341F28832026083804BF6FF7203813B
:100A100043814FF48043C28083817047038829B9A2
:100A200023F001031B041B0C038070479BB243F0AF
:100A300001030380704700BF038829B923F4807342
:100A40001B041B0C038070479BB243F4807303802C
:100A5000704700BF038829B923F400731B041B0CE3
:100A6000038070479BB243F400730380704700BF5C
:100A70001AB901F0FE010182704741F001010182C3
:100A8000704700BF038829B923F480631B041B0C43
:100A9000038070479BB243F480630380704700BFBC
:100AA000038819B95B045B0C038070476FEA43430A
:100AB0006FEA53439BB20380704700BF01827047C7
:100AC000008AC0B2704700BF82B000230A0F0093B3
:100AD000019301900092009B21F07F4153B1019B53
:100AE00014330193019B1B6819420CBF00200120A5
:100AF00002B07047019B1833090C0193F2E700BF65
:100B000010B44FF46053C4F202039A6802F00C026E
:100B1000042A22D0082A26D04FF41052C0F2F40240
:100B200002604FF46053C4F2020320499C68C4F38E
:100B300003140C5D22FA04F242609C68C4F3822420
:100B40000C5D22FA04F484609B68C3F34233CB5CEF
:100B500022FA03F2C26010BC70474FF49052C0F208
:100B60007A020260DDE75C68596814F4800F5C6803
:100B700015BF4FF490534FF41053C0F27A03C0F2F4
:100B8000F40301F03F01B3FBF1F24FF46053C4F200
:100B90000203C4F388145B68C3F30143013302FB0F
:100BA00004F25B00B2FBF3F20260BAE7000000203F
:100BB0004FF46053C4F202031A6B19B922EA000021
:100BC0001863704710431863704700BF4FF46053B9
:100BD000C4F202031A6C19B922EA000018647047C3
:100BE00010431864704700BF4FF46053C4F202030F
:100BF0005A6C19B922EA00005864704710435864CF
:100C0000704700BF4FF46053C4F202031A6A19B967
:100C100022EA00001862704710431862704700BF54
:100C2000002270B44FF48064C4F201020388C4F25D
:100C30000104904218BFA0429BB214BF00220122BF
:100C400008D04FF48064C4F20004B0F1804F18BFA4
:100C5000A04223D14FF68F754C881D4045EA04030E
:100C60004FF4A0564FF48055C4F20005C4F20006BC
:100C7000B04218BFA8421FBF0D894FF6FF441C4069
:100C800044EA050303804B68C3620B8803850AB1FD
:100C90008B7A03860123838270BC70474FF44065D2
:100CA0004FF40064C4F20005C4F20004A04218BF6F
:100CB000A842D5D1CEE700BF00234FF0FF314160FD
:100CC0000380038143808372704700BF038829B982
:100CD00023F080031B041B0C038070479BB243F07E
:100CE00080030380704700BF038829B923F0010304
:100CF0001B041B0C038070479BB243F0010303806D
:100D0000704700BF038C23F001031B041B0C0384FA
:100D10002DE9F001038C8D8984884F88028BB1F80E
:100D200000C02F4322F07302002523F002034FF48A
:100D3000806612041B04C4F20106C4F20105120C01
:100D40001B0CBFB2A84218BFB042A4B242EA0C02C8
:100D500047EA030316D14FF6F775B1F80EC0B1F8A4
:100D600012800F8A8E881D4045EA0C0C4FF6FB73EB
:100D70004FF6FF4548EA070725400CEA0303BCB2DB
:100D800033432C43848002838A6842630384BDE832
:100D9000F001704700230380438083808360838158
:100DA000C381038243827047038B23F008031B0433
:100DB0001B0C194301837047B0F8443021B95B0420
:100DC0005B0CA0F8443070476FEA43436FEA53432B
:100DD0009BB2A0F84430704783899BB21AB923EACA
:100DE000010181817047194381817047C94389B2EC
:100DF0000182704783899BB21AB923EA010181817C
:100E0000704719438181704770B5038ACA8823F4FB
:100E100040531B041B0C1343038283898A880446B6
:100E200008890D4623F4B0534989024323F00C038B
:100E30001B040A431B0C92B21343A381A38AAA8901
:100E400023F440731B041B0C84B01343A382684635
:100E5000FFF756FE4FF4A0524FF48053C4F2010343
:100E6000C4F201029C4218BF9442A2890CBF039BAA
:100E7000029B12B2002A21DB286803EB830303EBF9
:100E800083038000B3FBF0F148F21F53A089C5F241
:100E9000EB13A3FB0152520900B21601642500288E
:100EA00002FB151213DB12013232A3FB0253C3F310
:100EB000431333439BB2238104B070BD2A6803EB14
:100EC000830303EB83035200B3FBF2F1DCE7D200B0
:100ED0003232A3FB0213C3F342133343EAE700BFEA
:100EE0004FF41652002302600C228380C3800381DA
:100EF00042818381704700BF838929B923F400535D
:100F00001B041B0C838170479BB243F40053838105
:100F1000704700BF838919B95B045B0C83817047FC
:100F20006FEA43436FEA53439BB28381704700BF2C
:100F3000C905C90D818070478088C005C00D704704
:100F400001F01F0310B4C1F342110124A14204FABD
:100F500003F30DD002290DD014302AB9026822EA19
:100F60000303036010BC7047026813430360F9E792
:100F70000C30F2E71030F0E7C1F3421310B401F087
:100F80001F020124012B04FA02F416D0022B0CBF1D
:100F9000028A828A92B2224003880124090A04FA52
:100FA00001F19BB219420CBF00200120002A0CBFA6
:100FB000002000F0010010BC7047828992B22240EC
:100FC000EAE700BF090A012303FA01F1C94389B224
:100FD0000180704770B52A4D2C688CB0002C4BD125
:100FE0006846FFF737FC06A8FFF79AF904200121AD
:100FF000FFF7DEFD10234FF40060C4F202006946E3
:10100000009303238DF804308DF80740FFF7C6FBEB
:1010100001214FF48070FFF7E7FD02A8FFF7A0F968
:101020004FF4803302A80393029404940594FFF7CD
:1010300081F94FF400500126C4F2010006A906947C
:101040008DF81C408DF81D4008940A948DF82C6092
:10105000FFF73EF94FF400502346C4F201000E2181
:101060003246FFF78DF94FF40050C4F201003146CB
:10107000FFF77CF9034B1E6001232B600CB070BDA1
:10108000C4020020586100204FF4005008B5C4F29B
:101090000100FFF7C5F940F2C023C2F200030122AC
:1010A0001A6008BD38B50D4C236805460BB9002001
:1010B00038BD4FF40050C4F201000221FFF7BAF925
:1010C0000028F4D04FF40050C4F20100FFF7AEF94D
:1010D000002328802360012038BD00BFC00200200B
:1010E00030B448F6396301EB4105941EC3F6E303BF
:1010F0000229C1EBC501D8BF144683FB0153D8BFF9
:10110000013AC917C1EB6301201848F21F54D51CDE
:101110000818C5F2EB1484FB02340430D31732EA0A
:10112000220228BF2A46A3EB641100EBA202C3EB04
:10113000E413521842F29340D218C9F2492080FBBE
:1011400002508018D317C3EBA000C0EBC000101AE8
:1011500030BC704770B40646002922D00078F0B148
:1011600000231846F25CA2F13004E4B2092CA2F18B
:1011700041050DD9052DA2F161049CBFA2F13704F0
:10118000E4B205D9052C9ABFA2F15704E4B20024B9
:101190000133DDB204EB0010A94280B2E2D870BC8A
:1011A00070470846FBE700BF0020C4F20200202180
:1011B0000122FFF75FBB00BF0020C4F20200202124
:1011C0000022FFF757BB00BF00B583B06846FFF7AA
:1011D00041FB01200146FFF7EBFC002020220346E3
:1011E0006946C4F20200009201228DF805308DF8A4
:1011F00004208DF806308DF80730FFF7CFFAFFF79F
:10120000DBFF03B000BD00BF00B583B06846FFF749
:1012100021FB04200121FFF7CBFC4FF400600023E9
:101220004FF40052C4F20200694600928DF8043077
:101230008DF80730FFF7B2FA03B000BD4FF400603D
:1012400008B54FF40051C4F20200FFF70DFBD0F1D6
:10125000010038BF002008BDF0B412490A680346F7
:10126000E2B11148114D066811482D680768114810
:101270009D6004681048114D00682D68D8600020FA
:10128000072C08BF04465D60013F06F164059C61C0
:101290000F245D611F6118621C6008601046F0BC7D
:1012A000704700BFF0020020C8020020F8020020B2
:1012B00000030020DC020020CC020020D402002029
:1012C000F0B583B068464FF40065FFF7C3FAC4F287
:1012D000020504200121FFF76BFC00244FF400639A
:1012E0006946284600938DF805408DF804408DF836
:1012F0000740FFF753FA6846FFF7ACFA04200121D4
:10130000FFF756FC4FF480570126284669460097A0
:101310008DF805408DF804608DF806408DF8074083
:10132000FFF73CFA284639463246FFF7A3FA03B0E6
:10133000F0BD00BFF8B5A44C2368FF2B56D04FF486
:101340000060C4F202004FF40061FFF78DFA054619
:10135000002833D0FFF728FF23689B4D0120012B85
:1013600033D04AD3022B4DD0984B1A68904200F0EC
:101370008680974E186033689A1F0221122A2960CE
:1013800063D9052B94BF93489348944F06F08CFF84
:10139000934806F089FF002323603B680F2B00F081
:1013A000CC81102B6ED0FF2B3AD001333B2B3B600E
:1013B00000F0CE8134D90023236031E0FFF7FCFE3A
:1013C0002368012B2846804DCBD1804B1A6882427E
:1013D00029D01860814BFF221A607D4B002814BF72
:1013E00003200220002220601A60F8BD7D4B1A689D
:1013F000642A19D001321A60F8BD01232B60734BA7
:101400001860F8BD714B1A68904238D0704E186061
:1014100033680322782B2A6012D9704B00221A609D
:1014200000233360F8BDF8BD4FF40060C4F2020041
:101430004FF480510022FFF71DFA00232360F8BD0E
:101440004A2BEDD800232B60EAE7644F0F2B3B6853
:1014500034D8232B00F097813A2B00F085811C2B88
:101460009CD1614A1268D0079FD5604806F01CFFE6
:101470005B4806F019FF002323603B688EE7544B5E
:101480001A68B7E75A4A002313605A4A1360564A4B
:101490001360594A1360594A1360594A1360594AF4
:1014A0001360594A1360594A1360594A1360594AE4
:1014B0001360594A136011233B60B1E7A3F1110295
:1014C000292A3FF66BAF01A151F822F0331700082B
:1014D0009D1300089D1300089D1300082D17000898
:1014E00027170008211700081B1700081517000808
:1014F0000F17000809170008F9160008F31600086E
:10150000ED160008E7160008E1160008DB160008D3
:10151000D5160008C5160008BF160008B916000841
:10152000B3160008AF160008AB160008A71600088F
:10153000A11600089B160008951600088F160008D3
:1015400089160008831600087F1600087B1600081D
:1015500069160008571600084516000833160008DB
:1015600021160008B7150008A515000893150008F6
:1015700075150008214A126812F001057FF415AFB5
:10158000264806F091FE164806F08EFE25603B6860
:1015900004E72149194A0D681068503501300D6083
:1015A0001060FEE61C49154A0D68106828350130A8
:1015B0000D601060F5E61849104A0D681068143582
:1015C00001300D601060ECE630000020E0020020E9
:1015D000F402002078BF000898BF00082C0000200B
:1015E000ACE10008FC020020D0020020B8BF0008D7
:1015F000F0020020E802002004030020D8020020AE
:10160000EC020020D4020020F8020020DC020020BE
:10161000CC02002000030020C802002000C0000807
:101620006549664A0D6810680A3501300D60106022
:10163000B7E66149614A0D681068083501300D60F0
:101640001060AEE65C495D4A0D68106804350130F3
:101650000D601060A5E65849584A0D6810680235BB
:1016600001300D6010609CE65349544A0D681068C3
:10167000013501300D60106093E65149D1E75049C2
:10168000D8E74F494D4ADFE74D494C4AE5E74C4919
:101690004A4AEBE74B49494AD6E74A49474ADCE719
:1016A0004849464AE2E7484986E74749B9E7464993
:1016B000C0E74549414AC7E74349404ACDE7424967
:1016C0003E4AD3E7414A126812F001057FF46DAE3D
:1016D0003F4856E73F493D4A6FE73E493B4AA1E74D
:1016E0003C493A4AA7E73B49384AADE73949374AC6
:1016F000B3E73849354AB9E7374A126812F00105AD
:101700007FF453AE35483CE73549334A4CE734491A
:10171000314A52E73249304A84E731492E4A8AE752
:101720002F492D4A90E72E492B4A96E72C492A4A01
:101730009CE72C4A0121116033E62B4B1A6822B139
:101740002A4A0121116000221A6010233B6067E6DB
:10175000274B204A196812689142264922D0204816
:1017600000681A6008605BE6144A1268D2077FF5C9
:101770001CAE214806F098FD204806F095FD002299
:101780003B682A600AE6114A1268D1077FF50DAE60
:101790000F4806F089FD194806F086FD00232B60EE
:1017A0003B68FBE50E480C68006801348442D8D1E0
:1017B0000D4C01252560D4E7C8020020D802002086
:1017C00000030020DC020020CC02002004030020E3
:1017D000DCBF0008F8020020D0020020B8BF0008DB
:1017E000D4020020EC020020E8020020F0020020D9
:1017F00008030020E402002000C00008ACE100085B
:10180000034B1A6812B11A68013A1A60704700BF98
:101810005C610020064B074A1B68012B1EBF064B6C
:101820001B68B0FBF3F010601368002BFCD170470D
:101830000C0300205C61002038000020044B054AA6
:101840001B6803FB00F010601368002BFCD170478D
:10185000340000205C610020084B094A1B684FF4EB
:101860007A7110F1FF3001FB03F106D311601368A8
:10187000002BFCD110F1FF30F8D27047340000206B
:101880005C610020012810B423D002282CD01C4B0E
:1018900064221A601B4B0A221A6042F21071032064
:1018A000194B1C684EF21003CEF200034FF46D4248
:1018B000B4FBF1F1CEF2000201395960F02182F857
:1018C000231000229A6007221A60104B186010BC87
:1018D00070470B4B18600B4B44F240214FF47A7267
:1018E0001A60C0F20F01DBE7054B0A221A60054BB4
:1018F00048F2A06164221A60C0F20101D0E700BF83
:101900003800002034000020D80100200C03002003
:101910002DE9F00140F2681040F2A41540F2741174
:10192000C2F20000C2F20001C2F2000540F26414EB
:1019300040F27C0240F28003C2F20002C2F20003D5
:1019400090F8008090F801C087780E7848782D686C
:10195000897882F80080C2F2000482F801C0256014
:1019600097701E7058709970BDE8F001704700BF05
:1019700040F2211009F0AAB840F2851009F0A6B88B
:10198000F8B506460F4640F2211440F28515204670
:101990003146013409F03AF9AC42F8D107B9F8BD43
:1019A000BDE8F840FFF7E8BF30B540F28002C2F270
:1019B00000024CF22443C0F6000311789478557865
:1019C00033F8111033F8152033F8143083B08DF844
:1019D0000410014601A88DF805208DF80630FFF7A8
:1019E000CFFF03B030BD00BF00B583B00023014678
:1019F00001A88DF804308DF805308DF80630FFF71A
:101A0000BFFF03B000BD00BF0E2A30B436D81F4B55
:101A10000C789B5C48F6890213FB04F4C8F6880234
:101A2000A2FB0452C2F3C70202700C7814B10AB9C7
:101A3000012202704C7848F6890213FB04F4C8F6C0
:101A40008802A2FB0452C2F3C70242704C7814B160
:101A50000AB9012242708C7848F6890213FB04F31C
:101A6000C8F68802A2FB0342C2F3C70282708B78D9
:101A700013B10AB90123837030BC70470B7803702F
:101A80004B7843708B788370F6E700BFA4C40008DE
:101A900010B5104B104C1A68104982B02046FFF761
:101AA000B3FF0F4B1B689BB10E4B2178A078627877
:101AB00033F8111033F8122033F810308DF8041079
:101AC00001A801218DF805208DF80630FFF758FF99
:101AD00002B010BD64010020800000207C000020C6
:101AE0007001002024C400080E4B1B68032B18D87B
:101AF000DFE803F013100A020B4B00223F2119709C
:101B00005A709A70FFF7C4BF084B012200201A6078
:101B1000FFF76ABF0020FFF767BF054B1868FFF7A4
:101B200043BF7047280400207C0000205C04002094
:101B30007001002030B5244B1B688DB0002B22D0E3
:101B4000224D00242A462346116911F0020F02F1AA
:101B5000140205D00CA800EB8401013441F82C3CA0
:101B600001330B2BF0D1002C1FD1194A23461460EE
:101B700003EB830305EB83056B689847154B002245
:101B80001A600DB030BD124A10481168114A01EBBD
:101B9000810100EB8100116884680131A14211606C
:101BA000EFD3416813608847EBE709F027FCB0FBEF
:101BB000F4F30CAA03FB140002EB8003044A53F86D
:101BC0002C3C1360D4E700BF58040020880000209C
:101BD000840300208C0300202DE9F00F0B0682B057
:101BE0004BD46FEA020ADFF808C1404B0AF1090A38
:101BF000072A88BF4FF0000A00F10806C2F1070863
:101C0000042703EBC10B8244CDF80480B61A0124EB
:101C1000ACF14805072A16D801990BEB07090346D2
:101C2000112B0CD819F8048C48FA01F818F0010FA0
:101C30001ABF4FF004080CF803800CF8034001337E
:101C40000139B342ECD1BAF1110F9FBF07EBC708BE
:101C5000534651464FEA480801D905E01946414428
:101C60000133112B6C54F9D901370C2F0CF1120CE4
:101C7000D0D102B0BDE8F00F7047B0394C2932D84E
:101C8000DFE801F02F313131313131313131313152
:101C900031313131313131312D3131313131313138
:101CA000313131313131313131312B31313131312A
:101CB00029313127313131312D313131313131312A
:101CC000313131313131313131312B31313131310A
:101CD0002900052185E7042183E7032181E702210B
:101CE0007FE701217DE720217BE700BF24C00008BA
:101CF000AC610020B0F5907F10D248F63963C3F68E
:101D0000E303A3FB00239B08DA0742BF03EBC303F3
:101D1000C0EB83001130013008F078BF704700BF7E
:101D200070B5294B1A6882B006460AB901261E60B2
:101D3000264A274B11785478907833F8111033F8ED
:101D4000142033F81030234D8DF8001000248DF846
:101D500001208DF802308DF804408DF805408DF893
:101D600006400BE0FFF7C6FF15F8013C013443F0D5
:101D70000103B4F5907F05F8013C16D015F8013B3E
:101D800003F00203DBB220466946002BEAD120466D
:101D900001A9FFF7AFFF15F8013C013423F001035F
:101DA000B4F5907F05F8013CE8D116B10A4B1B68E9
:101DB00033B1FFF7DDFD094B01221A6002B070BD9F
:101DC0000120FFF7F1FDF6E7400400207401002038
:101DD00024C4000864610020280400206061002001
:101DE00008B5064B1A6822B1002210461A60FFF7A8
:101DF00097FF034B01221A6008BD00BF5804002062
:101E00006061002008B50D4B0D481A680D49FFF7B9
:101E1000FBFD0D4B1B68032B03D00C4B1B68990774
:101E200008D40B4B1B6803B908BD0120BDE808406E
:101E3000FFF776BFFFF76CFDF3E700BFA4010020BA
:101E40007401002068010020280400208400002084
:101E5000700100202DE9F041864B1A6884B03AB930
:101E600085490B68002B00F0E48004B0BDE8F081E8
:101E7000824A81491678DFF81C824CF6CD40CCF6B8
:101E8000CC40A0FB0650002400091C600C6000F050
:101E9000B580C8F800005578DFF8FCC14CF6CD439A
:101EA000CCF6CC43A3FB05031B0902D1002D40F067
:101EB000BE80CCF800309478714F4CF6CD43CCF610
:101EC000CC43A3FB04231B0902D1002C40F0AD80BE
:101ED0006C4A3B606C4B00201070507090701E700C
:101EE0005D709C70D8F800301C4693B1664A147837
:101EF000A34240F2968014B1002010700124614A80
:101F00005E4815780078EB18834200F2A2801370C7
:101F10000124DCF800308BB15B48427893427CD9D5
:101F200012B1002242700124564A54485578407834
:101F3000EB18834200F29280537001243868002825
:101F400063D0514B9A78904263D912B100229A70B3
:101F500001244C4D494AAF7896783818B0429CBF5E
:101F6000C0B2A87003D9B7424FD0AE7030464749CF
:101F700092F800C092F801E06C782F785A781D78BA
:101F80009B7831F81C8031F8177031F81EC031F899
:101F9000122031F816E031F8133031F8146031F8BE
:101FA000104031F815008DF80A40394D8DF8048045
:101FB0008DF805C08DF806E08DF808708DF8096081
:101FC0008DF80C008DF80D208DF80E30002407E000
:101FD000012B34D0032B37D00134B4F5907F0AD0D5
:101FE000635D022BF4D1204602A90134FFF782FE83
:101FF000B4F5907FF4D1FFF7BBFC36E7002E3FF439
:1020000048AF0123C8F8003045E764BB01230B60EB
:102010002BE7121A9A7001249BE7D21A427001240E
:1020200082E7E41A1470012469E7012350E70123D1
:102030003FE7DFF86080DFF860C0114F52E72046CD
:1020400003A9FFF757FEC7E7204601A9FFF752FE95
:10205000C2E785421CBF107001245AE785421CBFAD
:10206000507001246AE7054A064D9678A878064B19
:102070007DE700BF5804002060610020740100204B
:1020800078040020A80300208003002024C4000856
:1020900064610020C0030020A003002070B5154A31
:1020A000154B94781178557833F8111033F81520C2
:1020B00033F81430114E82B000248DF8001005461C
:1020C0008DF801208DF802308DF804408DF8054020
:1020D0008DF80640A35D2B42204601A918BF694632
:1020E0000134FFF707FEB4F5907FF3D1FFF740FC12
:1020F00002B070BD7401002024C400086461002097
:102100002DE9F8435A4B5B4D1A682AB92E68002E08
:1021100000F09980BDE8F883DFF8608100221A6042
:102120002A60C8F80020544C4FF0000E7646A446B2
:102130000EEBCE00400012230CEB00095A1E811852
:102140006718615C11F0010F45D0112A00EB0306FE
:102150004AD01CF80660F60741D421F0010139701D
:10216000002A46D0023B0126002BE7D10EF1010EDA
:10217000BEF1100FDCD10120FFF790FF002E5ED0E2
:10218000D8F800300126012B08BF3B4CC2D13A4F92
:102190004FF0000EB8460EEBCE004000002308EBD7
:1021A000000CC21804EB0209A25C02F0060102292D
:1021B00026D00133112BF4D90EF1010E1237BEF1E6
:1021C000100FE8D10420FFF769FF002EA2D10123F0
:1021D0002B60BDE8F8831346002BAFD1C6E713464A
:1021E0000126002BAAD1C1E721F0010189F81110C5
:1021F000B8E70EF1010E0126BEF1100F98D1BAE733
:1022000043B302F00401C9B20029D2D142F0040262
:10221000112B89F8002022D00133C218A25C02F0F1
:102220000202D2B24AB1112B03F1010317D0FA5CBA
:1022300002F00202D2B2002AF5D10126BAE7012348
:10224000C8F80030A3E7DFF83480D8F80030002B5E
:1022500099D168E742F004028CF80020DCE70EF127
:10226000010E01261237BEF1100F94D1AAE700BF6C
:1022700058040020606100206461002034040020C4
:102280002DE9F00F6A4B1A6832B96A4A1368002BBD
:1022900067D0BDE8F00F704700201860654A664EB1
:1022A000664B106001213160196033688BB164485E
:1022B00010256C1E0023C25C02F00301012936D0F8
:1022C0000133122BF7D112382546002CF1D134609E
:1022D0003FE0DFF868A1DAF8001000293ED0DFF80F
:1022E00074B1DBF80020002A3DD0564D564A2968CB
:1022F0001068564A564E01EBC10400EB440401310C
:10230000175D296027F0040701EBC10500EB4500CC
:1023100017553668145CB14244F0040508BF44F018
:102320000504155404BFCBF80030145411E004EB3D
:10233000C400464903EB400022F001020F2C0A546E
:1023400007D005EBC50503EB4503CA5C42F001026B
:10235000CA540520BDE8F00FFFF7A0BE01231360AB
:1023600097E7354EA1E740F2A431C2F2000140F2F6
:102370007C330F68324840F26431C2F20003C2F28B
:102380000001D3F80090D1F8008094461026A0F503
:102390008775741ED30748D40023C25C02F0030182
:1023A000022905D00133122BF7D14B46002210E051
:1023B000A4B112F0010216D006EBC60203EB4202F2
:1023C000B046A95C41F00401A9544FF0010C274626
:1023D0000122264612388CB19946DAE7EA5C42F0CF
:1023E0000502EA54F3E7BCF1000FF0D1E95C41F0DB
:1023F0000401E9544FF0010C9046E8E740F2A431A3
:10240000C2F20001CBF800C00F6040F27C31C2F292
:1024100000010B6040F26433C2F20003C3F8008095
:10242000002A96D1CAF8002093E74B46D1E700BFB7
:1024300058040020606100204C0400209803002014
:1024400072620020640300207C030020646100208D
:10245000A40300201C0400202DE9F843694B1A68EE
:1024600032B9694D2B68002B00F0A180BDE8F883DC
:1024700000201860654C644B206018604FEAC00C67
:102480000CEB00035B00624A1918C0F112061546F6
:10249000F3188A18EF18A8461346197841F004017A
:1024A00003F8011BBB42F8D1C0F10F0E431C73456A
:1024B00028BF4FEACE0C1BD20CEB0007C0F1110372
:1024C00000EB08014FEACE0C03EB470312390CEB8B
:1024D0000E075B1901EB4707917C41F0040102F8FC
:1024E000121F997CBA4241F0040103F8121FF3D184
:1024F0000CEB0E0205EB42020346D15C41F00401F5
:10250000D1540133B342F8D3002848D0421EC0F161
:102510001307BA420FD202EBC20149000B185B1934
:102520007E19013B761813F8011B21F00401B34218
:1025300003F8011CF7D1C0F11008404528BF4FEA4D
:10254000C8091DD200EBC0034FEAC80902EB4303E0
:10255000511909EB080CC0F112065B1901EB4C0C88
:1025600093F800E0991A2EF0040E83F800E011F8B9
:1025700006E012332EF0040E634501F806E0EFD1B9
:1025800009EB080300EB43035B19013B13F8011B44
:10259000013221F00401BA4203F8011CF6D30420F1
:1025A000FFF77CFD236801332360BDE8F883174CF7
:1025B000206807287FF662AF08281CBF144B03F57C
:1025C000907404D119E0A34203F8010C0ED013F863
:1025D000012B02F00201C9B242F0040022F0040211
:1025E0000029F0D1A34203F8012CF0D10420FFF719
:1025F00055FD01232B60BDE8F88307220B27044D0E
:1026000089E700BF58040020606100207C0400209E
:102610006461002070B5264A264813681BB9036818
:10262000002B3BD070BD00231360234D234A036071
:102630002B6013602E6886B9214B03F590711A78D0
:1026400022F0040203F8012B8B42F8D10420FFF79B
:1026500025FD2B6801332B6070BD184A13680133C8
:102660001360DA07DED5741EA4B2B4F5907F10D2E1
:1026700013490B5D03F00202D2B22AB110E00B5DE8
:1026800003F00202D2B25AB90134A4B2B4F5907F79
:10269000F5D10123036001362E6070BD064DC9E7F8
:1026A00043F0040304200B55661CFFF7F7FCF2E728
:1026B0005804002060610020B4030020240400209E
:1026C000646100202DE9F00F8D4A136886B043B98C
:1026D0008C4B1A68002A00F0098106B0BDE8F00FA3
:1026E000704700231360884C864A2360136003936D
:1026F000864F002000EBC00207EB42020023117856
:10270000013321F00401122B02F8011BF7D1013033
:102710001028EFD1039B03F10109C3F10806C4F8A7
:10272000009001960020C21900231178013321F096
:102730000801122B02F8011BF7D11230B0F5907F7F
:10274000F1D1019A714DCDF80890534293469A46C3
:1027500000269946BAF1080F2CBFD0464FF0080862
:102760004A4601990023BBF1070F34BFDC464FF006
:10277000070C17E0082934BF08460820082B6446D8
:1027800003D9092A2CBF1046092004EBC40400EB2E
:1027900044003C5C44F008043C54013301310132F4
:1027A000122B15D0E85C00F00200C0B20028F4D073
:1027B000072EDFD9082B05D8082934BF0846082082
:1027C0004446E2E7082A8CBF104609204446DCE76D
:1027D00001361235102E0AF1010A0BF1010BB9D1A5
:1027E000039EDDF80CB0DDF80890002301936FF034
:1027F000110303FB067302936FF0120C6FF02303B7
:102800005A460CFB06FCD24303FB06F60596CA4665
:102810004FF000080492039E049B0BEBCB056D0068
:10282000AA19019EED18F119D219ED194C46002391
:102830001DE0082B2ED8C14509D8994507D8059E1B
:10284000A81910F8126C46F0040600F8126C11F882
:10285000010B00F00806F6B21EB140F0040001F8CA
:10286000010C0133013201350134122B29D012F849
:102870000C00C007EBD5B8F1070FDAD9082B16D832
:10288000BAF10F0FE3D89945E1D8A87C40F00400D5
:10289000A874DCE7C145DAD8112CD8D8029E3019CB
:1028A00010F8126C46F0040600F8126CCFE7BAF18B
:1028B0000F0FCCD8112C9EBFD07C40F00400D074F8
:1028C000C5E7019A029B08F1010812321233B8F1F0
:1028D000100F01920BF1010B02930AF1010A9AD138
:1028E000042006B0BDE8F00FFFF7D8BB064C226805
:1028F000082A03927FF6FCAE01221A60EDE600BFC3
:1029000058040020606100207404002064610020ED
:102910002DE9F84FA94C2368002B40F0A880A84B64
:102920001B68032B12D8DFE803F0764613022368F6
:10293000002B40F0CA80A34A13683BB9A2490B6838
:10294000B3F5907FC0F0C88001231360BDE8F88F15
:102950002368002B00F0A18098499C4B00220A605C
:1029600098491A600A609A4C02F1120504F11208A3
:102970001D600021C2EB08088B1A1B1908EB01002F
:102980000DE013F8126C16F0010F9E5C00F0088148
:1029900046F004069E540133984200F008818D42AF
:1029A000EFD993F80E6106F00206F6B2002E00F0A1
:1029B000F6809E5CECE72368002B79D07F49854A3E
:1029C00000230B607F4913600B605F1C804C176015
:1029D0001E4603F5907C594203F1130033193A4621
:1029E0000DE05D7815F0010F5D5C00F0CB8045F0E7
:1029F000040501325D540133824200F0CB80112A7C
:102A0000EFD913F8115C05F00205EDB2002D00F0CE
:102A1000B8805D5CEBE72368002B33D0674A6E4BD0
:102A200000211160674A19601160481C684C1860E9
:102A30004E42C1F59077331900220EE013F8015C85
:102A400015F0010F5D5C00F08F8045F00405013248
:102A50005D540133122A00F08F809042EED95D7CE4
:102A600005F00205EDB2002D7DD05D5CEDE708F0CC
:102A7000C5FCC3179B0FC21802F00302D31A504AB9
:102A800013604EE74F4A1368002B7FF45FAF524B41
:102A9000196811293FF658AFC7E74A490B68002B60
:102AA0007FF454AF494B1A68B2F5907F09D25AE7C8
:102AB00044490B68002B7FF449AF464A1368112B39
:102AC00083D901230B60BDE8F88F3C4A3E490023BF
:102AD00013603C4A0B6013603D4C4FF6EE7A03F1F5
:102AE0001202CFF6FF7A0A6003F5997B04F112080F
:102AF000C3EB0A0A40F21F16A2F590710AEB02001E
:102B00000919131902EB080510E091F82071C2EBC6
:102B10000309FF07CC4614D519F80070013347F0BC
:102B200004070131AB4209F8007014D0B242ECD96D
:102B30000F7807F00207C2EB030CFFB2E146002F4B
:102B4000EAD11CF80070013327F004070131AB42D1
:102B50000CF80070EAD112325A45CDD10420BDE8FC
:102B6000F84FFFF79BBA5D5C25F0040501325D5418
:102B70000133122A7FF471AF1236BE427FF45BAF8D
:102B8000ECE75D5C25F0040501325D5401338242BF
:102B90007FF435AF123666457FF420AFDEE79E5CEA
:102BA00026F004069E54013398427FF4F8AE1231A9
:102BB000B1F5907F7FF4E0AED0E700BF580400206D
:102BC000BC030020606100203004002010040020BD
:102BD0006461002014040020800400202DE9F04FDF
:102BE000B24AB34E136885B033B93368002B00F096
:102BF000968005B0BDE8F08F00231360AD4AAE4C5F
:102C00001360AE4AAE4D1360AE4A336023602B6052
:102C100013602368002B43D1AB4A11781F295FD979
:102C200051781F2900F2C6803F228DF808308DF8B8
:102C300009208DF80A30A54B9E4F1A6803A802A9F7
:102C4000FEF7E2FEA2492E689DF80C809DF80DC0AB
:102C50009DF80EE09F4B38689F4A31F8188031F894
:102C60001CC031F81EE083F8008006EBC60100EBC3
:102C700041000026194683F801C083F802E016706F
:102C800056709670FFF736F823682968934A3868BB
:102C9000D15493495A1CC8542260FEF769FEA8E734
:102CA0002A681C2A24D98F4B03F5907403E0A342B1
:102CB00003F8010C0ED013F8012B02F00201C9B287
:102CC00042F0040022F004020029F0D1A34203F8EC
:102CD000012CF0D10420FFF7E1F90123336088E7EC
:102CE0003F228DF808208DF809308DF80A30A2E7D0
:102CF000DFF8C8E16F4FDEF80030D7F800C09A4225
:102D000077D0704B1B6802F00109B9F1000F4AD16E
:102D100063452DD90CF101033B602A682FE0664C16
:102D2000674D76E7BBF1110F19D85B4608EBC80079
:102D300046F2641C03EB4000C2F2000C1CF800C019
:102D40001CF0010FDDF800C004D0E0E0C85CC00753
:102D500000F1DD800133122BF8D1CDF800C008F16D
:102D600001081231B8F1100F65D11D23CEF80030E3
:102D7000DEF800309A4228D301232A6833600F2AF4
:102D80002ED92368DFF854810D2B78D0544E296852
:102D90003A6808F803100C2BF25401D80133236071
:102DA000FEF7E6FD25E76345E2D20CF1FF333B6019
:102DB0002A68E4E792781F2A0AD88DF808308DF83F
:102DC00009303F238DF80A3035E701322A60D6E713
:102DD0003F228DF808308DF809208DF80A202AE767
:102DE00038683C4902EBC20200EB4200FEF782FF6A
:102DF000C7E740F29030C2F2000003689C4582D1E0
:102E000012F0010900F08B800CF1FF3B9246BCF1FF
:102E1000000F02D102F1010AE346BAF10F0FA4D864
:102E200046F264130AEBCA01C2F2000303EB41014C
:102E3000D046CDF800C0D0455FD018F001033FF474
:102E400075AF112308EBC80046F2641CC2F2000CF7
:102E500003EB40001CF80000DDF800C0C00706D4FA
:102E6000002B3FF47AAF013BC85CC007F8D540F2B5
:102E70009030C2F20000CEF80080036045E798F879
:102E80000030174E0F2B2FD90023013308EB03021C
:102E900018F80300F15C02F8010CF2180C2B02F890
:102EA000011CF2D12368013B236070E75804002025
:102EB00060610020380400200C0400209C030020E6
:102EC000480400209003002068010020A401002095
:102ED00024C40008540400202004002060040020C2
:102EE00068030020646100203078114903EBC303BC
:102EF00000EB4300FEF7FEFEC6E718F0010F3FF4BB
:102F000011AFBBF1FF3F18BF5B469BD127E740F2F3
:102F10009031C2F20001CEF800800B60F5E6BCF102
:102F2000100F9CBF0CF1010B92467FF676AF71E754
:102F3000200400202DE9F04F804B814C1A6885B0A9
:102F4000002A40F098802368002B57D1DFF808B2A0
:102F5000DBF800202F2A54D8DFF8F0A1DFF8F48145
:102F60009AF800009AF801109AF802208DF80C00E7
:102F70008DF80D108DF80E20994658F8044B182C3A
:102F80002DD9A4F11805012D63D0A4F11A030F2B3C
:102F900067D90F2D5DD904EBC407193CA9F5EA7375
:102FA0000126A51E0F2C03EB470709D90E2D45D985
:102FB0000136243F6B1C2C460FD0A51E0F2CF5D8D4
:102FC0009AF8013007F11200B3FBF6F303A98DF86C
:102FD0000D30FEF78FFE002CE8D158F8044C09F1B3
:102FE00001090134B9F1120F48F8044CC5D1FEF7BC
:102FF000BFFCDBF800300133CBF8003005B0BDE892
:10300000F08F504B03F5907503E0AB4203F8010CD1
:103010000ED013F8012B02F00201C9B242F00400F5
:1030200022F004020029F0D1AB4203F8012CF0D1C8
:103030000420FFF733F801232360DFE79AF801301B
:103040003846B3FBF6F303A98DF80D30FEF752FEB8
:10305000AEE705EBC50009EB40003B49FEF74AFE31
:1030600099E705EBC500A9F1240303EB40003749BC
:10307000FEF740FE8DE7364A364FD2F80080002634
:103080001E60354B26603F25424602A869461E60F9
:1030900010238DF806308DF800508DF801508DF812
:1030A00005508DF802608DF80460FEF7ADFC4246D5
:1030B00003A801A9FEF7A8FC284B9DF808809DF8FD
:1030C00009C09DF80AE09DF80C509DF80D009DF890
:1030D0000E901D491D4A33F8155033F8188033F807
:1030E0001CC033F81EE033F8100033F819301570A7
:1030F00081F8008081F801C081F802E0507093707F
:1031000035460DE008F07AF9C3171B0FC01800F020
:103110000F00C31ABB5101350436122D3FF413AF13
:10312000EA07EFD408F06AF9C3171B0FC01800F0C4
:103130000F00C31A0833BB51EDE700BF580400204D
:1031400060610020646100202C040020AC0300209A
:10315000A4010020C40300205004002024C400085F
:1031600010B582B0002914BFFF230023002814BF2C
:10317000FF240024002A14BFFF220022002001A9FE
:103180008DF804408DF805308DF8062007F03EFDDF
:10319000012007F09BFC02B010BD00BF074B0120CF
:1031A00003F5907113F8012B12F0020214BF03F81B
:1031B000010C03F8012C8B42F4D1704764610020AC
:1031C0002DE9F84F1746814688460AB9BDE8F88FC1
:1031D0000020FEF7A5FD39077FD4FA0679D44B4AC3
:1031E0004B4B126803EBC20113F832B091F801A007
:1031F0007B07EBD5474E48484B22002107F069FE7C
:1032000006F590750122334613F8014B14F00204C1
:1032100014BF03F8012C03F8014CAB42F4D13F4B2F
:103220001B68002B67D03E4B1B68D80767D53A4B0D
:1032300001225A709A703B4B374CCBEB0B1B08EBBF
:103240008B0103EBC10101200023CA18013352781E
:1032500012B1072BA054F8D10B782F4C9944B9F137
:10326000180F0AEB8A0A88BFA9F119092E4B0AEB3D
:103270008A0A0AEB090003EB800001210023C25CEB
:10328000013312B1042BA154F9D1284CDFF8A8C0A6
:1032900004F14B07002514F8013F93B105EB0C0333
:1032A00015F80C2098785B7858B102EBC202181818
:1032B00006EB4202D15C41F00201D154013383425A
:1032C000F8D10335BC42E6D1194B01221A60BDE8A2
:1032D000F88F0120FEF788FB81E706F08BFDC82000
:1032E000FEF7ACFA134B1B68002B7FF478AF01207C
:1032F000FEF75AFB73E7F9067FF568AFE4E7B8F12C
:10330000000F18BFB8F11E0F95D190E7B803002049
:10331000DCDE000864610020100300207001002042
:103320008400002028C50008C8D900080F03002029
:103330005804002028040020F8DD000840F284032F
:10334000C2F200031868704738B50B4B0B4D1B6871
:10335000032B044604D0830702D52B68980707D5B2
:10336000FEF7C2FB064B2C6001221A60204638BDD6
:10337000FEF7CEFAF4E700BF280400208400002006
:103380005804002040F22843C2F200031868704736
:10339000032810B509D8074C2368834203D0206066
:1033A000FEF7A2FB2368184610BD024B1B681846A7
:1033B00010BD00BF2804002040F27813C2F20003C1
:1033C000186870476328024B88BF642018607047F4
:1033D0007801002040F2A813C2F200031868704779
:1033E0006228024B88BF002018607047A8010020A7
:1033F00040F2B833C2F20003186870471128044B3A
:1034000004D81860034B01221A607047186870478F
:10341000B803002058040020064B1868102805D96E
:1034200000201860044B01221A60704701301860B8
:10343000F8E700BFB803002058040020054B1868C7
:1034400028B101381860044B01221A60704711201E
:103450001860F8E7B80300205804002040F23C430D
:10346000C2F2000318687047074B10B5186000B12E
:1034700010BD064B0F241C60FEF7C4FC044B1C60FF
:10348000BDE81040FEF704BB3C040020A40100206E
:103490006401002040F2A013C2F2000318687047D4
:1034A000024B0A288CBF186818607047A0010020E2
:1034B000044B1868092802D90020186070470130B1
:1034C00018607047A0010020044B186810B1013843
:1034D000186070470A201860704700BFA0010020E4
:1034E000064B1B68012B00D07047054B00223F2183
:1034F00019705A709A70FEF785BC00BF180400203E
:103500006801002040F21843C2F2000318687047B7
:10351000012810B5034602D9054B186810BD044CAC
:103520002068984203D02360FFF7DAFF206810BDBF
:1035300018040020F0B5584B1B68012B83B00446DB
:1035400042D0022B01D003B0F0BD20B9534B1A6812
:10355000002A7AD018600020FEF746FA504B1B680C
:103560003B2B2ED81D2B73D967081E254D4A4E4B79
:1035700010785178927833F8100033F8111033F83E
:103580001220464B8DF804001B688DF805108DF84D
:103590000620002B46D1AF423CBF444E3C4606D3EA
:1035A00039E000F2211007F031FBAC4233D2306831
:1035B00020180134A84201A9F3D33C386328F4D879
:1035C000EFE727463C25D1E70020FEF70DFA344B04
:1035D0001B683B2B48D9354B1A683C23A418314A49
:1035E000A34298BFC3EB040411782F4B9078557811
:1035F00033F8111033F8152033F810308DF804101B
:10360000632C8DF805208DF8063004D804F22110C3
:1036100001A907F0FBFA264B1B68002B93D0FEF79D
:10362000ABF990E7214E002405E000F2211007F0ED
:10363000EDFABC42EFD83368E0180134A84201A982
:10364000F3D33C386328F4D8EFE701221A6082E70D
:10365000132B7FF678AF4AF6AB27CAF6AA27A7FB4B
:1036600004377F08142581E71D2B0ED8132B7FF616
:103670006AAF0E4A4AF6AB23CAF6AA231268A3FB26
:10368000041402EB54041423A9E7084B1A681E2300
:1036900002EB5404A3E700BF280400205C040020D0
:1036A000780100208000002024C40008A801002028
:1036B0007001002038B5874B1B680A2B1DD8864A3D
:1036C000864C126892B9864D2A68DAB9042B00F04C
:1036D000E2808449844A03EB830301EB830311688E
:1036E000986801318142116045D238BD7D4A03EBB3
:1036F000830302EB83035B689847794B1B68002BBD
:10370000F3D0764C794B1B68012B1FD0784B1B688C
:10371000032B06D02368002BE7D1BDE8384006F024
:1037200087BB744B74491A68496B0132B2EB411F75
:103730001A60EFD371490A680020013A1860052A1F
:103740003AD8DFE802F050A19A938C856C4B6D4912
:103750001A6849690132B2EB411F1A60D6D36A492F
:103760000A680020013A1860052A0CD8DFE802F048
:1037700069625B544D4400215B68116098472B6877
:10378000002BBED1B1E7614A13680133072B00F06B
:103790009E805F48136002680B6001320D2A5A490F
:1037A000026000F08B800E2AB0D1013B08BF0623D7
:1037B0000B6000230360A9E7564A13680133072B07
:1037C0007AD05548136002680B6001320D2A4B49CC
:1037D000026068D00E2A9DD1013B08BF06230B6012
:1037E0000023036096E74D4B5A783E2AE4D8013215
:1037F0005A70FEF74DF98DE7494B9A78002AC2D0EE
:10380000013A9A70FEF7FEFA80E7454B1A783E2A95
:10381000B9D801321A70F5E7414B5A78002AB2D074
:10382000013A5A70EEE73E4B9A783E2AABD8013205
:103830009A70E7E73A4B1A78002AA4D0013A1A7036
:10384000E0E7374B5A783E2A9DD801325A70D9E7C3
:10385000324B9A78002AAFD0013A9A70C9E72F4BC1
:103860001A783E2AA8D801321A70C2E72B4B5A7830
:10387000002AA1D0013A5A70BBE7284B9A783E2A19
:103880009AD801329A70B4E7244B1A78002A93D060
:10389000013A1A70ADE7134B5B6D98472B68002B0C
:1038A0007FF42FAF21E70133072B18BF0B607FF4A4
:1038B00031AF01230B602DE7012382E70133072B92
:1038C00018BF0B607FF422AF01230B601EE70123BA
:1038D0005FE700BFA0010020580400207001002015
:1038E00060610020880000204404002018040020AB
:1038F00028040020940300203C00002088030020BE
:10390000600300208001002070040020B00300202C
:103910007C0100205C0300206C0100207C00002062
:1039200068010020064B1A783E2A07D803D13F22AF
:103930001A70FEF767BA02321A70FAE7704700BFD2
:1039400068010020064A137843B1012B03D10023FC
:103950001370FEF757BA023B1370FAE7704700BFC7
:1039600068010020064B5A783E2A07D803D13F222F
:103970005A70FEF747BA02325A70FAE7704700BF32
:1039800068010020064A537843B1012B03D100237C
:103990005370FEF737BA023B5370FAE7704700BF27
:1039A00068010020064B9A783E2A07D803D13F22AF
:1039B0009A70FEF727BA02329A70FAE7704700BF92
:1039C00068010020064A937843B1012B03D10023FC
:1039D0009370FEF717BA023B9370FAE7704700BF87
:1039E0006801002040F26813C2F200031A780270E6
:1039F0005A7842709B788370704700BF10B440F2D1
:103A00006813047841788278C2F200033F2C34BFF7
:103A100020463F203F2928BF3F213F2A28BF3F2281
:103A2000187059709A7010BCFEF7ECB940F27C0324
:103A3000C2F200031A7802705A7842709B78837041
:103A4000704700BF10B440F27C030478417882785C
:103A5000C2F200033F2C34BF20463F203F2928BF3D
:103A60003F213F2A28BF3F22187059709A7010BC1E
:103A7000FEF70EB840F2A413C2F2000318687047B4
:103A80000F2803D8034B1860FEF7BCB9014B0F2277
:103A90001A60F9E7A4010020034B1A6802B97047C5
:103AA000013A1A60FEF7AEB9A4010020044B1A686F
:103AB0000E2A00D9704701321A60FEF7A3B900BF81
:103AC000A401002040F26413C2F20003186870479A
:103AD0000F2803D8034B1860FDF7DABF014B0F2204
:103AE0001A60F9E76401002070B5012682B040F247
:103AF000851516F0010F0CBF0021392116F0020FB9
:103B00000CBF0022392216F0040F0CBF002339230A
:103B10008DF804108DF805208DF80630002420461D
:103B200001A9013407F072F8AC42F8D1204606F042
:103B3000CDFF01360320FDF78FFE082ED9D10020DE
:103B4000FEF7EEF8002001460246FFF709FB02B03F
:103B500070BD00BF2A4B2DE9F04103F5907101249F
:103B600013F8012B12F0020214BF03F8014C03F802
:103B7000012C8B42F4D1017800293FD080460746C2
:103B800008260020C6F10802FEF726F898F8011072
:103B9000013759B3112E16D83D46344601E0112C99
:103BA00011D820460022FEF717F815F8011F093436
:103BB0000029F4D105E02046202100220934FEF737
:103BC0000BF8112CF7D90420FEF768FA3220FDF724
:103BD00035FE013E0CD017F8011C0020C6F108028A
:103BE000FDF7FAFF98F801100029D3D13446E8E731
:103BF00018F8011F0029C3D1BDE8F081BDE8F081AC
:103C000064610020F8B5324B1B681BB1A0F11405AC
:103C10003B2D00D9F8BD0020FEF782F82D4B2E4C2D
:103C200093F88830C3EB031305EB83052B4B04F5A6
:103C3000907103EBC5050120234613F8012B12F008
:103C4000020214BF03F8010C03F8012C8B42F4D1DB
:103C5000234E7079F278337958B102EBC20218180A
:103C600004EB4202D15C41F00201D15401338342A2
:103C7000F8D1307AB279F37958B102EBC202181850
:103C800004EB4202D15C41F00201D1540133834282
:103C9000F8D10027EB195B78ABB103EB4303F118C4
:103CA000F25C88784B7858B102EBC202181804EB2A
:103CB0004202D15C41F00201D15401338342F8D178
:103CC0000137072FE6D1074B01221A60F8BD00BF6C
:103CD00070010020DCDE00086461002028C50008B7
:103CE000F8DD0008580400202DE9F04FB94B1B689F
:103CF000044693B0184613B913B0BDE8F08F3F26C1
:103D00008DF834603C2603258DF8236016260023A9
:103D10000CA92A46A4208DF824600F268DF8353092
:103D20008DF836308DF825308DF826308DF82B3013
:103D30008DF827508DF8296000F0AEFB01220DF1BF
:103D40002101A72000F0A8FB01220DF12501A820E8
:103D500000F0A2FB01220AA9BD2000F09DFBBE20BD
:103D600001220DF12A0100F097FBB4F5843F80F0A9
:103D7000A3809DF821809DF822C09DF825E09DF844
:103D80002610B8F1110F84BF4FF000088DF8218084
:103D9000BCF1030F84BF4FF0000C8DF822C0BEF1C0
:103DA0000A0F84BF4FF0000E8DF825E0012902D9DB
:103DB00000218DF826109DF828700F2F02D90F27AB
:103DC0008DF828709DF829600F2E71D89DF82A0073
:103DD000012802D000208DF82A009DF82320642AB3
:103DE000009203D964258DF8235000959DF8243066
:103DF000632B02D916238DF82430774C079325685E
:103E0000764B01959DF827509DF834B002959DF8AA
:103E100030509DF835A003959DF831509DF83690AF
:103E200004959DF8325083F800B005959DF82B500D
:103E300083F801A0069540F2B835C2F2000583F878
:103E40000290C5F80080DFF8C081029DC8F800C06C
:103E5000DFF8B8C1624BCCF80050DFF8B4C1614A5A
:103E6000CCF800E0DFF8ACE11F60CEF800105E4B4C
:103E70000399049D11701E6005995C4B55709170FB
:103E80001860009A5A4B079D1A605A4B06991D609C
:103E9000594B196000232360FDF7FAFDFDF7B2FFCF
:103EA000019A2260FFF71CFBFDF71EFE012023E7AD
:103EB0000F268DF8296089E7A92001220DF126013E
:103EC00000F0EAFA40F6FF03C0F201039C427FF6DD
:103ED00050AF01220DF12701BC2000F0DDFA0DA941
:103EE0002A46D72000F0D8FA01220DF12901DA2064
:103EF00000F0D2FADB2001220DF1220100F0CCFA11
:103F0000B4F5003FFFF435AF01220DF12301DC20B1
:103F100000F0C2FADD20012209A900F0BDFAFF235A
:103F2000C0F202039C427FF624AF0DF12B01012267
:103F3000E02000F0B1FA0FA90B22E52000F0ACFA66
:103F40000EAE0BA9022240F2251000F0A5FA40F2B5
:103F500035103146042200F09FFA0DF14605274B3B
:103F60000DF13B0005E042F002021A611433A84251
:103F700012D010F8012FFF2AF8D002F01001C9B2B8
:103F800002F00F029A601A690029ECD122F00202B5
:103F90001A611433A842ECD19DF82C301848FF2B3D
:103FA0001EBF184A03F00F0353609DF82D30FF2BFE
:103FB0001EBF144A03F00F0353610023F25CFF2A73
:103FC0001EBF00EB031102F00F024A600133042B05
:103FD000F4D1CEE6A4040020700100207C00002073
:103FE000A401002068010020640100203C0400209E
:103FF00078010020A801002078030020880000201C
:104000003C000020800100202804002084000020C3
:10401000A0010020180400202DE9F04F854B1B68FB
:10402000A3B0002B00F08B80834B844A93F8008070
:1040300093F801C093F802E0814B92F800B01F683A
:10404000804B92F801A01E687F4B92F802901D6889
:104050007E4B8DF819501C687D4B8DF81A401B68FB
:104060008DF820B000937B4B009C1B688DF81B40A3
:104070000193794B019C1B688DF821A00293774B2B
:104080008DF822901B688DF824800393744B8DF873
:1040900025C01868734B8DF826E01968724B8DF8AF
:1040A00015701A688DF816608DF81C40029C6F4BD5
:1040B0008DF81D40039C8DF817008DF81E408DF87B
:1040C000181000208DF81F2012ACFF250A2888BF89
:1040D000255409D89A68196902F00F0289072254F9
:1040E00044BF42F010022254013014334028EDD175
:1040F0005F4800230AAEFF22012B97BF00EB03119C
:10410000F254496801F00F0198BFF1540133102BAC
:10411000F2D1584900230EADFF2001EB0312032B0F
:1041200097BF5268E85402F00F02EA540133102B93
:10413000F3D1A42008A9032200F0C8F918B900207F
:1041400023B0BDE8F08FA7200DF11501012200F08A
:10415000BDF90028F3D0BC200DF11901012200F0B7
:10416000B5F90028EBD0A8200DF11A01012200F0CA
:10417000ADF90028E3D0A9200DF11B01012200F0C8
:10418000A5F90028DBD0BD2007A9012200F09EF987
:104190000028D4D0BE200DF11E01012200F096F9B6
:1041A0000028CCD0D72009A9032200F08FF90028DD
:1041B000C5D0DA200DF11D01012200F087F9002899
:1041C000BDD0DB200DF11601012200F07FF900289F
:1041D000B5D0DC200DF11701012200F077F900289D
:1041E000ADD0DD2006A9012200F070F90028A6D08C
:1041F000E0200DF11F01012200F068F900289ED097
:10420000E5202146402200F061F9002897D040F2D5
:1042100025103146102200F059F900288FD01022C5
:1042200040F23510294600F051F9003018BF012046
:1042300086E700BFA40400207C0000206801002065
:10424000B80300202804002084000020A0010020E2
:1042500018040020A4010020640100203C04002078
:1042600078010020A80100207803002088000020A9
:10427000800100203C00002006F0F4BC2DE9F8434A
:1042800081468846174605F071FC10B90020BDE84C
:10429000F883552005F002FD2E48082105F026FD83
:1042A000442005F0FBFC002443F2144505F0C0FC5B
:1042B0000134AC4298BF002814BF00260126F5D077
:1042C00043F214439C4227D805F050FC0028DDD06F
:1042D000552005F0E3FC204C1E48082105F006FDA2
:1042E000BE2005F0DBFC0921204605F0C9FC05F0E5
:1042F0003DFC1A4B1B68222B13D0282B11D009230D
:10430000C9F8003094F90130DB0FC8F80030237889
:1043100001203B60BDE8F88305F028FC3046BDE88D
:10432000F883237962782578C3F34113093302F0C7
:104330000704C3F10C00191F45FA00F004FA01F15B
:104340000143D209C9F800300120C8F800203960C3
:10435000BDE8F88398040020840400209404002021
:10436000F8B5A0F10905032D044602D90026304610
:10437000F8BD05F0EBFC05F0F9FB0028F6D02E4F58
:10438000384605F0C1FC3B782C4A13602C4A0121C9
:10439000222B0646116001D0282BE8D105F0E6FB60
:1043A0000028E4D0552005F079FC264F224808214A
:1043B00005F09CFCBE2005F071FC0921384605F093
:1043C0005FFC3B79C3F341130933A342CFD005F01F
:1043D000CDFB0028CBD0552005F060FC0821164805
:1043E00005F084FC4E2005F059FC7F2005F056FCBA
:1043F000802005F053FC680100F0E00005F04EFC61
:1044000005F0B4FB05F0B2FB0028B0D0552005F054
:1044100045FC0948082105F069FC482005F03EFCF0
:10442000002405F005FC0134F92C98BF0028F8D0D1
:1044300005F09CFB9BE700BF98040020940400203B
:1044400090040020840400202DE9F04184B003F0A2
:1044500035F8DFF8408000240127650045F0A0050D
:10446000012600972846002132460DF10F03A419BA
:10447000C8F8005003F076F830B1082CEDD1044BA9
:10448000186804B0BDE8F081014B30461E60F8E7C3
:10449000A4040020A004002010B50A4B1C6882B0C0
:1044A0000B4614B9204602B010BD0092064A1268AD
:1044B00001461046012203F055F8D0F1010038BF43
:1044C0000020F0E7A4040020A00400202DE9F0471C
:1044D000144B1B6882B0174603B3EAB1DFF84CA057
:1044E000114C0646C0EB01094FF001080025DAF82F
:1044F0000000CDF800803146012209EB060303F0ED
:10450000AFF858B910202368002BFCD00138256083
:10451000F9D10136013FEAD1012000E0002002B0CC
:10452000BDE8F087A404002084620020A0040020DD
:1045300070B53E4B1A68824288B0064674D002A815
:104540001E60FCF787F904A8FCF7CAFC01200146AD
:10455000FCF72EFB01200146FCF72AFB202001215D
:10456000FCF742FB0020C4F202000B210822FCF7FA
:1045700087F900200822C4F202000C21FCF780F920
:10458000022300208DF80C30032304460125C4F2D9
:10459000020002A98DF80D304FF4006302938DF8EC
:1045A0000E408DF80F50FCF7F9F820464FF4805379
:1045B000C4F2020002A90293FCF7F0F84FF4A050F5
:1045C000C4F201002946FCF7A5FC4FF4A0500C23CF
:1045D000C4F2010004A9ADF81A300496ADF81440F5
:1045E000ADF81640ADF81840ADF81C40FCF70CFCD7
:1045F0004FF4A050C4F201002946FCF77DFC4FF4B3
:10460000A050C4F2010040F225512A46FCF798FC64
:10461000472301A88DF804308DF805408DF8064039
:104620008DF80750FBF714FE08B070BDC0060020DF
:1046300030B40F4A13687F2BFCD80E490E4D0B681F
:104640005C1C7F2C45F8230098BF0C6001D9002327
:104650000B6072B613680133136062B64FF4A0505A
:10466000C4F2010040F22771012230BCFCF768BCA3
:10467000BC060020B8060020B004002010B5044697
:10468000007828B1FFF7D4FF14F8010F0028F9D102
:1046900010BD00BF40F2AC43C2F200031868003006
:1046A00018BF0120704700BF30B40D4B1A6882B1AB
:1046B0000C490D4D0A68541C802C55F8225018BF27
:1046C0000C6009D072B61A68013A1A6062B601220B
:1046D0000560104630BC704700220A60F2E700BF58
:1046E000AC040020A8040020C4060020024A13687D
:1046F000002BFCD1704700BFBC0600204FF4A05037
:1047000038B5C4F2010040F22551FCF735FC002811
:104710002BD14FF4A050C4F2010040F22771FCF7F6
:104720002BFC00B938BD4FF4A050C4F2010040F298
:104730002771FCF747FC234B1A68002A38D0224A1D
:10474000224C1168481C802808BF002054F8211012
:1047500010601A684FF4A050013AC4F2010089B207
:104760001A60BDE83840FCF7E3BB4FF4A050C4F238
:10477000010040F22551FCF725FC4FF4A050C4F293
:104780000100FCF7D9FB124B1A687F2AC1D81149E6
:10479000114D0A68541CC0B27F2C45F8220098BF06
:1047A0000C6001D900220A601A6801321A60B0E771
:1047B0004FF4A050C4F2010040F22771BDE8384028
:1047C000FCF7BEBBBC060020B0060020B0040020F1
:1047D000AC040020B4060020C40600202DE9F043FC
:1047E00083B06846FCF736F800260120C4F20206C2
:1047F00001460124FCF7DCF900254FF08009304622
:104800006946CDF800908DF805508DF804408DF87C
:1048100006508DF80750FBF7C1FF20462146FCF7F4
:10482000C7F94FF0400830466946CDF800808DF852
:1048300005508DF804408DF806508DF80750FBF7B1
:10484000ADFF20462146FCF7B3F9102730466946F4
:1048500000978DF805508DF804408DF806508DF8BE
:104860000750FBF79BFF304649462246FCF702F80B
:10487000304641462246FBF7FDFF30463946224688
:10488000FBF7F8FF03B0BDE8F08300BFF8B5094DB2
:1048900004460F46002601E02B6833B92046FFF797
:1048A00003FF0028F8D00120F8BD0136BE42286081
:1048B000F4D3F8BD886200202DE9F04F85B005469D
:1048C00003F020FDFFF712FFFFF7E4FE002843D0BE
:1048D0000024624FDFF888A10126A346294603A8D9
:1048E000FFF7D4FFDFF874914FF00108034600286A
:1048F00035D0039B3E600A2B07D00D2BEED0FF2C4A
:10490000ECD80AF804300134E8E70AF804B0002CC7
:1049100032D103F0F7FCE1E7514852491A4606F05C
:1049200004FE00284CD04E484F49032206F0FDFDFE
:1049300000284FD04A484D49052206F0F6FD0028D0
:1049400055D14B484B49022206F0EFFD002849D1D2
:104950000123C9F80830062005B0BDE8F08F4648AD
:10496000019303F0A1FC454803F09EFC444803F08A
:104970009BFC019B1846EFE73F48019303F094FC32
:10498000374803F091FC3E4803F08EFC34483D4923
:10499000022206F0CAFD38B131483B49052206F033
:1049A000C4FD18B90220D7E74046D5E72C4837495F
:1049B000022206F0BAFD019B0028ADD10320CBE70F
:1049C00009F13C0032490F2206F0C8FDC9F8048005
:1049D0000420C1E709F11C002E491F2206F0BEFD8C
:1049E0000520B9E70023C9F808300620B4E71C48C1
:1049F0002949052206F099FD98B11948274909224D
:104A000006F093FD10B316482549042206F08DFDEB
:104A1000A8B113482349092206F087FD40B1FF20C1
:104A20009AE7214812490F2206F098FD072093E7E4
:104A30001E481F49FF2206F091FD0A208CE71D4801
:104A40001D491F2206F08AFD092085E71B481849E9
:104A50000F2206F083FD08207EE700BFC408002077
:104A6000400A00208CDF000898DF00089CDF000867
:104A7000450A0020A4DF00086CDF000870DF000892
:104A800078DF00087CDF000880DF000888DF00088E
:104A90004A0A0020430A0020A8DF0008B0DF00080F
:104AA000BCDF0008C4DF0008300A00201009002025
:104AB000490A0020100A0020440A0020D0080020E3
:104AC000F0B583B0074606F028FD06461A4803F005
:104AD000EBFBBEB13C46F61904E0184603F0BEFB02
:104AE000B4420FD014F8013B1449A3F120055E2D08
:104AF00068461A46F1D906F0CDFC684603F0D4FBAF
:104B0000B442EFD10E4803F0CFFB03F0FBFB384675
:104B1000FFF7B4FD0B48FFF7B1FDFFF7E7FD02E03B
:104B2000022807D020B10A20FFF7C6FE0128F7D1DE
:104B300003B0F0BD0020FBE7D0DF0008E4DF000891
:104B4000D8DF0008ACE1000838B539B10446451893
:104B500014F8010BFFF76CFDAC42F9D1BDE8384009
:104B6000FFF7C4BD40F6C400C2F20000704700BFAA
:104B700010B50020C4F202008021002282B0FBF7B1
:104B800079FE0C4A0521144600201368002BFCD046
:104B900001392060F9D10020C4F2020080210122F5
:104BA000FBF768FE01A83221FFF770FE0028F9D15B
:104BB00002B010BD8862002008B502460B460748C7
:104BC000074906F067FC0548FFF77AFF20B1054B5F
:104BD000002283F83C205A6008BD00BF440B00202F
:104BE000ECDF0008C408002008B502460B46074861
:104BF000074906F04FFC0548FFF762FF20B1054B5F
:104C0000002283F83C205A6008BD00BF440B0020FE
:104C1000FCDF0008C408002008B5024608B103788C
:104C200023B90748BDE80840FFF74ABF05490648D1
:104C300006F030FC0448BDE80840FFF741BF00BF64
:104C400028E600080CE00008440B002030B54FF4C3
:104C5000E13083B003F0F0FBFFF7C0FD4FF4E1302B
:104C6000FFF766FC0020C4F2020010210022FBF7CF
:104C700001FE1E4C00200022C4F202008021FBF73E
:104C8000F9FD05252246002321680029FCD0013DBD
:104C90001360F9D1002080210122C4F20200FBF749
:104CA000E9FD124932222368002BFCD0013A0D6045
:104CB000F9D10020C4F2020010210122FBF7DAFD35
:104CC00003E001A803F0FCFA60B901A8FFF7ECFCCF
:104CD0000028F6D0019803F0C1FA01A803F0F0FA19
:104CE0000028F2D00198FFF7A3FCEEE788620020CD
:104CF00008B50B4B1A6802B108BD01224FF4E13030
:104D00001A6003F099FB074803F0CEFAFFF766FD3F
:104D10004FF4E130FFF70CFCBDE80840FFF728BF77
:104D2000940B002018E0000810B403781649FBB17A
:104D3000002208601446013005E001300E2A14DC20
:104D400010F8013C8BB13D2B02BF01EBC20300F810
:104D5000014C5860F1D0262BEFD1013200F8014C04
:104D600041F8320001300E2AEADD531C0F2B08DC1B
:104D7000002201EBC30011460133815008320F2B92
:104D8000FADD10BC704700BFF40B0020F8B50A4DE7
:104D90000646002455F83430E70031461846013401
:104DA00023B106F0A8FB18B1102CF3D10348F8BDCD
:104DB000014BDF197868F8BDF40B002034E10008DE
:104DC00008B5FFF7E3FF4EF21011C0F6000106F040
:104DD00092FBD0F1010038BF002008BD00B50B46A2
:104DE00085B04EF218110246C0F60001684606F082
:104DF00051FB6846FFF7CAFF05B000BD10B5044679
:104E000006F08BFB014600B910BD2046BDE81040FE
:104E1000FFF79ABE10B504464EF22010C0F600000F
:104E2000FFF7ECFF4EF23010C0F60000FFF7E6FF90
:104E30004EF23810C0F60000FFF7E0FF4EF24410CB
:104E4000C0F60000FFF7DAFF4EF25010C0F6000087
:104E5000FFF7D4FF2046FFF7D1FF4EF25810C0F6FF
:104E60000000FFF7CBFF4EF26410C0F60000FFF722
:104E7000C5FF4EF27010C0F60000FFF7BFFF4EF204
:104E80007C10C0F60000FFF7B9FF2046FFF7B6FF21
:104E90004EF28410C0F60000BDE81040FFF7AEBF30
:104EA00038B504464EF28C10C0F600000D46FFF7F0
:104EB000A5FF2046FFF7A2FF4EF29810C0F60000B3
:104EC000FFF79CFF2846FFF799FF4EF29C10C0F6B3
:104ED0000000BDE83840FFF791BF00BF4EF234102C
:104EE0004EF2B01108B5C0F60000C0F60001FFF7A1
:104EF000D7FF4EF2B8104EF2C011C0F60000C0F657
:104F00000001FFF7CDFF4EF6CC104EF2C811C0F6EF
:104F10000000C0F60001FFF7C3FF4EF2D4104EF2BE
:104F2000D811C0F60000C0F60001FFF7B9FF4EF639
:104F300048304EF2DC11C0F60000C0F60001FFF769
:104F4000AFFF4EF2E4104EF2F011C0F60000C0F6D2
:104F50000001FFF7A5FF4EF2FC104EF20821C0F64B
:104F60000000C0F60001FFF79BFF4EF214204EF246
:104F70001C21C0F60000C0F60001FFF791FF4EF2C1
:104F80002420C0F60000BDE80840FFF737BF00BF8F
:104F9000054A136801331360DB0702D40348FFF7A7
:104FA0002DBF0348FFF72ABFB00C002040E20008E5
:104FB00028E2000810B504464EF24820C0F6000072
:104FC000FFF71CFF2046FFF719FF4EF25020C0F6F6
:104FD0000000BDE81040FFF711BF00BF70B584B0FE
:104FE0000C4605461B49164668461A4606F052FA14
:104FF00002A81849089A06F04DFA3CB123782BB163
:105000002046FFF7FBFE1448FFF7F8FE1348FFF7B2
:10501000F5FE2846FFF7F2FE1148FFF7EFFE28469F
:10502000FFF7ECFE0F48FFF7E9FE3046FFF7E6FE1C
:105030000D48FFF7E3FE6846FFF7E0FE0B48FFF779
:10504000DDFE02A8FFF7DAFE0948FFF7D7FE04B03D
:1050500070BD00BF64ED0008F8E8000858E20008E1
:1050600070E200087CE2000888E2000898E200088C
:1050700098E1000810B504464EF2A420C0F60000E6
:10508000FFF7BCFE2046FFF7B9FE4EF2D820C0F66F
:105090000000FFF7B3FE4EF2E820C0F60000BDE8C6
:1050A0001040FFF7ABBE00BF70B505460F480E4677
:1050B000FFF7A4FE0E48FFF7A1FE002E0EDD043D13
:1050C00000240C48FFF79AFE55F8040FFFF796FEF0
:1050D00001340948FFF792FEB442F2D10748FFF7C6
:1050E0008DFE074B00221A6070BD00BFF0E2000881
:1050F00040E200080CE3000824E3000804E3000891
:10510000B00C00204EF23430C0F60000FFF776BE3F
:1051100038B504464EF24430C0F600000D46FFF7A5
:105120006DFE2046FFF76AFE4EF29810C0F60000B2
:10513000FFF764FE2846FFF761FE4EF27030C0F6BE
:105140000000BDE83840FFF759BE00BF08B54EF279
:105150008030C0F60000FFF751FE4EF28C30C0F6F2
:105160000000BDE80840FFF749BE00BFF0B50446A7
:1051700083B01F481E460D461746FFF73FFE2046E8
:10518000FFF73CFE1B48FFF739FE2046FFF736FECF
:105190001948FFF733FE002E24DD043D00240BE008
:1051A0001648FFF72BFE55F8040FFFF727FE1448AB
:1051B000FFF724FEB44215D02246124901A806F09A
:1051C00069F91148FFF71AFE01A8FFF717FE0F480B
:1051D000FFF714FEBC4204F10104E1D10C48FFF7D3
:1051E0000DFEDDE70B48FFF709FE03B0F0BD00BF81
:1051F00098E3000870E20008A8E30008A4E40008AF
:10520000D8E3000864ED0008BCE3000884E200086D
:10521000CCE30008B0E3000870B50E4605460E4822
:105220001446FFF7EBFD3046FFF7E8FD0B48FFF7AC
:10523000E5FD2846FFF7E2FD0948FFF7DFFD14B161
:105240000848FFF7DBFD0848FFF7D8FD0748BDE831
:105250007040FFF7D3BD00BF48E20008E4E3000858
:1052600008E400081CE40008A4E4000850E2000878
:105270002DE9F041069F079D04461646984611B158
:105280000B78002B49D12848FFF7B8FD2046FFF7DF
:10529000B5FD2648FFF7B2FD2046FFF7AFFD2448D5
:1052A000FFF7ACFD3046FFF7A9FD2248FFF7A6FD4A
:1052B0004046FFF7A3FD2048FFF7A0FD3846FFF763
:1052C0009DFD55B12B7843B11C48FFF797FD28464B
:1052D000FFF794FD1A48FFF791FD1A48FFF78EFD7E
:1052E0002046FFF78BFD1848FFF788FD2046FFF7A3
:1052F00085FD1648FFF782FD1548FFF77FFD204624
:10530000FFF77CFD1348FFF779FD3046FFF776FD88
:105310001148BDE8F041FFF771BD0846FFF76EFD8B
:105320000E48FFF76BFDAEE724E4000870E20008CA
:105330007CE2000840E4000848E4000850E400086B
:1053400060E4000864E4000870E4000880E40008F9
:105350008CE400089CE40008A8E40008F8E80008D1
:105360004EF2B440C0F600000321FFF7EDBB00BFD2
:1053700010B504464EF24820C0F60000FFF73EFD8F
:105380004EF2B8412046C0F60001FFF7C1FE4EF2D2
:10539000E820C0F60000BDE81040FFF72FBD00BFB9
:1053A00070B506464EF2482082B0C0F600000D46A9
:1053B0001446FFF723FD4EF234114EF2C043C0F6FF
:1053C0000001C0F600033046009301912A462346AF
:1053D000FFF74EFF4EF2E820C0F6000002B0BDE835
:1053E0007040FFF70BBD00BF38B505460C46FFF710
:1053F000CFFD2846FFF7DEFD2046FFF7DBFD4EF22E
:105400003410C0F60000FFF7D5FD4EF20430C0F6B0
:105410000000BDE83840FFF7F1BC00BF10B50446FE
:105420004EF2C440C0F60000FFF7E8FC2046FFF74C
:10543000E5FC4EF2A830C0F60000BDE81040FFF7D2
:10544000DDBC00BF10B50446FFF7A2FD2046BDE855
:105450001040FFF7E3BF00BF4EF2E440C0F600008B
:10546000FFF7CCBC08B5FFF7F7FF4EF20430C0F6EB
:105470000000BDE80840FFF7C1BC00BFF0B583B035
:105480000E4614461F46089DFFF7DCFF3046FFF727
:1054900091FD4EF24820C0F60000FFF7AFFC4EF23F
:1054A0003411C0F600013A462B4620460095FFF71E
:1054B00095FD4EF25020C0F60000FFF79FFC2046FD
:1054C000FFF7D8FD03B0BDE8F040FFF7CBBF00BF4A
:1054D000F8B5069D0E4614461F46FFF7B3FF30464B
:1054E000FFF768FD204639462A46FFF795FE20461D
:1054F000FFF7C0FDBDE8F840FFF7B4BF2DE9F0416C
:105500000F4614469846069E079DFFF79BFF3846B8
:10551000FFF750FD4EF24820C0F60000FFF76EFC8A
:10552000414632462B462046FFF720FE4EF25020E1
:10553000C0F60000FFF762FC2046FFF79BFDBDE8C8
:10554000F041FFF78FBF00BF2DE9F04F83B08B46CE
:1055500092469946DDF830800D9F124EFFF772FF9C
:105560001148FFF727FD1148FFF748FC00243D597B
:105570005BF804005AF8041059F8042058F8043075
:105580008DE86000FFF774FE04340948FFF736FC2D
:105590000C2CECD10748FFF76DFD03B0BDE8F04FD0
:1055A000FFF760BF00E50008F0E40008F8E4000839
:1055B00004E50008B0EB00082DE9F04F05460E4663
:1055C000C7B0A7482946924602F026FF33781BB39E
:1055D000741C4FF02008002706E02B2B08BF04F8AE
:1055E000018C14F8013BBBB1252BF6D120460221DA
:1055F000FBF7B0FDA27804F8010C002A00F03F850B
:10560000234603F8012B9A781946002AF9D10F7026
:1056100014F8013B002BE7D13146924802F0FCFE22
:105620003046FFF781FB28468F4905F064FF0028CC
:1056300042D028468D4905F05EFF0446002800F060
:10564000CB8328468A4905F056FF002800F06F8476
:105650002846884905F04FFF0446002800F0938152
:105660002846854905F047FF002800F0698528464F
:10567000824905F040FF002800F0EE872846804967
:1056800005F039FF002800F04D8228467D4905F0DD
:1056900032FF002800F004877B48FFF7AFFB7B4810
:1056A000FFF7ACFB7A48FFF7A9FB0026FFF758FE8F
:1056B000304647B0BDE8F08F764C94E803001AAD51
:1056C00004F1080685E803000FCE3EAF07953D467E
:1056D0000FC596E80300059704F1200785E803004D
:1056E0000FCF25AD04F1340E2E460FC6BEE80F00D5
:1056F0003F68089504F1480C2AAD069537600FC540
:10570000BCE80F002FAF48343E460FC60FCC0DF15A
:10571000D00844460FC4DCF80030DEF800203360C7
:10572000236015A92A6014A816AA1CAC0DF1600B01
:1057300013AE3C913D920994CDF8E4B03A963B907B
:1057400002F0BCFF814602F0BFFF5349C0F307429D
:10575000C0F30723099805F09DFE02F0BBFF4269E4
:10576000002A044632DB0369002B2FDBC1680029C5
:105770002CDB8068002829DB6568002D26DBB2F56C
:10578000966F23DC0C2B21DC1F291FDC17281DDC66
:105790003B2D1BDC02F26C725846404905F07AFE44
:1057A00022693F490132304605F074FEE2683C4907
:1057B00014A805F06FFEA268394915A805F06AFE25
:1057C00016A83749626805F065FE0AE000238DF8E7
:1057D00060308DF84C308DF850308DF854308DF8A5
:1057E00058303048FFF7D2FA0546002801F084808F
:1057F0002D4905F080FE002841F04D802B4C4926B4
:105800002B48DFF8C4A0FFF705FBFFF767FB0798FD
:105810000221FFF749FC27484946FFF7E5FDDAF882
:105820000030254A25492648002B18BF1146FFF7AE
:10583000DBFDDAF80030002B41F02780FFF762FC37
:1058400005980621FFF730FC1E48FFF7FBFDDA46FE
:1058500009954FF000090594089DDDF818B038E06F
:1058600098E60008ACE60008C4E60008ECE700088B
:1058700060E9000844EA0008CCEA000804EC0008EB
:10588000C0EC000868ED0008B4ED000830E1000845
:10589000CCED00082CE00008C8E60008D4E60008BB
:1058A000D8E60008E0E60008E8E600081CE5000885
:1058B00038E7000844E70008D0F500086CE5000868
:1058C0004CE7000834E10008A404002039AB59F883
:1058D00003A07548FFF792FA58F8094055F80900F7
:1058E0005BF8091057F8093000945246FFF776FB31
:1058F00009F104096D48FFF781FAB9F1140FE5D1F8
:105900006B48059C099DFFF7B5FBFFF7ABFDFFF763
:10591000F9FB07980221FFF7C7FB6648664A67490B
:105920001E2703460097FFF7A9FDFFF7EBFB614831
:10593000FFF774FD62486349FFF7EAFB6248634979
:10594000FFF7E6FB62486349FFF7E2FB6248634901
:10595000FFF7DEFBFFF780FD44B16148FFF74EFA29
:105960002046FFF74BFA5F48FFF748FA28465A49A6
:1059700005F0C1FD0446002800F0E384FFF7E6FBD4
:10598000FFF7EEFC94E6584B93E803003EAD85E844
:1059900003000595FDF762FD80465448FFF7F6F9D0
:1059A0000546002801F0F881514905F0A4FD06469E
:1059B000002801F03F8128464E4905F09CFD06462F
:1059C000002801F0198028464B4905F094FD054652
:1059D000002841F0DD814948FFF7F2F910F1000895
:1059E00018BF4FF00108CAF800804C2600238DF83C
:1059F000BC300A24FBF748FB0DF13A00FBF752FBE1
:105A0000002841F001810A20FBF718FF013CF3D187
:105A100046AF3F2327F85C3D02F06CFA384982B26A
:105A200034A805F037FD02F06BFA354982B239A887
:105A300005F030FD3348FFF7EDF9FFF74FFA059811
:105A40000221FFF731FB30483946FFF7CDFC2F48E4
:105A500034A9FFF7C9FC2E4839A9FFF7C5FC274A2E
:105A60002C4B29492C48CDF80080FFF731FDFFF77A
:105A700049FB2948FFF7D2FC1D482849FFF748FB9E
:105A80001C482749FFF744FBFFF7E6FC002D3FF4D5
:105A900075AF1348FFF7B2F92846FFF7AFF9114881
:105AA000FFF7ACF96AE700BF48E2000850E20008DF
:105AB00008E7000834E1000830E7000864E7000860
:105AC000F0E600086CE70008F8E6000878E7000850
:105AD000E8E6000884E700089CE70008A8E700085B
:105AE000B4E7000854E900082CE00008E0E60008EC
:105AF0004CEA000854EA00085CEA000860EA000882
:105B000068EA00086CEA0008D8E100087CEA0008AE
:105B100080EA000884EA0008D4E100089CEA000852
:105B2000B4EA0008914E924D96E8070006F1500342
:105B300020AC84E807000FCB3EAF06F10C0E87E8DF
:105B40000F009EE8070025AB08930597089F06F114
:105B5000180387E8070093E807002AAB0693069F1F
:105B600006F1240387E8070093E807000DF1D00849
:105B7000303688E8070096E807002B687D4F0DF166
:105B8000E40989E807004BB97B4E3B6A39683A69FA
:105B9000386B86E80E000123F0602B60FDF7F2FB06
:105BA0000790FDF709FC0A90FDF714FC0B90FDF738
:105BB000C5FB00F002000C90FDF784FF0990FDF793
:105BC0004DFC0D900FA8FDF731FF6C48FFF7DEF894
:105BD0000546002800F01587694905F08CFC8346CE
:105BE000002801F083802846664905F084FC83463E
:105BF000002801F0FB802846634905F07CFC8346C1
:105C0000002801F0BB812846604905F074FC064677
:105C1000002801F04F8328465D4905F06CFC0646DC
:105C2000002801F0F08228465A49072205F07DFC41
:105C30000646002801F0DE8228465749042205F076
:105C400074FC0646002801F052832846534905F0AB
:105C500052FC0026B34610B9DFF878B153267A6BB0
:105C60004F4915A805F016FC4D490A9A16A805F0EB
:105C700011FC4B490B9A18A805F00CFC11AD4849D2
:105C8000099A10A805F006FC0DF1480A44499DF850
:105C90003C20284605F0FEFB13AF41499DF83D200E
:105CA000504605F0F7FB9DF83E203D49384605F08B
:105CB000F1FB3C482F950325CDF8C0A03197FFF7A5
:105CC000A9F8FFF70BF920462946FFF7EDF936480A
:105CD0003649374A009516ABFFF7D0FB009532489E
:105CE0003449354A18ABFFF7C9FB0C9C5CB90D9DD4
:105CF000002D01F01D818DE800032B480899069ABC
:105D00002FABFFF721FC079F2C4A1B4B26482C4941
:105D1000009704240194FFF7F1FBFFF7F3F9214604
:105D20000598284DFFF7C0F900242B68DA0700F129
:105D3000948601341035042CF7D1FFF7E3F91A48A3
:105D4000FFF76CFB15482049FFF7E2F9FFF784FBEA
:105D5000BBF1000F3FF412AE1C48FFF74FF8584656
:105D6000FFF74CF81A48FFF749F807E690E00008FB
:105D7000980B00203C0000209C0B0020E0E600086F
:105D8000F4EA000804EB0008CCEC0008DCEC0008A6
:105D9000ECEC0008FCEC00080CED000850EB0008EF
:105DA00064ED000814ED0008FCE1000828ED00088F
:105DB000E0EC000830ED0008F0EC0008D0EC000842
:105DC00048ED000848000020F8EB0008B4E70008A0
:105DD00054E9000878E60008AB4B93E803000DF1A6
:105DE000E409083389E8030093E807003EAD85E83D
:105DF00007000595FEF7B6FE0546A448AF68FEF716
:105E0000C5FF05F10C088246002800F0EA87A0498A
:105E100005F071FB0646002800F04A8650469D4971
:105E200005F069FB0646002800F0F78650469A49BF
:105E300005F061FB0646002800F00E8750469749A2
:105E400005F059FB002800F05B852646B24604F0B9
:105E500093FD9349024634A805F01CFB9148FEF7D8
:105E6000D9FFFFF73BF805980321FFF71DF98E488E
:105E700005F13C01FFF7B8FA41468C48FFF7B4FA48
:105E80008B48FFF7DFFA8B48FFF794F88A48FEF754
:105E9000B5FF4FF00F08894849463A460223FFF7FD
:105EA00065F987498748CDF8008005F11C02202359
:105EB000FFF794F88448FEF7A1FF14238349844A2E
:105EC000844800934023FFF789F88348FEF796FF44
:105ED0008248FFF7CFF8FFF7C5FA04F06FFD80495D
:105EE000804ACDF8008003467148FFF7C7FA0323C4
:105EF0007D497E4A6E48009334ABFFF7BFFAFFF747
:105F000001F96B48FFF78AFA64487949FFF700F90D
:105F1000FFF7A2FA002C00F005827648FEF76EFF2C
:105F20002046FEF76BFF7448FEF768FF26E5734BCB
:105F300093E803000DF1D00888E803005348FEF70A
:105F400025FF0446002800F0EE846D4905F0D3FAE1
:105F50000646002800F04E8620466A4905F0CBFA36
:105F60000646002800F0A5862046674905F0C3FADA
:105F7000002840F0D884654D5726654B1B68002BE0
:105F800000F0628504F09EFA0DF1E409044662080F
:105F90004846434905F07EFAE70700F1B2864846D5
:105FA00005F0BBFA5B4B09EB000201469C881868C0
:105FB0009B7949F8010094809371574B1B68002B23
:105FC00000F0398504F014FC3EAF04466208384600
:105FD0003349059705F05EFAE40700F19F860598BE
:105FE00005F09BFA059C4B4B059F221801469C88A7
:105FF00018689B7978509480937104F053FA0246A4
:10600000002840F0778546AF07F85C0D04F040FCAF
:106010000246002840F0668546AC04F8700D0694F0
:106020003E48FEF7F7FEFEF759FF40460221FFF714
:106030003BF83B484946FFF7D7F902243948059910
:10604000FFF7D2F938483949394A00943B46FFF7FF
:1060500015FA3849384A069B33480094FFF70EFA80
:10606000FFF750F83048FFF7D9F927483349FFF7D1
:106070004FF8FFF7F1F9002D7FF40BAD7EE42146D8
:106080000F70FFF7C5BA00BF88E00008E0E600081F
:10609000F8E7000894E80008A4E80008B4E800085D
:1060A00064ED000818E80008BCE80008C8E800082B
:1060B000B8E10008DCE8000848E2000804E800084D
:1060C000E4E8000810E80008ECE8000800E900082F
:1060D00034E10008DCF6000850E20008FCE70008A4
:1060E00004E9000898E8000810E90008A8E800089A
:1060F00024E9000834E9000850E900082CE0000811
:1061000070E9000880E9000890E9000830E600081E
:1061100054130020A8E9000890040020B0E900080A
:10612000C8E90008D8E90008CCE90008E0E900085F
:1061300074E9000808EA000884E9000830EA000869
:10614000AD4B93E8070003F10C0425AE86E8070089
:1061500094E807002AAD03F1180485E8070094E8E5
:1061600007002FAF03F1240487E8070094E8070035
:1061700030330DF1E40989E8070093E80700089639
:106180003EAE86E8070006950596FDF731F90B90BF
:10619000FDF7D4F80546FDF7B5F90C90FDF76AFC5C
:1061A0008046FDF75BF9954C0D9016A8FDF71AFC9B
:1061B000236805F00102C5F3400B079253B9904ADA
:1061C0009048191808334968902B42F8041FF8D1F9
:1061D000012323608C48FEF7D9FD0446002800F017
:1061E000F8858A4905F087F9002800F06183204688
:1061F000874905F080F9002840F09B858548FEF727
:10620000DFFD002800F01386012645F002050996FF
:10621000CAF80050472620467F4905F06CF905462C
:10622000002800F0578520467C4905F064F90028D5
:1062300040F09D857A4DDFF864A20A9558260DF14D
:10624000600B424677490DF16808584605F022F97F
:106250001CAD74499DF85820404605F01BF91EAC52
:1062600070499DF85920284605F014F99DF85A20E8
:106270006C49204605F00EF90A9BCDF8D0801A68CB
:1062800035953694002A40F01E8546AC04F8982DCA
:106290006548FEF7BFFDFEF721FE08980321FEF7D3
:1062A00003FF079D61486249624A634B0095FFF70F
:1062B0000FF90B9D5D48009512256049604A614BBE
:1062C0000195FFF71BF9099D584800955E49514A11
:1062D0005E4BFFF7FDF80D9D002D00F0CC840C9D6A
:1062E000002D00F0DA840223594A5A494F4800939E
:1062F0002346FFF7C3F8FEF705FF4C48FFF78EF87B
:1063000055485649FEF704FF55485649FEF700FF29
:1063100042485549FEF7FCFE54485549FEF7F8FE41
:10632000FFF79AF8BAF1000F3FF428AB5148FEF797
:1063300065FD5046FEF762FD4F48FEF75FFDFFF733
:106340001DBB4E48FEF75AFDA0461EAD20AC42468E
:106350004B49284605F09EF82846FEF74FFD494870
:10636000FEF74CFD404621461022FEF795F8002826
:106370003DD000270CE0E25D284605F08BF828466A
:10638000FEF73CFD01374048FEF738FD102F0BD0DB
:1063900007EB0803B3F5A27F3C493D48EBD9013731
:1063A000FEF72CFD102FF3D13748FEF727FD002311
:1063B00020212E2003EB0802B2F5A27F88BFE15412
:1063C00004D8E25C203A5E2A88BFE0540133102BE7
:1063D000F0D1002320468DF8903008F11008FEF728
:1063E0000DFD2C48FEF70AFDB8F5A87FAFD12A486D
:1063F000FEF704FDFFF7C2BA90E00008AC0C0020E5
:10640000A80B0020DCDE0008E0E60008D8EA00085F
:10641000E4EA0008E8EA000834EB000844EB00086E
:106420007803002064ED000858EB000848EB0008F2
:106430006CEB0008DCEA000874EB000894EB000841
:1064400028EB0008AC0B002008E20008A4EB0008D1
:1064500038EB0008D0EB0008F0E600086CE7000815
:10646000F8E6000878E70008E8EB000850EB0008C1
:10647000F8EB0008B4E7000854E90008CCE700088E
:10648000D4E70008DCE7000818E40008B8F40008C6
:10649000E8E70008ACE10008E0E7000864E600086F
:1064A000B34D0FCD3EAC05940FC495E80F0084E8C2
:1064B0000F00B048FEF76AFC044630B1AE49062230
:1064C00005F033F8002800F03282DFF830B30DF128
:1064D000E409AA48FEF79EFC25ACFEF7FFFC0598F0
:1064E0000821FEF7E1FD1AAD08941CAC4FF0000A3C
:1064F000079509942AAD20AC069556462FAF0DF1AD
:10650000D0081EAD05940BEB0A0C48F68904DCF8A4
:1065100004209B49CDF80CC0C8F68804A4FB0202F5
:106520005209099804F0B6FFDDF80CC09449DCF874
:106530000420A4FB02035B09C3EB0313A2EB830259
:10654000284604F0A7FF8F48FEF77CFF32468E49AD
:10655000079804F09FFF32468C49059804F09AFF93
:1065600032468B49089804F095FF324689490698CF
:1065700004F090FF32468849384604F08BFF3246DB
:106580008649404604F086FF0798FEF713FD5BF846
:106590000A2083490898C2F3C012FEF73DFE5BF85B
:1065A0000A207F490698C2F38012FEF735FE324674
:1065B0007C49484604F06EFF5BF80A207A48C2F333
:1065C000C204FEF71BFC0723224678494846FEF723
:1065D000CDFD7748FEF712FC32467649484604F076
:1065E00059FF5BF80A20704802F00704FEF706FC2A
:1065F000224607236D494846FEF7B8FD6C48FEF772
:10660000FDFB02246848FEF7F9FB6549099A0094EE
:1066100023463846FEF7E2FC6548FEF7EFFB62488A
:10662000FEF7ECFB5E4900942A4623464046FEF7FF
:10663000D5FC5F48FEF7E2FB01360598FEF71AFD30
:10664000FEF710FF082E0AF1080A7FF45CAFFEF790
:1066500059FD0026FFF792B9574F584D97E80700AC
:1066600007F13C040DF1D00888E807000FCC3EAEDE
:10667000503705960FC697E80F0024682F683460DE
:106680000DF1E40989E80F00002F00F02181DFF807
:1066900070B1FCF7FFFE0746FCF734FF05463548AE
:1066A000FEF774FB0446002800F0BE83444904F062
:1066B00022FF0346002800F0C2822046414904F030
:1066C0001AFF0346002800F0718320463E4903224A
:1066D00004F02BFF0646002800F06B8420463B495F
:1066E000062204F022FF0646002800F0B884204667
:1066F0003749072204F019FF0646002800F0968467
:1067000020463449042204F010FF0646002800F019
:1067100058852046304904F0EEFE0026B24610B9F6
:10672000DFF8E0A053262D48DFF8D4B0FEF772FB67
:106730000B24FEF7D3FB40460321FEF7B5FC2848A7
:106740002849294A294B019400970224FEF7D6FED6
:106750002749284A284B224801940095FEF7CEFE8F
:10676000FEF7D0FC05980521FEF79EFC002451E0C1
:10677000F0E00008E0E6000870ED000888ED000891
:10678000D8E6000814E2000864ED00089CED00085B
:10679000A4ED0008A8ED0008ACED0008B0ED00087D
:1067A00034E1000880ED000848E2000810000020F5
:1067B00050E2000884ED000890E00008740C00200E
:1067C00010EC000820EC000834EC000838EC00085D
:1067D00050EC000860EC000850EB000868EC000882
:1067E000E4E1000880EC000814EC0008800C0020B4
:1067F0008CEC000824EC0008780C0020B06200202B
:106800008800002078E6000801340B2C0BF1140BF3
:1068100000F0FB80DBF81030D807F5D52246B949E7
:106820001AA804F037FE2246B7491CA804F032FE2D
:106830002246B6491EA804F02DFE2246B44920A8DF
:1068400004F028FEDBF80820B24918A804F022FE64
:10685000B148FEF7F7FDDBF80000FEF7ABFB18A927
:106860001CA8AE4AFEF79CFD1EA8FEF781FDDBF8D2
:106870001020AB49C2F3400220A8FEF7CDFC1AA8B5
:10688000FEF7F8FBFEF7EEFDBEE7A6480999FEF716
:10689000ABFDFEF7D3BF2846A34904F02CFE002829
:1068A00034D10123CAF800305026A04CFEF7A8BF0F
:1068B0009F48FEF785FA002800F05582012645F032
:1068C00001050796CAF80050CDF824B04726A2E487
:1068D000984ADFF8C0B23B4653F80B101433DC2B58
:1068E00042F8041FF8D1944B94491A681B6981E857
:1068F0000C0001232B60CCE606460446FEF780BF61
:10690000DFF894A24E260446FFF7A1BA28468C4928
:1069100004F0F1FD002840F01D83CAF80000502665
:10692000884CFEF76DBF00263546FFF726BBA01D3D
:1069300004F06AFA072804463FF6C7AD01468248CC
:10694000FEF74CFA814904F0D6FD002800F0588388
:10695000DFF848B25BF8343023F080034BF8343072
:1069600021467B48FEF73AFA784904F0C4FD002836
:1069700000F03F835BF8343023F040034BF83430B1
:106980000DF1E40922467349484604F083FD484668
:10699000FEF7FCF904F038FA22466F4905464846EE
:1069A00004F078FD4846FEF7F1F904F02DFA5BF8A3
:1069B0003430ED0000F0070023F03F0340EA03020B
:1069C00005F0380313434BF8343021466348FEF793
:1069D00005FA04F019FA214605466148FEF7FEF96A
:1069E00004F012FA0BEBC404C5EB051500EB8500AF
:1069F000606003F051F86CE501F0A4FA594DFEF720
:106A0000F5BF06468346FFF72AB9FEF77BFB4846EB
:106A10000421FEF749FB544D00242B68D90700F1EF
:106A2000BF8001341035022CF7D1FEF76BFB3A48DA
:106A3000FEF7F4FC70E44D4B93E803003EAC059484
:106A400084E80300FFF7D9BA484B93E803000DF13F
:106A5000E40989E80300FFF7B0BA224644491AA8BE
:106A600004F018FD224643491CA804F013FD2246F9
:106A700041491EA804F00EFD55F8082C254914A81C
:106A800004F008FD3D48FEF7DDFC55F80C0CFEF760
:106A900091FA14A93A4A1CA8FEF782FC1EA8FEF738
:106AA00067FC1AA8FEF7E6FAFEF7DCFCFFF741B92F
:106AB0003448FEF76BF904F0A7F907463248FEF7B1
:106AC00065F982463148FEF761F90446002F00F06F
:106AD000B38104F022FD092800F2C8812C4CB24693
:106AE000FFF7B5B92AAC20460A49069404F0D2FC57
:106AF000FFF796BA2FAF3846064904F0CBFCFFF7F4
:106B000085BA00BF9CEC000840EC0008A4EC00082B
:106B100048EC000864ED0008E4E10008ACEC000873
:106B200034E1000854E70008F0E600083CE50008FE
:106B3000DCEA00087C0C002080010020780C00209A
:106B4000F8E6000854E5000878ED000810E10008B8
:106B50007CED000880ED000884ED000820E70008C7
:106B6000B4F000084CE600088C0100206CE5000839
:106B700058ED000804ED000860ED0008FCE1000895
:106B8000CCEB000804E8000810E80008DCF6000878
:106B900074E50008880000201CE60008B0620020B0
:106BA0002246BF4925A804F075FC2246BD492AA803
:106BB00004F070FC2246BC492FA804F06BFC55F889
:106BC000082CBA4916A804F065FCB948FEF73AFC4F
:106BD00055F80C0CFEF7EEF916A9B64A2AA8FEF7EE
:106BE000DFFB2FA8FEF7C4FB25A8FEF743FAFEF74C
:106BF00039FC16E7B048FEF7C9F804F005F903F0D0
:106C000057FC3546FFF7B9B92FAF3846AB49BDF849
:106C10003A2004F03FFCFEF7FFBEA948FEF7B6F8A5
:106C200003F0D2FE002800F0BB803446DFF8ECA26F
:106C3000FFF70DB901F06AF9A24DFEF7D7BEA248E1
:106C40000493FEF7A3F804F0DFF8CAF80000049BF1
:106C5000074641269A4666E59C48FEF797F804F0F9
:106C6000D3F803F08FFE002800F0AD803446DFF843
:106C7000B0A2FFF7ECB89648FEF7E4FB9548FEF7A4
:106C800099F98C4A94485946FEF78AFB9248FEF7D8
:106C9000F1F9FEF7E7FBFFF722BB059DCDF8009069
:106CA00001958B4806993A4634ABFEF74DFCFFF749
:106CB0001ABB8A48FEF76AF804F0A6F803F0EEFD66
:106CC0003546FFF75AB920AC2046784904F0E2FB7C
:106CD000FFF7DEBA824B83480A93FEF757F804F0B9
:106CE00093F80A9CAA462060FFF7A9BA7A48FEF7F3
:106CF0004DF804F089F862260990CAF80000FEF702
:106D0000AEBF484604F009FC774B09EB0002198836
:106D10009B7829F800109370FFF741B9059804F0AB
:106D2000FCFB714B3A1819889B7839529370FFF726
:106D300056B920466D4904F0DEFB002800F04C8176
:106D400020466B4904F0D7FB002800F0BC812046A8
:106D5000684904F0D0FB002800F05B81CDF824B036
:106D60000026FFF758BA25F001050790AAE520464E
:106D7000614904F0C0FB002840F00B81584D01230D
:106D8000CAF800305026DFF89CA10A95FFF757BAE1
:106D900026462546FEF72ABE06460546FEF726BECF
:106DA00006460446DFF880A1FFF751B85348049324
:106DB000FDF7ECFF04F028F8CAF80000049B054634
:106DC00046269A46AFE406460446DFF860A1FFF780
:106DD0003EB8434BCDF824B0064682460A93FFF7EF
:106DE0002EBA064604468246FFF731B84448FDF7FE
:106DF000CDFF04F009F88DF83C004248FDF7C6FFCE
:106E000004F002F88DF83D003F48FDF7BFFF03F0A6
:106E1000FBFF8DF83E000F9B1A0CAAF800308AF891
:106E200002206326FEF71BBF064682467BE425F060
:106E300002050990FFF7ECB93448FDF7EBFF344841
:106E4000FDF7DCFFFEF782F9FEF78AFA4FF4FA70DD
:106E5000FAF7F4FC2F4B6F6085F83C7050462146E2
:106E60001F603E46FDF7A8FEFEF722BC2748FDF74F
:106E7000D1FF2948FDF7C2FFFEF768F9FEF770FA67
:106E80004FF4FA70FAF7DAFC224B6E6085F83C603A
:106E9000504621461E60FDF7A7FEFEF709BC00BF65
:106EA000B0EC000858EC0008B8EC000864ED0008ED
:106EB000E4E10008CCEB000874E9000868EA000887
:106EC00098E800084CE6000814EC0008A8E8000860
:106ED00048EB0008B8EB000820FA000884E9000835
:106EE0007803002038EB0008A4E90008F4EA000861
:106EF00004EB000824EB0008F0E6000824EC00088E
:106F000010EB000814EB00081CEB000818E8000860
:106F10002CE80008C812002060E8000894E500088A
:106F2000DCE500083CE50008B8E50008FCE50008E1
:106F3000C248FEF787FAC248FEF73CF8C14AC24889
:106F400010A9FEF72DFAC048FEF794F8FEF78AFA6A
:106F5000FEF7D1BE2846BD4904F0CDFA0A900028BC
:106F600000F0D1802846BA4904F0C5FA044600284A
:106F700000F0358100263446FEF742BCB548FDF7E7
:106F800005FF03F041FF64260790CAF80000FEF7F2
:106F900066BE2046B04904F0AEFA002840F03E81BB
:106FA000AE4BCAF800005026DFF800A30A93FFF7A3
:106FB00046B9E01C03F028FF0A280AD800EB80003D
:106FC0000BEB800BB246DBF80C30CBF80830FFF748
:106FD000AABBB246FFF7A7BB9B48FDF7D7FE03F05D
:106FE00013FF42268046CAF80000CDF824B0FFF710
:106FF00012B95BF8343043F040034BF83430BFE44F
:10700000DFF8ACB25BF8343043F080034BF8343037
:10701000A6E49348FDF7BAFE03F0F6FE44260B9073
:10702000CAF80000CDF824B0FFF7F5B8E01D03F072
:10703000EBFE01280446CCD802468A492AA804F06F
:1070400029FA2AA8FDF7A2FE03F0DEFE0F28C0D819
:10705000854B03EB0414B2466060FFF764BBA01DD0
:1070600003F0D2FE0A288246B3D802467F4920ACFC
:107070001CA804F00FFA7E495246204604F00AFA92
:107080001CA8FDF783FE03F0BFFE431E0E2B4FEA44
:107090008A069CBF06EB0A030BEB8303564498BF9A
:1070A00098602046FDF78CFE0BEB860B002800F065
:1070B0002A81DBF81030002643F00203CBF81030B1
:1070C000B246FFF730BB6B48FDF760FE03F09CFE55
:1070D0008DF858006848FDF759FE03F095FE8DF8CD
:1070E00059006648FDF752FE03F08EFE8DF85A00F7
:1070F000169BCDF824B01A0CAAF800308AF80220AA
:107100004326FFF788B85E48FDF740FE03F07CFE9B
:1071100003465C480493FDF739FE03F075FE844690
:107120005948CDF80CC0FDF731FE03F06DFE044662
:107130005648FDF72BFE03F067FE0B905448FDF711
:1071400025FE03F061FE049B0C901A4651495846F7
:1071500004F0A0F9DDF80CC04F496246304604F057
:1071600099F922464C4914A804F094F94A490B9A1B
:1071700015A804F08FF948490C9A16A804F08AF96A
:107180000B9E049BDDF80CC0CAF808600C9ECAF880
:107190000C40CAF804600A9EA3F26C710CF1FF3235
:1071A000CAF81C10CAF81020CAF8006020466146D0
:1071B0001A46F9F795FF5426CAF818000A9CFEF7FC
:1071C0001FBB201D03F020FE01283FF602AF264B17
:1071D00003EB0013B2469A685A60FFF7A4BA2F482F
:1071E000FDF7D4FD1E220146504604F0B7F9702683
:1071F000FEF706BBE81D03F007FE0328054664D929
:10720000B346FEF72CBD2648FDF7C0FD03F0FCFD9C
:10721000FCF7E6F8B3460B90FEF721BD20460F4C75
:1072200020490A9404F067F91F4B00280CBF9A46C6
:107230004FF0000A08BF5326FFF701B8FCE1000831
:10724000B8EB0008CCEB000820FA000804E70008BF
:107250002CE70008D0EC0008F8E6000878030020CE
:1072600028EB000858EC00088001002040EC0008E2
:1072700048EC000810EB000814EB00081CEB0008B9
:1072800014E700081CE7000824E70008CCF9000810
:1072900028E70008D4E60008D8E6000830E7000830
:1072A000F0EC000850EB000878E6000854E5000810
:1072B000B06200201948FDF769FD03F0A5FDFCF759
:1072C00081F8B3460A90FEF7CABC024614491CA8CE
:1072D00004F0E0F81CA8FDF759FD03F095FD0F2818
:1072E0008ED807EB0515B3466860FEF7B8BC281DBD
:1072F00003F08AFD032883D807EB0013B3469A688E
:107300005A60FEF7ACBCDBF8103023F002030646EF
:10731000CBF810308246FFF706BA00BFE0EC000859
:1073200004ED000830B585B04FF480446846F9F7A5
:1073300067FB0022200448F2A063C0F20103012190
:10734000ADF80420ADF8082040F4B8404FF4806256
:107350004BF6FF75ADF80650ADF80A20ADF80C40BD
:107360000093F9F75BFB200440F4B8406946F9F755
:10737000D7FA05B030BD00BF10B54FF4B844C4F221
:10738000000420460121F9F765FB20460121F9F7A9
:1073900087FB20460021F9F783FB2046F9F788FA9E
:1073A000BDE81040FFF7BEBF70B505460E4643F27C
:1073B000010401E0013C13D04FF4B8402946C4F267
:1073C0000000F9F781FB0028F4D04FF4B840C4F274
:1073D00000003146F9F778FB0028EBD0012070BDA2
:1073E000FFF7CAFF204670BD38B5054619B1BDE8A4
:1073F0003840FFF7D9BF43F2010401E0013C0AD055
:107400004FF4B840C4F200002946F9F75DFB0028AC
:10741000F4D0012038BDFFF7AFFF204638BD00BFD4
:10742000F8B507464FF4B840C4F200000E460121FB
:1074300015461C46F9F700FB0120C1F200000021AF
:10744000FFF7D2FF002832D04FF4B840C4F200005A
:1074500034BB0121F9F716FB4FF4B844C4F2000421
:107460002046F9B20022F9F703FB0220C1F2000026
:107470000021FFF7B9FFB8B18020C1F20000002160
:10748000238BFFF7B1FFA8B125B1C6F30721204632
:10749000F9F714FB2046F1B2F9F710FB0020F8BD14
:1074A0000021F9F7EFFAD7E76FF00100F8BD4FF0D0
:1074B000FF30F8BD6FF00200F8BD00BF30B5284BBB
:1074C0001C6883B00CB103B030BD012568461D6057
:1074D000F9F7C0F929464FF40000F9F777FB284681
:1074E0002946F9F765FB04202946F9F761FB29468F
:1074F0004FF40000F9F786FB21464FF40000F9F73E
:1075000081FB002008210422C4F20200F9F7B8F937
:107510004FF4006004220921C4F20200F9F7B0F927
:107520000223002069468DF804308DF80530C4F23E
:1075300002004FF4807300938DF806508DF80740D9
:10754000F9F72CF94FF400604FF40073C4F2020015
:1075500069460093F9F722F9FFF7E4FEB3E700BFAD
:10756000B40C00202DE9F041069D6F1E1E467B42A3
:107570007B418046FFF754FF074610B13846BDE80F
:10758000F08180200421C1F20000C1F20001FFF768
:107590000BFF00285BD04FF4B844C4F2000420462F
:1075A0000121F9F749FA0120C1F200003946FFF73D
:1075B0001BFF00284ED020465FFA88F10122F9F720
:1075C00057FA0220C1F200003946FFF70DFF0028EC
:1075D00043D0238B8DB33C4611E040200021C1F203
:1075E0000000FFF701FF18B34FF4B840C4F20000E9
:1075F000F9F766FA3219AC4202F8010C1DD00134D9
:10760000AC42EAD14FF4B840C4F200000021F9F7CF
:1076100039FA4FF4B840C4F200000121F9F71AFA20
:1076200040200021C1F20000FFF7DEFE0028DBD180
:107630006FF006073846BDE8F0814FF4B840C4F259
:1076400000000121F9F71EFA3846BDE8F0816FF01D
:10765000030793E76FF0040790E76FF005078DE7E6
:1076600070B51C460023FFF7DBFE064608B1304626
:1076700070BD8020C1F200003146FFF7B5FE28B38F
:10768000049BD3B1049BE51801E0AC4215D04FF444
:10769000B84014F8011BC4F20000F9F70FFA80207B
:1076A0000421C1F20000C1F20001FFF77DFE0028B5
:1076B000EBD16FF00306304670BD4FF4B840C4F212
:1076C00000000121F9F7C6F9304670BD6FF00206DF
:1076D000CDE700BF70B43A4A3A49546A0B689C42FD
:1076E00007D8956AAB4204D2D56B002D4FD0364DEA
:1076F00013E0D46A324DA34208D21268032A15D08F
:10770000052A20D001330B6070BC70472E6BB3424A
:10771000F3D2ED6B002D40D02C4D2E681C1B00FACF
:1077200004F426432E601268032AE9D1102BE9D90C
:10773000142BE7D8264AA3F11105146800FA05F0C6
:1077400004431460DEE7A3F11402032A16D9A3F15F
:107750001804032C27D81F4C256800FA02F21543A1
:107760002560DA0810BB1C4803F00704855C01267D
:1077700006FA04F425EA04048454C3E7134AA3F187
:107780000805146800FA05F52C431460E9E70E4C6F
:10779000256840EA45052560AFE70C4C256840EABE
:1077A00045052560A9E72F2BACD8DAE70A4803F096
:1077B0000704855C012606FA04F42C438454A1E7EF
:1077C000E00C0020C80C0020240D0020400D0020FB
:1077D000380D00203C0D0020B80C002000B583B00F
:1077E0006846F9F737F804200121F9F7E1F94FF479
:1077F000006000234FF48062C4F2020069460092E8
:107800008DF804308DF805308DF806308DF807308E
:10781000F8F7C4FF03B000BD70B4294A1368002B09
:107820002BD028490B68022B17D0032B264B26D0D0
:10783000264C0E682168264DA0F8011019680670C4
:10784000A0F803102E680021196046712160012004
:1078500029600023136070BC70471B4B1D681C68B7
:10786000E443E4B2B4EB152F1BD0184C266848F261
:10787000EE75AE421AD00020EBE71846EBE71D6824
:107880001C68E443E4B2B4EB152FF4D11D680F4C2F
:10789000EDB21D600F4D2E681D6845EA06251D607E
:1078A000C7E71D68094CEDB21D60C2E70B250D60EE
:1078B0001D68C5F3072525601D68EDB21D60B8E79A
:1078C000480D0020C00C0020C40C00202C0D00200E
:1078D000300D0020D00C00202DE9F0474FF400605F
:1078E0009E4CC4F202004FF48061F8F7BDFF23689C
:1078F00093B99B4E356895B99A4B002800F0C28029
:107900001B68002B40F00C81974B1A684FF6FE71F4
:107910008A4201D801321A602068BDE8F087934F8F
:107920003A68002A70D0002800F0B280904A11789E
:107930000131C9B2E929117000F206818D4B8E49DF
:107940005A6B09688A42E7D1996B0029E4D1DFF8C4
:1079500068828A49D8F800C00D68AC4500F078818B
:107960008748002707601B68012B00F06481052B06
:1079700000F079810A2B18BF292B03D10068C007BA
:1079800000F155810120022B206040F09C81002AEB
:1079900040F0028274480368B3F5E16F80F016820C
:1079A000784D794FD5F800903B68DFF8F4A1C1F825
:1079B00000C049F00109C5F80090CAF80030026023
:1079C0006546724A3B6002201060714A1360714B39
:1079D0001A68714B1D60714B1A60236863B10B68A4
:1079E0009C4500F0BA816E4A5F481568664FC8F83A
:1079F000003000233D6003605A4A002313605C4A54
:107A000033600B60137087E7664F3B68002B00F014
:107A10008180584B002840F0D1801A68032A00F07A
:107A20005581DFF84C81DFF83C915A68D9F8001095
:107A300050488A420BD88268914208D898F800C012
:107A4000C268944503D30269944540F2B3815B69EF
:107A5000484A99420BD39369994208D898F8001084
:107A6000D369994203D3136A994240F2A981002550
:107A7000356088F800500123C9F80030002D3FF42C
:107A80004BAF5BE71A6801321A602068BDE8F087E7
:107A9000DFF8D090DFF8D880D9F80030A3F11F02CA
:107AA0000A2A17D898F80020052A13D90A2A11D8CB
:107AB0003D493048442203F003FA2F4A0023136063
:107AC0000122C9F8002088F800303B60002D3FF407
:107AD00023AF33E7A3F15E02532A08D898F80020B9
:107AE0002D2A00F29F80162A01D93049E1E7A3F13F
:107AF0003C020F2A40F28980283B162B00F28F802F
:107B000098F80030122B40F28A801F2B00F28780F9
:107B10002749CEE7E8B9134B1A6801321A600DE71E
:107B2000204B124A1D6001231360144A3360156014
:107B30001B4A15601F4A1560164A15600E4AFF2140
:107B400011600B4A1370E7E6064933600B6013704F
:107B5000E2E6074A01233B601370EFE6480D002080
:107B6000CC0C0020440D0020D40C0020280D002057
:107B7000DC0C0020E00C0020C80C0020400D002090
:107B8000340D0020300D0020B0010020C00C00207A
:107B90002C0D0020380D0020C40C0020D00C00203B
:107BA000240D0020D80C00206CEE000838EF0008EF
:107BB000B0EE00083C0D0020AC0100208C49D3F849
:107BC0003490D1F800C0E14500F09180DFF8548294
:107BD0001A6898F800A087480AF1010A5FFA8AFA41
:107BE000012A88F800A000F09A80BAF1E90F7FF628
:107BF00045AF09F1FF32944500F0C4807E4A00236E
:107C00003360136088F8003086E698F800203B2A3D
:107C10007FF672AF4B2A3FF66FAF784949E70025F0
:107C200035604AE7592A3FF662AF754941E7754822
:107C300000230360D1E60268013A012A88BF23606D
:107C4000F5D9714A714812680360714B1A60BEE63B
:107C50006C480068B0F5966FBFF482AE6D48076857
:107C6000013707607FE60368012BE0D00123236022
:107C7000694B1F7858789A7887EA000909F00F094C
:107C800089EA171787EA101002F00F09814501D021
:107C90000020206093F803901F79587982EA090345
:107CA0007B40984201D0002323605C4B5C4A1F68F4
:107CB0001068554A38431860544B12680520186004
:107CC000534B1A6083E6052BD2D0BAE748490A68BD
:107CD000102A7FF4A6AEDFF82091D9F80020053AEB
:107CE000072A79D94F4B306018700546C3E6986B68
:107CF00001287FF46BAFDFF800915869D9F80010C4
:107D0000884205D89869814298BF9A637FF6B6AEDB
:107D1000444A00233360C9F800301370FCE5BAF11F
:107D20000B0F7FF6ABAEBCF10A0F7FF65EAFDFF84C
:107D3000D890C16AD9F80020ACF10B0A614442EA3C
:107D40000A220CF1010C0131C9F800200A22C0F806
:107D500034C0016388F8002065E62B48324F05687F
:107D60003A682848AA427FF442AE026840F6C90C3D
:107D700062459FBF294AD2F800C04CF0010CC2F8FE
:107D800000C034E69B6B002B7FF438AFC1F8009045
:107D9000002D3FF4C1ADD1E51B4B234F1B6810E60E
:107DA0000A200F3A2021186010200F2AD862196388
:107DB000596305D80120FFF78DFC00233B605AE68C
:107DC0000020FFF787FC00233B6054E6174B164F5B
:107DD0001A600D4B1B68F4E5124A12783B2ADFD972
:107DE0004B2ADDD800233B6011230B6043E600BF24
:107DF000C80C0020E00C0020440D00207CEF00089F
:107E0000F4EE0008D40C0020240D0020C00C00204B
:107E10002C0D0020340D0020B80C0020300D002067
:107E20003C0D0020DC0C0020B0010020480D00209B
:107E3000F9F72AB910B582B004460DF10600F9F73A
:107E400031F978B1084B09491B88BDF8062009882B
:107E5000D21AC2EB0212CB1A92FBF3F30F2B28BFFC
:107E60000F23236002B010BD4C0D00204E0D0020EA
:107E700008B50F4B1B686BB1FF23C0F20203984299
:107E80000AD80C4B00221A800B4B40F2FF321A80AA
:107E9000012008BD184608BD02220649E120FCF772
:107EA000FBFAE32004490222FCF7F6FA012008BDA0
:107EB000A40400204C0D00204E0D002008B50A4BF4
:107EC0001B680BB9002008BDE12008490222FCF71D
:107ED000FDFA0028F6D00222E3200549FCF7F6FA65
:107EE000003018BF012008BDA40400204C0D002064
:107EF0004E0D002040F64C53C2F200031888704724
:107F000040F64E53C2F200031888704710B582B095
:107F1000F9F7BAF80A240DF10600F9F7C3F840B9E9
:107F20000A20F9F78BFC013CF5D1054C208802B002
:107F300010BD034CBDF806302380FFF7BFFFF5E707
:107F40004C0D002010B582B0F9F79EF80A240DF10F
:107F50000600F9F7A7F840B90A20F9F76FFC013CD1
:107F6000F5D1054C208802B010BD034CBDF8063099
:107F70002380FFF7A3FFF5E74E0D0020F9F72AB89D
:107F8000F0B507468DB00A20FCF796FC092828D0EA
:107F90000A2813D0072803D0002420460DB0F0BDD6
:107FA000FCF7E0FD0A2201A900F5B67003F004FC1D
:107FB0000146384602F01AFD7424EEE7FCF7D2FDC4
:107FC00000F14C042021204603F088FA014610B14C
:107FD000002301F8013B20463A46FDF7EDFA04463E
:107FE000DBE7FCF7BFFD01AE00F5A674002502E05B
:107FF00002340A2D12D0237820460221002B7BD098
:108000006378002B78D0F9F7A5F8A37846F8040F29
:108010000135202BECD103340A2DECD1029CA4F1C4
:1080200041032F2BB8D801A252F823F0ED800008AD
:10803000ED80000847810008ED800008997F000866
:10804000ED800008ED800008997F0008997F000806
:10805000997F0008997F0008ED800008997F00084B
:1080600001810008997F0008ED800008997F0008D1
:10807000997F00080181000821810008997F00088C
:10808000997F000801810008997F0008997F000806
:10809000997F0008997F0008997F0008997F000860
:1080A000997F0008997F0008997F0008997F000850
:1080B000ED80000847810008ED800008997F0008E6
:1080C000997F0008997F0008997F0008997F000830
:1080D000997F0008997F0008997F0008997F000820
:1080E000997F0008997F000809810008022D7FF41C
:1080F00053AF039B3B6050E7002D3FF44DAF8DE73E
:10810000012D7FF449AF48E73846202300F8013BB2
:108110000DF109011E2203F021FA0023FB773CE751
:10812000072D7FF439AF059BFB60039B03F16402CD
:10813000049B7A61013B3B61069BBB60079B7B60B4
:10814000089B3B6029E7042D7FF426AF039B3B701F
:10815000049B7B70059BBB701FE700BF70B53E4B57
:108160001A68824288B0064673D002A81E60F8F7EB
:1081700071FB04A8F8F7B4FE01200146F8F718FDDA
:1081800001200146F8F714FD4FF400300121F8F703
:108190001DFD0020C4F2020002210722F8F770FB47
:1081A00000200722C4F202000321F8F769FB022332
:1081B00000208DF80C30032304460125C4F2020090
:1081C00002A98DF80D30042302938DF80E408DF82E
:1081D0000F50F8F7E3FA20460823C4F2020002A980
:1081E0000293F8F7DBFA4FF48840C4F20000294606
:1081F000F8F790FE4FF488400C23C4F2000004A965
:10820000ADF81A300496ADF81440ADF81640ADF84C
:108210001840ADF81C40F8F7F7FD4FF48840C4F261
:1082200000002946F8F768FE4FF48840C4F20000C9
:1082300040F225512A46F8F783FE262301A88DF83F
:1082400004308DF805408DF806408DF80750F7F79B
:10825000FFFF08B070BD00BF680F002030B40F4AA8
:1082600013687F2BFCD80E490E4D0B685C1C7F2CCD
:1082700045F8230098BF0C6001D900230B6072B64B
:1082800013680133136062B64FF48840C4F20000F3
:1082900040F22771012230BCF8F752BE640F002073
:1082A000600F0020580D002010B50446007828B15A
:1082B000FFF7D4FF14F8010F0028F9D110BD00BF5B
:1082C00030B40D4B1A6882B10C490D4D0A68541C2C
:1082D000802C55F8225018BF0C6009D072B61A686D
:1082E000013A1A6062B601220560104630BC704740
:1082F00000220A60F2E700BF540D0020500D00205C
:108300006C0F0020024A1368002BFCD1704700BF9D
:10831000640F00204FF4884038B5C4F2000040F2EA
:108320002551F8F729FE00282BD14FF48840C4F2DC
:10833000000040F22771F8F71FFE00B938BD4FF476
:108340008840C4F2000040F22771F8F73BFE234B4F
:108350001A68002A38D0224A224C1168481C80280A
:1083600008BF002054F8211010601A684FF48840AC
:10837000013AC4F2000089B21A60BDE83840F8F74B
:10838000D7BD4FF48840C4F2000040F22551F8F701
:1083900019FE4FF48840C4F20000F8F7CDFD124BEF
:1083A0001A687F2AC1D81149114D0A68541CC0B2FD
:1083B0007F2C45F8220098BF0C6001D900220A608A
:1083C0001A6801321A60B0E74FF48840C4F2000026
:1083D00040F22771BDE83840F8F7B2BD640F0020C5
:1083E000580F0020580D0020540D00205C0F002075
:1083F0006C0F002010B541F26C14C2F2000402466A
:108400000B4620464FF4807103F000FD2046BDE886
:108410001040FFF749BF00BF0FB400B583B004ABF5
:1084200053F8040B19460193FFF7E4FF03B05DF81E
:1084300004EB04B0704700BFFFF790BE10B584B0E6
:1084400001A8F8F739FC01200146F8F7BFFB00232B
:10845000ADF80C30ADF80630072301A902934FF0B8
:10846000804003F52D73ADF80430F8F7D9FB0121F6
:108470000A464FF08040F8F7AFFC01240F2368460E
:108480001C228DF800208DF803408DF801308DF806
:108490000230F7F7DDFE4FF080402146F8F724FC6C
:1084A00004B010BD38B54FF080400121F8F79EFCB4
:1084B0006A4B1C68002C34D0694B1A6843F698212B
:1084C00001328A421A6000D038BD664C6649674A5C
:1084D000012020600C6824180C60116809181160D4
:1084E000146800213C2C1960EED1614B11601A68B0
:1084F00012181A605F4A10601A683C2AE4D15E4A7A
:10850000196013681B1813601368182BDCD15B4BC0
:1085100011601A6812181A601A68072AD4D11960F3
:1085200038BDFFF7D9F950490B68012B07D9544BD7
:108530001A6840F6A660013282421A6043D0514B5D
:108540001A680132EA2A1A6054D04F4B1A68013275
:10855000962A1A6048D04D4B1A680132962A1A6042
:108560003CD04B4B1A6801320F2A1A6030D03C4B7A
:108570001A6843F69820013282421A60A4D1394C1D
:108580003A4A012020600C6824180C601168091810
:108590001160116800242D291C6031D01268334B02
:1085A0003C2A38D01B681E2B53D03A4B1A68002A3D
:1085B0008AD01A68013A1A601B68002B84D1364BA6
:1085C00001221A6080E71C60344B01221A60B6E772
:1085D000334A0120106000221A60C8E7314A0120A6
:1085E000106000221A60BCE72F4A012010600022B0
:1085F0001A60B0E72D4A0120106000221A60A4E73B
:108600002B4B1B491C680D68AC421FBF09681960E1
:10861000284B1860C2E7164A00211960136801331D
:108620001360144B0120186013683C2BBDD1124B12
:1086300011601A6812181A601A68182AB5D10F4A00
:10864000196013681B1813601368072B08BF1160AB
:10865000ABE7194B01221A60A7E700BFB812002050
:108660009412002074120020C012002080120020FA
:10867000CC12002088120020A412002078120020C2
:10868000B4120020BC120020B01200206C12002096
:1086900070120020B401002098120020A8120020BF
:1086A0008462002088620020A0120020C4120020F2
:1086B000C0010020901200208C1200204EF6C070E5
:1086C000C0F60000704700BF40F2B813C2F20003CA
:1086D0001868704741F2A42141F2CC2241F2802374
:1086E000C2F20001C2F20002C2F2000346F28C2084
:1086F000C2F20000096812681B6881604260036072
:10870000704700BF2DE9F04F9FB001F07FFF02F0EE
:1087100025F84FF4E130FFF78FFEFFF75FF801F027
:108720003DFB01F067FBFFF789FE0120F9F7AAF88E
:10873000F8F74AFDF8F768FD01F01AFDFBF784FE33
:10874000F8F77CFD002841F00A81BE48DFF830933D
:10875000FFF7AAFDBC48FFF7A7FDBC48FFF7A4FD43
:10876000B948FFF7A1FDBA48FFF79EFDB948FFF7EA
:108770009BFDB548FFF798FDD9F80030002B01F0BC
:108780009680B548FFF790FDAF48FFF78DFDB34DDC
:10879000FBF772FD2B68002B01F08080B048FFF7DB
:1087A00083FDA948FFF780FD2B68002B41F0B480C2
:1087B000AC4CAD482168FFF72FFE226822F47F03FE
:1087C00023F47F43EBB940F2FF43C0F201039A4226
:1087D00001F2E38040F2FF632268C0F201039A4293
:1087E00001F2D180A148FFF75FFD9748FFF75CFDDC
:1087F000206802F013F8206801F01AFE2068FFF7E5
:1088000037FBFFF7BBFBF8F75BFD01F0ADF941F279
:10881000B820C2F200000123036002F049F841F2DF
:10882000B821C2F2000100260E60FAF7B7FCFAF791
:10883000DFFD41F27C22C2F2000241F29C2A10606C
:10884000FAF728FE41F2AC23C2F20003C2F2000A9A
:108850001860FAF757FECAF80000FAF7FFFD41F278
:10886000842EC2F2000E2B68CEF8000083B34FF4C2
:10887000807523687B4FC0F20205AB4228D07C484C
:108880002946FFF7C9FD754B3D601B68002B41F081
:10889000B7807848FFF708FD6B48FFF705FD01F04A
:1088A0001FFC002801F0A480FBF7B6FB002801F0B4
:1088B000978002F033F8002801F08A8001F0ECF88C
:1088C000002801F058804FF48073C0F20203236047
:1088D00041F29021C2F2000141F2C0220120C2F215
:1088E000000208601468014602460334FAF738FCB7
:1088F00041F2C025C2F200050BA82B689C421ED98C
:10890000FEF78AFF0028F3D000210A460120FAF77B
:1089100027FC0120F8F7A0FF0BA8FEF77DFF002041
:1089200001460246FAF71CFC5348FFF7BDFC4648D7
:10893000FFF7BAFC01F0DAFA08B101F0D1FB002030
:108940000146024606460890FAF70AFCFCF7D0F901
:10895000FCF708F94FF0010A0696089ECDF81CA016
:10896000DFF82081454F059600F13C0A8346042537
:108970003446CDF824A015A8FFF702FB8246002854
:1089800040F02D81D8F800303BB141F28422C2F290
:1089900000021368002B40F02F86069E002E40F048
:1089A0009783DBF80030002B40F0D3853348F8F78D
:1089B00053FC002840F0A08341F29020C2F2000056
:1089C00003685BB1D9F80030002B40F0CC8541F250
:1089D000902EC2F2000E0023CEF80030D8F80030FE
:1089E0006BB141F28420C2F2000003683BB141F256
:1089F000A821C2F200010B68002B40F08E8641F2E4
:108A00009822C2F20002136893B1DBF80430002B05
:108A100040F0318641F29826C2F2000640F2B41AC4
:108A20000023C2F2000A336040F6D863CAF800306F
:108A300041F2882EC2F2000EDEF80030002B40F02A
:108A4000A38321E0C8EF0008ACE10008E8EF0008CC
:108A500008F00008C0EF000814F00008A40400208B
:108A600034F00008B801002048F0000800F10008C8
:108A70003CF1000860F1000820F200088C62002040
:108A8000541300206061002041F28C20C2F20000EB
:108A90000368002B00F0708240F2783AC2F2000ABC
:108AA000AF4ADAF8003000211160002B00F0648238
:108AB00041F2CC2EC2F2000EDEF80020B2FBF3F140
:108AC00003FB1123002B40F0578240F29040C2F28A
:108AD00000000368002B40F0B185D9F80030002B6E
:108AE00000F01F8501F0EEFC9E4B9F4A064616F0F3
:108AF000010F9E484FEA560118BF1A46FFF78CFC3B
:108B0000FF2E0AD03046FBF77DF841F2C02EC2F2AC
:108B1000000EDEF8003006330893002D40F040824E
:108B200041F2C425C2F200052B68002B40F071828F
:108B300041F2742AC2F2000ADAF80030002B40F049
:108B40007B8241F2A020C2F200000368002B40F0BB
:108B5000868201F089F9FF28054600F08B8200210A
:108B60000A460120FAF7FCFA132D00F2A886DFE886
:108B700015F0B901E301D101F0018401B0019601C2
:108B80006A0132011301EA00DD00D000C300A90030
:108B9000B60094007F00A60614007548FFF784FB1A
:108BA0007448FFF781FB0126322405960025069EB6
:108BB000DDF81CA016EA0A0F52D1002C3FF4DBAE00
:108BC000013C7FF4D8AE204621462246FAF7C8FA87
:108BD00015A8FFF7D5F9824600283FF4D3AE00214F
:108BE00001200A46AAF1410AFAF7BAFABAF1330F9C
:108BF00000F21883DFE81AF060044D0448043204E0
:108C000016037B04FD0316030B0316031603DC0394
:108C100016039D0316038503160316037A03220326
:108C200016031603D103C603160316031603160311
:108C300016031603160316031603BB03AC036F03D8
:108C4000160316031603160316031603160316035C
:108C500016031603160364031603160316031903FB
:108C6000F8F7ECFA002840F0148501260796A4E7EF
:108C70004148FFF719FB3F48FFF716FB41F28426F6
:108C8000C2F200063368002B40F0CF850025FAF7CA
:108C90000DFF32240595022589E73848FFF704FBCC
:108CA0003448FFF701FB41F28426C2F20006336824
:108CB000002B40F0AB850025FAF7EEFE3224059537
:108CC000022574E72E48FFF7EFFA2A48FFF7ECFA7F
:108CD0000025FAF777FE32240595022567E7294833
:108CE000FFF7E2FA2348FFF7DFFA0026FAF75AFE09
:108CF0003224059602255AE72348FFF7D5FA1D4886
:108D0000FFF7D2FA0026FAF72DFE32240596022547
:108D10004DE71E48FFF7C8FA1648FFF7C5FA0025C9
:108D2000FAF730FE32240595022540E71848FFF790
:108D3000BBFA1048FFF7B8FA0026FAF7F3FD322421
:108D40000596022533E71348FFF7AEFA0948FFF707
:108D5000ABFA0025FAF7F6FD32240595022526E741
:108D60008C120020A4E9000834E1000880F6000815
:108D7000D0F80008ACE10008B4F8000898F8000842
:108D800058F8000878F8000834F8000810F80008CF
:108D9000F0F70008D0F70008B848FFF785FAB848A0
:108DA000FFF782FA41F2CC23C2F200031A68B54BF6
:108DB0003A2A00F2E0841A6801321A6041F28024F3
:108DC000C2F2000400232360D9F80060FEB9322407
:108DD00005960425EBE6AC48FFF766FAA848FFF7CE
:108DE00063FA41F2CC21C2F20001A64B0A68002AC4
:108DF00000F0CD841A68013A1A6041F28022C2F272
:108E00000002D9F8006000231360002EDFD041F289
:108E1000A42A41F2CC2E41F28020C2F2000EC2F20E
:108E20000000C2F2000A0025DAF80010DEF8002087
:108E300003689648B9607A603B60322401F0F4F927
:108E400005950425B3E69248FFF72EFA8C48FFF704
:108E50002BFA41F2A42EC2F2000E8E4BDEF8002057
:108E6000162A00F28C841A6801321A6041F28020BE
:108E7000C2F2000000230360A6E78748FFF714FA58
:108E80007F48FFF711FAFAF71FFB41F2AC26C2F256
:108E900000060025059532243060042587E67F48CA
:108EA000FFF702FA7648FFF7FFF941F2A426C2F273
:108EB0000006784B3268002A00F065841A68013A8F
:108EC0001A6041F2802AC2F2000A0023CAF8003078
:108ED0007AE77348FFF7E8F96948FFF7E5F9FAF729
:108EE000E7FAD2E76F48FFF7DFF96548FFF7DCF9EB
:108EF00040F27013C2F200031D68D5F1010538BFBE
:108F0000002500261D6032240596B5420CBF1425AD
:108F10000C254CE66448FFF7C7F95948FFF7C4F938
:108F2000FAF78CFA41F27C25C2F20005002628608F
:108F30003224059604253AE65C48FFF7B5F9504817
:108F4000FFF7B2F900240594FBF766F83224059D7B
:108F50002DE65748FFF7A8F94948FFF7A5F9FAF7B2
:108F60005BFA41F27C2AC2F2000A00250595322400
:108F7000CAF8000004251AE6059E002E7FF4A5AD70
:108F8000089E002E3FF4C9AD41F2C02AC2F2000A89
:108F9000DAF80030B342FFF4C0AD059E0425089610
:108FA00041F27C2A4348C2F2000AFFF77DF93448B7
:108FB000FFF77AF9DAF80030112B40F0BA8240F26C
:108FC000904EC2F2000EDEF80030002B40F0B58368
:108FD000D9F80030002B00F0A78301F073FA364B6C
:108FE000364A064616F0010F4FEA5601344818BFBC
:108FF0001A46FFF711FAA6F114012A4641F2C425D8
:10900000C2F200050020FAF7DBF82B68002B3FF4D2
:109010008FAD40F27016C2F2000641F2742A294B5D
:109020003068C2F2000A00221A60FAF743FBDAF84D
:109030000030002B3FF485AD234B41F2802E0022FF
:10904000C2F2000E1A60DEF80000FAF773FA41F27D
:10905000A020C2F200000368002B3FF47AAD1B4B46
:1090600000221A60F8F766F900F0FEFEFF280546B8
:109070007FF475AD00260596354698E5B8F70008EB
:10908000ACE10008CC120020A0F700088C620020A0
:1090900088F70008A412002030F7000870F70008D5
:1090A00050F70008D0F60008F0F60008E0F60008D7
:1090B00010F70008C0F60008A4E9000834E1000831
:1090C00080F60008C412002074120020A0120020B4
:1090D00041F2C82AC2F2000ADAF8003023B9DBF8FC
:1090E0000430002B40F0FB820126C7480696F8F7B3
:1090F000B3F800283FF460AC012001460022FAF7E3
:109100002FF8D9F80030002B40F0BF8241F2A42A9A
:10911000C2F2000ABC68DAF80030BB4A9C4200F098
:10912000D282D2F804E0042540F21000B9693E6909
:10913000D7F800C07A69C2F2000041F2782A50F8EC
:109140002130F868CDF80CC0C2F2000A8DE8114059
:10915000CAF80010194641F2CC2A731C41F2A42629
:10916000C2F20006C2F2000A3460CAF800E041F21E
:10917000802EC2F2000EA548CEF800C002F26C723A
:10918000FFF74AF9322417E4A14B00221A6041F29A
:10919000782041F2A422C2F20000C2F2000241F2A1
:1091A000CC25C2F20005016813682A68994D40F287
:1091B0007016C2F20006C3EB0313306802EB8302A1
:1091C00000F096FC002800F0148241F2A42A41F23B
:1091D000CC2E2968DFF860C28F48C2F2000AC2F2C2
:1091E000000EDAF80020DEF80030D1F1010E38BFB1
:1091F0004FF0000E8949C5F800E0BEF1000F08BF2E
:1092000061460CBF14250C25FFF706F93CE48448A1
:10921000FFF74AF88348FFF747F800F067FE002899
:1092200040F07A813224FFF7ADBB159B40F2B414B5
:10923000C3F56E63C2F2000402332360D9F8003034
:10924000002B40F0018341F2A426C2F20006179CD5
:1092500033689C4200F0FC82DDF858E0042540F2BF
:1092600010001B9B189ADDF854C0C2F2000041F2B6
:10927000A42650F82310009241F2CC2A41F2782221
:10928000C2F20002C2F20006C2F2000A0194CDF856
:1092900008E0CDF80CC013603460CAF800E041F279
:1092A000802E1A9A199B6048C2F2000E02F26C726C
:1092B0000133CEF800C03224FFF7AEF8FFF762BBEF
:1092C00015A8FAF747FC594815A9FFF7A5F8042592
:1092D0003224FFF757BB1598FAF75AF8014654485D
:1092E000FFF79AF804253224FFF74CBBFAF794FEF7
:1092F0005048FEF7D9FF4B48FEF7D6FF3224FFF760
:1093000041BB40F27010C2F20000159B026893420C
:1093100088D0404A41491360002B474B474808BF5B
:10932000194614BF0C2514253224FFF775F8FFF7F2
:1093300029BB41F29821C2F20001012340480B6091
:10934000FEF7B2FF3748FEF7AFFF3224FFF71ABB34
:1093500015A8FAF777FB3B489DF854109DF8552067
:109360009DF85630FFF758F83224FFF70BBB1598DD
:10937000FAF7AEFB34481599FFF74EF80225322470
:10938000FFF700BB3148FEF78FFF2648FEF78CFF42
:109390003224FAF7A9FBFFF7F5BA2D48FEF784FF50
:1093A00001242048FEF780FF05943224FFF7EABA33
:1093B000159B002B00F0588241F2842AC2F2000A69
:1093C00024480123CAF80030FEF76EFF1548FEF767
:1093D0006BFF41F28421C2F2000140F2BC12C2F2E2
:1093E0000002FF23086813603224FAF73DF8FFF704
:1093F000C9BA1598F9F7A8FF17481599FFF70CF89F
:1094000004253224FFF7BEBA8C620020E0F5000884
:10941000881200207001002038F600080CF90008BE
:1094200034F50008ACE10008DCF400086CF5000835
:1094300024F300084CF5000820F90008E8F20008C1
:1094400014F50008BCF200080CF40008C0F4000891
:1094500098F3000838F4000898F4000841F27C21E1
:10946000C2F2000115980B6898423FF4DBAEF9F7A1
:10947000C5FFCE4A03460146CD4813600425FEF7DA
:10948000CBFF3224FFF77EBA15A8FAF7B7FAC9481E
:1094900062E741F28425C2F200052B68002B40F000
:1094A000F0811598FAF7ECFAC3481599FEF7B4FF66
:1094B00002253224FFF766BA41F2AC22C2F2000262
:1094C0001598136898423FF4ADAEF9F7E9FF41F201
:1094D000C424BA4B0146C2F200041960B848002304
:1094E00023600425FEF798FF3224FFF74BBA41F2C0
:1094F0009C26C2F200061598336898423FF492AE5B
:10950000FAF706F8AF4A03460146AF481360322423
:10951000FEF782FFFFF736BA00F0E2FD3224FFF7D4
:1095200031BAAA48FEF7C0FEA948FEF7BDFEFFF714
:10953000F4BA41F2A42E41F2CC22C2F2000EC2F2E1
:109540000002DEF8000011682A46F9F739FEFFF73D
:10955000E7BAA048FEF7A8FE01269D48FEF7A4FE44
:109560000696FFF723BADFF884A2504600F0E8FE23
:1095700000283FF42CAA41F2A421C2F20001DAF83B
:1095800008E00B689E4500F00681DAF804C0042567
:1095900040F21006B969F868C2F2000641F278227A
:1095A00056F821307E69CDF808C08DE80140C2F23E
:1095B0000002386841F2CC2A0390116006F26C7206
:1095C00041F2A426C2F20006C2F2000AC6F800E088
:1095D000CAF800C041F2802A19463E683B697E48BD
:1095E000C2F2000A0133CAF80060FEF715FFFFF768
:1095F000EEB90425FFF748BA0AA8FEF71BFC0028BD
:109600003FF4CBA940F2BC13C2F200030A9A1968D6
:10961000531C8B4203D34B1C9A427FF6BEA96F4862
:10962000FEF7FAFE40F2BC150A9BC2F2000518468E
:109630002B60FAF725FA0225FFF7AFB941F2B821FE
:10964000C2F2000101230B6001F0D2F841F2B82A06
:109650000646634B634A644816F0010FC2F2000AE3
:1096600018BF1A464FEA56010023CAF80030FEF729
:10967000D3FEFFF745BA002001460122F9F770FD3D
:10968000322401F0ADF9FFF7C5B9584800F0CCFD20
:109690003CE55748FEF708FE4D48FEF705FE41F24F
:1096A000C82E4FF0000AC2F2000ECBF804A08BF8CF
:1096B0003CA050495048CEF800A0CDF81CA0FBF7C4
:1096C00093FAFFF77ABA41F2CC2EC2F2000EDEF81E
:1096D0000030D2F804E09E457FF425AD24E5474BE9
:1096E00047484FF0010AC3F800A0FEF7DDFD3848F7
:1096F000FEF7DAFD4349099A0DA801F0CBFE0DA84B
:10970000FAF728FA41F2982EC2F2000E0425CEF89C
:1097100000A0CDF818A0FFF749B9FEF789FB3A4B36
:1097200000221A60FFF76BB92848FEF7BDFD2848F4
:10973000FEF7BAFD6FF013015FE441F2B820C2F208
:1097400000000123036001F053F841F2B82A0646F5
:10975000234B244A244816F0010FC2F2000A4FEAB4
:10976000560118BF1A460023CAF80030FEF754FE0F
:10977000A6F1140141E400221A60FFF71FBB00228A
:109780001A60FFF773BB17221A60FFF79ABB3B22E0
:109790001A60FFF732BB41F2CC22C2F20002DAF8C3
:1097A00004C013689C457FF4F2AEF1E67C12002001
:1097B00000F3000890F20008B4F30008AC12002097
:1097C00048F300089C1200206CF30008A4F600087F
:1097D000ACE10008B4F500080CF6000888F50008B4
:1097E000A4E9000834E1000858F600088C62002063
:1097F0003CF2000884F2000878F20008C812002049
:10980000C4F50008D8F50008A8120020814A40F2EB
:10981000BC1A0023C2F2000A18461360FF23CAF8DC
:109820000030F9F721FEFFF746BA7A4A40F2BC1A37
:109830000023C2F2000A18461360FF23CAF8003062
:10984000F9F712FEFFF722BA15A800F0EDFCFAE4D2
:1098500041F2CC2AC2F2000ADDF858E0DAF8003012
:109860009E457FF4FBACFAE441F2842EC2F2000E76
:109870006948CEF80030FEF717FD6848FEF714FD82
:10988000A7E5644A40F2BC160023C2F2000618465F
:109890001360FF233360F9F7E7FD02E66048614C8F
:1098A000FEF702FD5D48FEF7FFFCFEF7AABF5E482B
:1098B000FEF7FAFC5948FEF7F7FCFEF768BF132DD8
:1098C00053D801A252F825F0F18E0008458F000808
:1098D000218F00085F8F0008878E0008DF8E000848
:1098E000AB8E0008538E0008E38D0008A58D00089C
:1098F000538D0008398D00081F8D0008058D000864
:10990000D18C0008EB8C0008A78C00087D8C000827
:1099100027990008A78B0008002042490422FAF783
:10992000BBFDFEF745BF41F2842AC2F2000A40F2B5
:10993000BC1EDAF80030D3F1010338BF0023C2F2B5
:10994000000E1846CAF800300025FF23CEF800307C
:109950003224F9F789FD05950225FFF728B9F7F7B5
:1099600023FCFBF773F9FEF7F0BE002405940025F5
:109970003224FFF71CB92D48FEF796FC2748FEF766
:1099800093FCFEF7A0BF2A48FEF78EFC2348FEF7A3
:109990008BFC00F05BF8FEF725BF2648FEF784FC41
:1099A0001E48FEF781FC00F071FB2348FEF77CFCAB
:1099B0001A48FEF779FC2068FAF796F91F48FEF777
:1099C00073FC1648FEF770FC00F076FFFEF702BF4E
:1099D0001B48FEF769FC1148FEF766FCFEF76EBFF8
:1099E0001848FEF761FC0D48FEF75EFCFEF761BF0C
:1099F0001548FEF759FC0948FEF756FCFEF754BF20
:109A0000304639460422FAF761FD00287EF447AF5C
:109A1000FEF73FBF8412002068F40008ACE10008A4
:109A200028F10008B801002024F00008F4F1000833
:109A3000DCF000086CF000088CF00008B8F00008BA
:109A4000C8F10008A8F1000884F1000830B5104BF7
:109A50001B6887B013B9002007B030BDBF2069462E
:109A60001822FAF719FD0028F5D00A486A460023A3
:109A70001478517895781C50C1EB01111C180833EB
:109A800005EB81010332402B6160F1D10120E3E756
:109A9000A4040020B062002070B548F6890686B0A4
:109AA000114C6A460023C8F68806181919594068EF
:109AB0001170A6FB00514909C1EB0115A0EB85000F
:109AC0000833517090700332402BEED1074B186869
:109AD00038B1BF2018226946FAF7F8FC003018BFE9
:109AE000012006B070BD00BFB0620020A4040020B9
:109AF000F0B400231B4D02E00833402B22D05C5908
:109B000014F0800F03EB0506F6D076689642F3D189
:109B1000C4F3C20604F0070704F0400418B1D4F1FE
:109B2000010438BF0024002CE6D0BE420DD8B1425B
:109B300034BF00260126B94288BF0026002EDBD0A4
:109B4000012000E00020F0BC7047B9428CBF002724
:109B50000127B14234BF3E4647F00106002ECBD06C
:109B6000EEE700BFB0620020704700BF70B54FF451
:109B70004064C4F2020404266420F7F74BFE6683B7
:109B80004FF40C70F7F746FE284D26831420F7F7A4
:109B900041FE00264FF496732B60344603E004B96F
:109BA0002C682B68ABB14FF440600421C4F2020072
:109BB000F6F75AFED6F1010338BF0023002C08BF88
:109BC00000230028EBD0002BEBD02E682B68002B55
:109BD000E9D13220002E18BF002C0CBF0025012532
:109BE00015D0F7F717FE4FF440600421C4F20200CD
:109BF000F6F73AFE05467820F7F70CFE6B1E584242
:109C0000C6EB040458411E2C98BF002070BDF7F726
:109C100001FE4FF440600421C4F20200F6F724FE76
:109C20007820F7F7F7FD284670BD00BF5C61002083
:109C300038B54FF44064C4F202040425052065835E
:109C4000F7F7E8FD25830A20F7F7E4FD29462046CB
:109C5000F6F70AFE04463220F7F7DCFD621E50429A
:109C6000504138BD70B5082401250026FFF7E0FFFC
:109C70006B0000B12E43013CDDB2F7D1304670BD20
:109C800038B54D1E0446EDB239B101354519FFF71F
:109C9000E9FF04F8010BAC42F9D138BD2DE9F041E0
:109CA0004FF44066804608250124C4F202060427CA
:109CB0000AE00520F7F7AEFD502037836400F7F780
:109CC000A9FD013DE4B20ED0502014EA080F7783BD
:109CD000EFD1F7F79FFD052037836400F7F79AFD72
:109CE000013DE4B2F0D1BDE8F08100BF38B54D1EB2
:109CF0000446EDB239B10135451914F8010BFFF7EF
:109D0000CDFFAC42F9D138BD10B50446FFF72EFFA8
:109D1000024680B9234603F8012B0133627003F831
:109D2000012B03F8012B03F8012B03F8012B03F897
:109D3000012B1A7010BD3320FFF7B0FF2046082119
:109D4000FFF79EFFFFF712FF012010BD70B5124B09
:109D50001A6882B00AB102B070BD012468464FF49F
:109D600040651C60C4F20205F6F774FD0820214628
:109D7000F6F71EFF042602232846694600968DF852
:109D800004408DF806408DF807408DF80530F6F751
:109D900005FD2E83DFE700BFD012002000B583B0A1
:109DA0006846F6F757FD04200121F6F701FF4FF44E
:109DB00080724FF40060002369460092C4F20200F2
:109DC00001228DF805308DF804208DF806308DF8CD
:109DD0000730F6F7E3FC4FF6E800C0F60000FEF7A8
:109DE00063FA4EF2AC10C0F60000FEF75DFA03B065
:109DF00000BD00BF10B50B4C2368012B10D04FF4F1
:109E000000604FF480710122C4F20200F6F732FDC7
:109E10000548FEF749FA0548FEF746FA0123236094
:109E200010BD00BFC4010020FCF80008ACE1000830
:109E300010B50A4C236883B14FF400604FF4807171
:109E40000022C4F20200F6F715FD0548FEF72CFAD1
:109E50000448FEF729FA0023236010BDC401002046
:109E600010F90008ACE10008F0B583B06846FDF7D2
:109E7000D3FC60B31A4A1B4B10681968013010609C
:109E80009DF8052031B302F001021749BDF80170B9
:109E9000BDF803C01A6000239DF8004018460E4626
:109EA00002E00130782B12D0CA5C0633A242F8D10E
:109EB00000EB400206EB4202B2F80150BD42F0D185
:109EC000B2F80320624503D00130782BECD1FF209B
:109ED00003B0F0BD12F00102D7D001221A60F6E7FC
:109EE000D8120020D4120020DC1200202DE9F04FFF
:109EF000DFF894814E4D002783B001263C46C246D0
:109F00002846F9F727FE2846FEF7CEF94948FEF71E
:109F1000CBF96846FDF780FC04EB440908EB4909DE
:109F20000AEB07054846FDF777FC0028FAD06A7966
:109F300012F00102F6D1D4B399F80010134602E0F2
:109F40000133A34231D018F80200884202F1060220
:109F5000F6D103EB430C0AEB4C0CB9F80100BCF84A
:109F600001E08645ECD1B9F803E0BCF803C0F44544
:109F7000E6D1FF2B19D00022134602E00133A342A1
:109F8000D0D018F802C08C4502F10602F6D103EBDE
:109F9000430C0AEB4C0CBCF801B08345EED1BCF885
:109FA00003C0F445EAD1002BBCD1142E37D0731E68
:109FB000122B3BD8DFE803F02F2D2B292725232157
:109FC0001F1D1B19171513110F0A31001A4D0134EB
:109FD0000136063794E7194DF9E7194DF7E7194DA2
:109FE000F5E7194DF3E7194DF1E7194DEFE7194D75
:109FF000EDE7194DEBE7194DE9E7194DE7E7194D85
:10A00000E5E7194DE3E7194DE1E7194DDFE7194D94
:10A01000DDE7194DDBE7194DD9E7194DD7E71948A9
:10A02000F9F798FD012003B0BDE8F08F004DCEE7B1
:10A0300038F90008ACE1000800FB0008E0FA00086D
:10A04000C0FA0008A4FA000888FA000868FA0008B4
:10A0500048FA00082CFA000810FA0008FCF9000879
:10A06000E8F90008D4F90008C0F90008A4F90008CC
:10A0700088F900086CF9000850F9000848F9000850
:10A0800024F900081CFB0008DC120020F0B5124B7C
:10A09000186883B0E8B10025104F04262C4605222D
:10A0A00030466946FAF7F8F99DF800C0BDF801108E
:10A0B000BDF8032007F805C004EB440307EB430396
:10A0C000013405360635142CA3F80110A3F803203B
:10A0D000E5D103B0F0BD00BFA4040020DC120020D5
:10A0E000F0B5114B186883B0E0B100250F4F04267E
:10A0F0002C4604EB440307EB43037A5DB3F801E01D
:10A10000B3F803308DF8002030460522694601344B
:10A11000ADF801E0ADF80330B6180635FAF7D6F918
:10A12000142CE6D103B0F0BDA4040020DC12002002
:10A1300010B582B004460B460092D0200022214682
:10A14000FDF710FAD0F1010038BF002002B010BDB9
:10A1500010B582B004460B460092D0200022214662
:10A16000FDF77EFAD0F1010038BF002002B010BD2B
:10A1700030B583B0FDF7A2F93F200DF107010122B0
:10A18000FFF7D6FF054620B301240720244B0DEB33
:10A19000000122461C60FFF7CBFF10B39DF807308B
:10A1A000002B29D100200DF107010122FFF7C0FF8C
:10A1B0000446B0B19DF807301A0619D503F07F03A5
:10A1C00000200DF1070101228DF80730FFF7C0FFD5
:10A1D0000EE00E200DF107010122FFF7A9FF044652
:10A1E00018B90024204603B030BD9DF807306BB984
:10A1F0000C4B01221A60F5E7072000230DEB00014C
:10A2000022468DF80730FFF7A3FFCBE70E200DF1B4
:10A21000070101228DF80750FFF79AFFE8E700BF1A
:10A220005C130020541300202DE9F04F434B1B68B2
:10A2300089B01BB9184609B0BDE8F08F8368026980
:10A240000193C368416902934668076880690132D7
:10A2500046F26763C6F2666303926439049183FB36
:10A2600006B90199DDF80CB0019A059083FB078AC5
:10A2700083FB0BBC83FB0118DDF810B00299DDF8FD
:10A280000CE0D017FD1783FB0121029A009183FB9C
:10A290000BB3DDF810B0C5EBAA05D1174FEAEE728B
:10A2A0004FEAEB7E05EB850BC0EBA800F417DDF859
:10A2B0000080A7EB4B0B019FC4EBA90400EB8009C6
:10A2C000C1EBA801A7EB4909029F01EB8108C2EB92
:10A2D000AC02A7EB4808039F04EB840A02EB820C54
:10A2E000CEEBA303A6EB4A06A7EB4C0C049F06EBB0
:10A2F000041603EB830E059C8DF81960A7EB4E0E38
:10A3000009EB001908EB01180CEB021C0BEB05170D
:10A3100001340EEB031E002006A907228DF81870E9
:10A320008DF81A908DF81B408DF81C808DF81DC09B
:10A330008DF81EE0FFF70CFF7DE700BF54130020EF
:10A340002DE9F04F394B1B688BB004461BB9002038
:10A350000BB0BDE8F08F002008A90722FFF7E8FE48
:10A360000028F4D09DF825A09DF820709DF8268047
:10A370009DF823909DF82430CDF818904FEA1A1BD1
:10A380004FEA171C0BEB8B0B4FEA1819CDF81CB0DA
:10A390000CEB8C0C9DF82220CDF800C009EB89094C
:10A3A00008F00F08DDF81CC005930AF00F0ACDF87D
:10A3B0000890CDF804809DF82150DDF81490DDF868
:10A3C0000480CDF80CA011090AEB4C0ADDF808C096
:10A3D00002F00F0201EB81012E091B0909F00F0B9E
:10A3E00002EB410108EB4C09069ADDF8008004936A
:10A3F00005F00F0507F00F0706EB860603EB830356
:10A4000005EB460602F1FF3C07EB48070BEB430365
:10A410000AF1FF3509F1640227606660A160C4F8A3
:10A4200018C0E3602561626192E700BF5413002009
:10A4300000B50E4B1B6883B053B1FF23C0F202037B
:10A44000984207D800220120094B1A6003B000BDD2
:10A450001846FBE70122DF200DF10701FAF71CF88F
:10A460009DF807200A2A88BF0022EDE7A4040020F7
:10A470005813002000B5094B094A1B68106883B0C7
:10A480008DF8073040B1DF2001220DF10701FAF706
:10A490001DF8003018BF012003B000BD5813002084
:10A4A000A404002041F25833C2F200031868704738
:10A4B00010B541F25834C2F200042060FFF7DAFF11
:10A4C000206810BD00B50D4B1B6883B0FF200BB991
:10A4D00003B000BD112001A90222FFF729FE0028C8
:10A4E000F6D09DF80500064B9DF804201B68C0F3CC
:10A4F000400040EA4200C01AEAE700BF54130020BF
:10A50000581300200649074A074B9A42BEBF51F82C
:10A51000040B42F8040BF8E704488047044800475E
:10A5200000FD000800000020A40200200DA6000885
:10A53000DD0100083349344A002301E041F8043BBF
:10A540009142FBD3FEF7DEF8FEE7FEE7FEE7FEE70B
:10A55000FEE7FEE7FEE7FEE7FEE7FEE7FEE7FEE7D3
:10A56000FEE7FEE7FEE7FEE7FEE7FEE7FEE7FEE7C3
:10A57000FEE7FEE7FEE7FEE7FEE7FEE7FEE7FEE7B3
:10A58000FEE7FEE7FEE7FEE7FEE7FEE7FEE7FEE7A3
:10A59000FEE7FEE7FEE7FEE7FEE7FEE7FEE7FEE793
:10A5A000FEE7FEE7FEE7FEE7FEE7FEE7FEE7FEE783
:10A5B000FEE7FEE7FEE7FEE7FEE7FEE7FEE7FEE773
:10A5C000FEE7FEE7FEE7FEE7FEE7FEE7FEE7FEE763
:10A5D000FEE7FEE7FEE7FEE7FEE7FEE7FEE7FEE753
:10A5E000FEE7FEE7FEE7FEE7FEE7FEE7FEE7FEE743
:10A5F000FEE7FEE7FEE7FEE7FEE7FEE7FEE7FEE733
:10A60000FEE70000A4020020F46200204FF46D4237
:10A61000CEF200024FF46053D2F88810C4F2020365
:10A6200041F47001C2F888101968002241F001015C
:10A6300019609A60186843F2100120F08470C2F229
:10A64000004120F4803018605960196882B021F40C
:10A6500080211960DA60009201921A6842F4803217
:10A660001A6003E0009AB2F5C06F09D01A6802F4CC
:10A6700000320192009A01320092019A002AF1D030
:10A680004FF46053C4F202031B6813F4003308BF95
:10A69000019301D001230193019B012B00D0FEE720
:10A6A0004FF46053C4F202034FF4E042196CC4F259
:10A6B000000241F080511964116841F48041116039
:10A6C0009A6822F0F0029A609A6822F460429A60D6
:10A6D0009A6842F480529A601A6822F080721A6076
:10A6E00019684FF460528801C4F20202F8D445F2AE
:10A6F0000843C0F241735360136843F080731360E2
:10A7000011684FF460538901C4F20203F8D54FF485
:10A710007052C4F20202116841F4407141F002012A
:10A720001160126802F00702022A00D0FEE79A6860
:10A7300022F003029A609A6842F002029A609A68D4
:10A7400002F00C02082AFAD14FF46D43CEF2000356
:10A750004FF000629A6002B0704700BF4FF4605340
:10A76000C4F202039A6802F00C02042A14D0082AE8
:10A770001CBF4FF41052C0F2F40212D04FF46053D9
:10A78000C4F2020318499B68C3F30313CB5C22FA9B
:10A7900003F2164B1A6070474FF49052C0F27A02DF
:10A7A000ECE75868596810F4800F586815BF4FF4EB
:10A7B00090534FF41053C0F27A03C0F2F40301F047
:10A7C0003F01B3FBF1F24FF46053C4F20203C0F354
:10A7D00088105B68C3F30143013302FB00F25B00A6
:10A7E000B2FBF3F2CAE700BFC8010020D801002085
:10A7F00000B585B001A802A903AAF9F73FFD10B979
:10A80000FF2005B000BD029B002BF9D1024B186858
:10A81000039B181AF5E700BF6013002000B50E4B2C
:10A820001B6883B053B1FF23C0F20203984207D8DC
:10A8300000220120094B1A6003B000BD1846FBE757
:10A840000122DF200DF10701F9F726FE9DF8072010
:10A850000A2A88BF0022EDE7A4040020601300202C
:10A8600000B5094B094A1B68106883B08DF80730A2
:10A8700040B1DF2001220DF10701F9F727FE00307A
:10A8800018BF012003B000BD60130020A404002005
:10A8900041F26033C2F200031868704710B541F20C
:10A8A0006034C2F200042060FFF7DAFF206810BDB8
:10A8B0000920F9F755BD00BF00B5144B1B6883B0E4
:10A8C0002BB1AA2012491022F9F7E6FD50B9102247
:10A8D0000F48104900F042FE0F4B01221A60002081
:10A8E00003B000BDBA2001A90222F9F7D5FD002866
:10A8F000EDD09DF804109DF80520074B01202D296F
:10A900001A60EDD152421A600120E9E7A404002048
:10A91000E00100202CFB0008DC01002000B5134BF7
:10A920001B68002B83B01ADB2B228DF804208DF8D6
:10A9300005300F4B1B6813B9002003B000BDAA20DF
:10A940000C491022F9F7C2FD0028F5D0BA200222E6
:10A9500001A9F9F7BBFD003018BF0120EDE75B420C
:10A960002D228DF804208DF80530E2E7DC0100206F
:10A97000A4040020E001002040F2DC13C2F2000336
:10A980001868704710B5014604460A48FDF744FDB3
:10A9900004F10C03182B0AD8074B1A68A24204D002
:10A9A0001C60FFF7BBFF012010BD012010BD00207F
:10A9B00010BD00BF3CFB0008DC01002040F2E010AD
:10A9C000C2F20000704700BF014608B540F2E01037
:10A9D000C2F2000000F099FDBDE80840FFF79EBFFD
:10A9E00040F2E010C2F20000FAF716B970B5284A3A
:10A9F00048F28013126882B0C7F65543CB1802AEF6
:10AA00004FF4616101FB023346F8043D05463046D0
:10AA100000F038FA0369DA1E052A04460CD9022B25
:10AA20002BD0092B10D18369C268D21A182A03DDF2
:10AA300053B98368022B07DC019B304603F5616341
:10AA4000019300F01FFA044663696B6123692B616F
:10AA5000E36804F10C00EB6007C8013102F26C728C
:10AA6000F6F73EFBA861236A2B62A368AB606368BC
:10AA70006B6023682B6002B070BD8369C268D21A14
:10AA8000182AE1DD002BD7D18368012BD4DCDBE76A
:10AA9000DC01002046F2700048F2200108B5C4F243
:10AAA0000200C2F20001F5F731FE60B146F270001B
:10AAB00048F22001C4F20200C2F20001F5F752FE92
:10AAC000014B00221A6008BD641300202DE9F047F5
:10AAD000DFF834E10646DEF80030002BFBD1002E13
:10AAE00000F08A80464D4748770007EB060CAC44DF
:10AAF0004FF0FF3415F802AC631C00EB440104F185
:10AB00000909802212EA0A0F0CBF4FF027084FF004
:10AB10004308013352084B4521F8028FF2D104F16A
:10AB2000080115F803AC00EB410104F11109802282
:10AB300012EA0A0F0CBF4FF027084FF04308013309
:10AB400052084B4521F8028FF2D104F1100115F89B
:10AB500001AC00EB410104F11909802212EA0A0F4D
:10AB60000CBF4FF027084FF04308013352084B4504
:10AB700021F8028FF2D1033518346545BAD100228D
:10AB800000EB4303114699520232602AFBD14FF485
:10AB9000806001240021C4F20000CEF80040F6F7E6
:10ABA000A3F846F270000021C4F20200F5F782FD1E
:10ABB000BB19DB00303346F270004FF6F8711940D4
:10ABC000C4F20200F5F780FD46F270001021224623
:10ABD000C4F20200F5F77AFD46F270002146C4F295
:10ABE0000200F5F767FD4FF48060C4F200002146D3
:10ABF000BDE8F047F6F778B8334602483746BEE777
:10AC00006B130020F817002064130020B0F5C27FFA
:10AC100010B409D80C78054A00EB400013181454FE
:10AC20004A785A708A789A7010BC7047681300206E
:10AC3000F0B469B10A4D01EB410700230478EC54EC
:10AC4000EC184678667086780333BB42A670F5D15F
:10AC50000AB9F0BC70470846F0BCFFF737BF00BF29
:10AC6000681300202DE9F041654D9AB0002401A839
:10AC70004FF40066C4F202062C60F5F7EBFD0420E9
:10AC80000121F5F795FF022703234FF040083046D6
:10AC900001A98DF809308DF80870CDF804808DF881
:10ACA0000A408DF80B40F5F779FD3A46062130460B
:10ACB000A6F81A80F5F7E4FD03A8F5F7FDFF06A84E
:10ACC000F6F768F838460121F5F780FF4FF40010D9
:10ACD0000121F5F76DFF4FF480606A23C4F2000094
:10ACE00003A90493ADF80C40ADF81440ADF80E4044
:10ACF000F5F796FF4FF4806060230126C4F2000050
:10AD000006A9ADF81830ADF81A600894ADF82440E3
:10AD1000F5F7F8FF4FF48060C4F200000821F6F761
:10AD200043F84FF48060C4F200003146F5F7CEFFDF
:10AD30004FF48060C4F200003146F6F73DF84FF45E
:10AD400080604FF400713246C4F20000F6F752F80A
:10AD50000F2268468DF800208DF801408DF80240E2
:10AD60008DF80360F5F774FA0BA8F5F791FC46F23D
:10AD700070002146C4F20200F5F79CFC46F2700018
:10AD8000C4F20200F5F75CFB40F23443C4F2000366
:10AD90000C934FF4006312934FF40053139303F595
:10ADA00095630F934FF4806311934FF440331593E1
:10ADB0004FF020630B9346F27000124B1494C4F2D0
:10ADC00002000BA91094CDF838800D9316941796B5
:10ADD000189419942746F5F727FC8DF82C408DF828
:10ADE0002D408DF82E402B68002BFCD10BA840F293
:10ADF00085110122FFF71CFF1AB0BDE8F08100BFEA
:10AE000064130020F817002000210A2200F046BC3D
:10AE100008B5074B044613B10021AFF30080054B82
:10AE20001868836A03B19847204601F071F800BFA3
:10AE30000000000054FB000870B50E4B0E4DED1ADB
:10AE4000AD1000241E4603E056F82420904701343C
:10AE5000AC42F9D101F05EF8084D094BED1AAD1086
:10AE600000241E4603E056F8242090470134AC42EB
:10AE7000F9D170BD9C0200209C020020A00200209D
:10AE80009C02002038B5074B1C68E36B05461BB9D4
:10AE9000242000F00DF8E063E16B2846BDE838405F
:10AEA00000F002B854020020002200F0C3B80000F5
:10AEB000024B0146186800F047BA00BF5402002058
:10AEC00010B5002302E0CC5CC45401339342FAD1A4
:10AED00010BD8218034601E003F8011B9342FBD129
:10AEE000704700002DE9F74F064600F09FFF40F243
:10AEF000B1739E42024640F396806FF4F663F318F6
:10AF0000A6F2B2719B1040F26D1505FB0135A6F259
:10AF10006D716FF0630391FBF3F36FF4C861ED188B
:10AF200071184FF4C87391FBF3F16D18642196FB0F
:10AF3000F1FC01FB1C6C96FBF3F103FB1161D1F1F9
:10AF40000101466006F0030638BF00210196034662
:10AF5000022407261F7A4A2F11D15F69019805EB59
:10AF6000070810B9BCF1000F00D121B13B2FD4BFAD
:10AF70000027012700E00F464744013F3FE0442FF0
:10AF800002D15F69EF193AE0019F37B9BCF1000FB8
:10AF90000CBF89464FF0010900E089462348D3F8E9
:10AFA0000CA04FF0300808FB09090127A84605E06E
:10AFB00009EB870B01375BF804BCD8445745F7DB36
:10AFC00008F1040797FBF6FB06FB1B7B5F6918691A
:10AFD000BAF1010FB8BF4FF0010A0AF1FF3AB7EB1F
:10AFE0000B0748BF073700F1FF3B072000FB0B773B
:10AFF00059F82A9000E0073F4F45FCDA474498692A
:10B00000DFF82C8008FB0707186A013C074443F867
:10B010001C7F9FD1936BD1699942ACBF0023012360
:10B020001360012000E00020BDE8FE8F58FB0008FF
:10B03000805101002DE9F84380460C46174600F088
:10B04000F5FED8F800109B4A91FBF2F3064602FB8E
:10B05000131104E001F5A83101F5C071013B00298D
:10B06000F8DB4FF4616091FBF0F200FB12113C2021
:10B07000A26091FBF0F200FB1211626021601A1DC8
:10B08000072192FBF1F001FB1022002AB8BF073222
:10B09000002BA26140F2B2754FF4C8704FF0640CFF
:10B0A000DFF81C9217DBA90704D195FBFCF20CFB1F
:10B0B000125242B995FBF0F100FB1151D1F101019F
:10B0C00038BF002100E0012159F82120934218DB0C
:10B0D00001359B1AE7E7013DAA0704D195FBFCF275
:10B0E0000CFB125242B995FBF0F100FB1151D1F16A
:10B0F000010138BF002100E0012159F821209B18EF
:10B10000E9D4A5F26C7262616B4AE3614FF03009D9
:10B1100009FB01290022226102E001319B1A216111
:10B12000216959F821209342F7DA0133E360002FB7
:10B1300040F0BA8000F0A6FC604B1B681BB373683C
:10B140009D4205D13168D8F80030F26931B90CE080
:10B150002846FFF7C7FE0028F4D110E093420CDB2D
:10B16000B26B934209DA01230BE09342FBDAB26B34
:10B170009342ACBF0023012303E0002301E04FF022
:10B18000FF33236200E02762236A2568012B0CBF8E
:10B19000F36B336A4FF4616093FBF0F200FB123300
:10B1A0003C2093FBF0F100FB11336068411AA0686A
:10B1B0006160EB1A821A3B2B2360A26003DD013130
:10B1C00061603C3B04E0002B03DA013961603C33F1
:10B1D000236063683B2B03DD0132A2603C3B04E04B
:10B1E000002B03DA013AA2603C336360A368172B9B
:10B1F0001FDDE2690132E261A2690132062AC8BF9D
:10B200000022A261E268183B0132A3602369E26078
:10B2100059F823108A4244DD0133521A0C2BE260A4
:10B2200023613ED162690023013223616261E361DF
:10B2300037E0002B35DAE269013AE261A269013AAE
:10B2400048BF0622A261E2681833013AE260A360B7
:10B250003ABB2369013B01D423611EE00B23236128
:10B2600063695A1E12F0030F626103F26B7305D11A
:10B27000642293FBF2F102FB113252B94FF4C8720F
:10B2800093FBF2F102FB1133D3F1010338BF00232A
:10B2900000E0012303F5B673E361236959F8233015
:10B2A000E36000F0F0FB01E0002323622046BDE8EC
:10B2B000F88300BF8051010058FB00085061002056
:10B2C000B8FB000830B500293BD051F8042C0B1F07
:10B2D0001C49002AB8BF9B180A6812B95A600B6053
:10B2E00030BD93420CD219685818904203D15A5875
:10B2F0008918426819605A60124A136030BD0A46C4
:10B30000516809B19942FAD9146815199D420AD1B8
:10B310001B68E318D0188842136012D108681B1804
:10B3200013604B680CE002D90C23036030BD186831
:10B330001C188C4203D10C684968001918605960C8
:10B34000536030BD4C610020F8B5CD1C25F00305DD
:10B3500008350C2D38BF0C25002D064645DB8D42E7
:10B3600000D242E0234B1B681C4612E02268521BAD
:10B370000DD40B2A02D92260A4181EE0A34203D1E7
:10B3800063681C4A136021E062685A601EE023462D
:10B390006468002CEAD123E03046214600F06AF8C8
:10B3A00038602946304600F065F8431C01461CD041
:10B3B000C41C24F00304844201D1256006E0304619
:10B3C000611A00F057F80130F7D10EE004F10B00DC
:10B3D000231D20F00700C31A0AD05A42E250F8BDDC
:10B3E000054F3B68002BDCD1D6E70C2333600020EF
:10B3F000F8BD00BF4C610020486100201A4B10B519
:10B400001C68A36BD3B91820FFF752FD43F20E332B
:10B41000A06303804AF6CD33438041F23423838016
:10B420004EF26D63C3804DF6EC63038105234381C7
:10B430000B23838101220023C0E90423A46B0B4961
:10B44000206962690A4B414303FB0212A0FB03011E
:10B45000511801220023121843EB0103C4E904230D
:10B4600023F0004010BD00BF540200202DF45158BD
:10B470002D7F954C38B5064C0023054608462360C1
:10B4800000F02CFD431C02D1236803B12B6038BDB2
:10B49000F06200200EB400B59CB04FF40271ADF81C
:10B4A00014106FF000411DAB049107914FF6FF712E
:10B4B000ADF81610084953F8042B0290069008685E
:10B4C000019302A900F0E6F9029B00221A701CB059
:10B4D0005DF804EB03B0704754020020C9B2034684
:10B4E00010F8012B12B18A42F9D102E0002918BFED
:10B4F00000231846704710F8012B11F8013B012A70
:10B5000028BF9A42F7D0D01A7047034611F8012B92
:10B5100003F8012B002AF9D17047034613F8012BD9
:10B52000002AFBD1181A0138704770B5A2B108E0A3
:10B53000012A03D128781B78C01A70BD013A002C6B
:10B54000F8D00B460546002AF4D010F8016B1C78A1
:10B550000131B442ECD0EDE7104670BD30B5013991
:10B56000034609E011F8015F03F8015B013A1C464C
:10B5700015B99B18002205E01C46002AF2D1F8E715
:10B5800004F8012B9C42FBD130BD00002DE9F74FA0
:10B5900001904148D0F800900846044614F8015B39
:10B5A00009EB05062046777807F00807FFB2002F61
:10B5B000F3D12D2D03D114F8015B012704E02B2DCD
:10B5C00004BF244614F8015B002B5ED0102B08D179
:10B5D00058E02078782801D058284ED1657810237B
:10B5E0000234002F0CBF6FF000404FF00040B0FB62
:10B5F000F3FA002603FB1A08304609EB050C9CF809
:10B6000001C00CF0040B5FFA8BFBBBF1000F01D003
:10B61000303D0BE01CF0030C1BD0BCF1010F14BF3C
:10B620004FF0570C4FF0370CCCEB05059D4210DA6C
:10B63000B6F1FF3F0AD0504506D801D1454503DC9D
:10B6400003FB0050012601E04FF0FF3614F8015BC8
:10B65000D3E7731C0AD1002F01990CBF6FF0004093
:10B660004FF0004022230B6022B912E007B14042A4
:10B670007AB106B1611E11600BE03025002BB0D10C
:10B680000823AEE7302DACD1A3E7302DA1D00A239B
:10B69000A7E7BDE8FE8F00BF5802002030B5134673
:10B6A000044A05460C46106829462246BDE830404B
:10B6B000FFF76CBF540200202DE9F74F01903D4881
:10B6C000D0F800900846044614F8015B09EB050623
:10B6D0002046777807F00807FFB2002FF3D12D2D11
:10B6E00003D114F8015B012704E02B2D04BF24468D
:10B6F00014F8015B002B57D0102B08D151E02078B3
:10B70000782801D0582847D16578102302344FF0AB
:10B71000FF3ABAFBF3FA03FB0AF000266FEA0008CF
:10B72000304609EB050C9CF801C00CF0040B5FFAE5
:10B730008BFBBBF1000F01D0303D0BE01CF0030C84
:10B740001BD0BCF1010F14BF4FF0570C4FF0370C5A
:10B75000CCEB05059D4210DAB6F1FF3F0AD050450B
:10B7600006D801D1454503DC03FB0050012601E06A
:10B770004FF0FF3614F8015BD3E7731C05D1019934
:10B7800022230B60304622B912E007B140427AB161
:10B7900006B1611E11600BE03025002BB7D10823E4
:10B7A000B5E7302DB3D1AAE7302DA8D00A23AEE7F4
:10B7B000BDE8FE8F5802002030B51346044A054606
:10B7C0000C46106829462246BDE83040FFF774BF9A
:10B7D000540200202DE9F0478D68AB4281460C46AB
:10B7E00092461F463FD38A8912F4906F39D026685B
:10B7F00009696369C1EB060803265E43022508F167
:10B80000010302F4806296FBF5F6DB1912B29E4248
:10B8100038BF1E4682B13146FFF796FD054600B996
:10B8200013E021694246FFF74BFBA38923F49063A1
:10B8300043F08003A3810CE0324600F022FB054672
:10B8400038B948462169FFF73DFD0C23C9F800309F
:10B8500018E0256166614544C8EB06062560A660D0
:10B860003D46AF4200D23D462A462068514600F090
:10B87000EFFAA3685B1BA36023685D1925600020B5
:10B88000BDE8F087A38943F04003A3814FF0FF3068
:10B89000BDE8F0872DE9F04F9DB0064603938B89F4
:10B8A00003F080031BB20D46144663B10B6953B914
:10B8B0004021FFF749FD2860286110B90C2333604F
:10B8C000D0E040236B610023099320238DF82930B9
:10B8D000DFF89C81DFF89C9130238DF82A302346D5
:10B8E0009A4613F8012B1AB9BAEB040B0FD002E0F9
:10B8F000252AF5D1F8E73046294622465B46FFF770
:10B9000069FF013000F0A780099B5B4409939AF816
:10B910000030002B00F09F8000234FF0FF32049393
:10B920000793059206938DF853301A930AF1010A92
:10B930004FF0010B05E0C8EB00000BFA00F00343E9
:10B94000049354464A482178052200F073FA0AF11C
:10B95000010A049B0028EED1D90602D520228DF8D9
:10B9600053201A0702D52B228DF8532022782A2A39
:10B9700003D0079B21460A2010E0039A111D12688C
:10B980000391002A01DB079204E0524243F00203D4
:10B9900007920493013408E000FB03230C460131B5
:10B9A0002278303A092AF7D9079323782E2B19D118
:10B9B00063782A2B09D1039B1A1D1B68039202345A
:10B9C000002BB8BF4FF0FF330BE0611C00230A20AF
:10B9D00001E000FB03230C4601312278303A092AAA
:10B9E000F7D9059323482178032200F023FA40B1C8
:10B9F0004023C9EB000003FA00F0049B03430493C7
:10BA0000013414F8011B1C488DF82810062200F0A0
:10BA100011FA88B1194B33B9039B073323F007039D
:10BA20000833039313E003AB0093304604A92A467E
:10BA3000134BAFF3008007E003AB0093304604A93B
:10BA40002A460F4B00F092F8431C074603D0099B8F
:10BA5000DB19099343E7AB8903F040031BB20BB931
:10BA6000099801E04FF0FF301DB0BDE8F08F00BF36
:10BA7000C0FB0008C6FB0008CAFB0008000000006D
:10BA8000D5B70008704770472DE9F04715461F46A7
:10BA90008A680B69DDF820809A42A8BF13462B60A4
:10BAA00091F8432006460C460AB101332B60236807
:10BAB000990602D52B6802332B60236813F0060920
:10BAC00016D094F843302268003318BF0123920641
:10BAD00016D41EE00123304639465246C047013095
:10BAE00003D14FF0FF30BDE8F08709F1010901E013
:10BAF00004F1190AE1682B68CB1A9945EADBE0E703
:10BB0000E218302182F8431094F84510023382F88D
:10BB100044103046394604F14302C0470130E0D0BA
:10BB200023682A68E16803F00603042B08BFC2EB10
:10BB300001052369A2680CBF25EAE57500259A4234
:10BB4000C4BFC3EB0203ED184FF000091A3408E03C
:10BB50000123304639462246C0470130C1D009F1A1
:10BB60000109A945F4DB0020BDE8F0872DE9FF4776
:10BB70000E7E0C9D6E2E914680460C469A4601F133
:10BB8000430200F0AF800FD8632E1DD006D8002EE0
:10BB900000F0C080582E40F0D0804FE0642E1CD0C2
:10BBA000692E40F0CA8018E0732E00F0B78005D8E7
:10BBB0006F2E2BD0702E40F0C08043E0752E25D024
:10BBC000782E40F0BA8041E02B681A1D1B682A606D
:10BBD00001F1420781F84230B3E021682B6811F08F
:10BBE000800F02D0191D296008E011F0400F03F109
:10BBF0000401296002D0B3F9005000E01D68002D57
:10BC000045DA2D236D4284F8433040E021682B68EB
:10BC100011F0800F02D0191D296007E011F0400FCC
:10BC200003F10401296001D01D8800E01D68237E16
:10BC30005F486F2B14BF0A23082324E081F8456076
:10BC40005B4807E00B6843F020030B6078235948FA
:10BC500084F8453021682B6811F0800F03F1040649
:10BC60002E6000D003E04F0601D51D8800E01D685E
:10BC7000CE0744BF41F0200121601DB9236823F0A5
:10BC8000200323601023002184F8431001E048487A
:10BC90000A236668002EA66003DB216821F00401F8
:10BCA000216005B96EB104F14201B5FBF3F603FB67
:10BCB00016550F46455D01F801593546002EF4D161
:10BCC00000E01746082B0AD12368DB0707D5616817
:10BCD0002369994203DC302307F8013C013FD21B62
:10BCE000226133E009682B6811F0800F05D0191D1F
:10BCF0002960196863690B600CE011F0400F03F1D3
:10BD00000401296003D0196863690B8002E061694E
:10BD10001B68196000232361174617E02B681A1D62
:10BD20002A601F683846FFF7F8FB63682061984275
:10BD300088BF23612369636005E004F1420784F84A
:10BD4000426001232361002384F84330CDF800A032
:10BD50004046214603AA4B46FFF796FE013002D12A
:10BD60004FF0FF3021E0404649463A462369D0472C
:10BD70000130F5D0236898070ED4E068039B984201
:10BD8000B8BF184611E00123404649463246D04725
:10BD90000130E5D0013502E0002504F11906E16823
:10BDA000039BCB1A9D42EEDBE7E704B0BDE8F087CA
:10BDB000D1FB0008E2FB000830B5141E9BB005461D
:10BDC00004DA8B2303604FF0FF301DE04FF4027262
:10BDD000ADF80C200091049101D0611E00E02146D5
:10BDE0004FF6FF7202910591ADF80E2028461A46D3
:10BDF00069461E9BFFF74EFD431C01DA8B232B6027
:10BE000014B1009B00221A701BB030BD73B50093B3
:10BE1000054B06460D461446186831462A46234609
:10BE2000FFF7CAFF7CBD00BF5402002000487047E6
:10BE30005C02002010B5C9B20346821803E0047802
:10BE400001338C4203D093421846F8D1002010BD34
:10BE5000814210B511D28C18A0420ED253428118E3
:10BE6000E418CB1801E0A15C995412F1FF32FAD228
:10BE700010BDCC5CC454013300E000239342F8D1E0
:10BE800010BDF8B5064615460C4621B91146BDE869
:10BE9000F840FFF759BA1AB9FFF714FA2C4612E026
:10BEA00000F013F8A8420ED230462946FFF74CFAAC
:10BEB000074638B121462A46FFF702F830462146A8
:10BEC000FFF700FA3C462046F8BD51F8040C002864
:10BED00002DA04390B58C01804387047094A13684D
:10BEE00063B118186946884298BF106004D9064BA0
:10BEF0000C221A604FF0FF3318467047034B136053
:10BF0000EFE700BF54610020F0620020F8620020DB
:10BF1000FEE700BFF8B500BFF8BC08BC9E467047FE
:10BF2000F8B500BFF8BC08BC9E46704765617374E5
:10BF3000657220646174653A20253034642D2530A3
:10BF400032642D253032640D0A000000536F00006A
:10BF50004D6F0000446900004D690000446F00000F
:10BF600046720000536100005375000054750000D4
:10BF70005765000054680000444346373720457237
:10BF8000726F723A20486967682070756C7365201B
:10BF90003C3D2035000000004443463737204572C1
:10BFA000726F723A20486967682070756C736520FB
:10BFB0003E3D20323500000044434637372045726D
:10BFC000726F723A20706172697479205031206901
:10BFD0006E636F72726563740000000044434637FD
:10BFE00037204572726F723A2070617269747920DD
:10BFF000503220696E636F727265637400000000D6
:10C000004443463737204572726F723A207061722E
:10C0100069747920503320696E636F72726563743E
:10C020000000000000000000000000003C42423C14
:10C0300000000000241824427E42420024003C42BA
:10C0400042423C002400424242423C007C427C424C
:10C050007C404000000000000000000000000000E4
:10C0600000000000000000000000000000000000D0
:10C0700000000000000000000000000000000000C0
:10C0800000000000000000000000000000000000B0
:10C0900000000000000000000000000000000000A0
:10C0A0000000000000000000000000000000000090
:10C0B0000000000000000000000000000000000080
:10C0C0000000000000000000000000000000000070
:10C0D0000000000000000000000000000000000060
:10C0E0000000000000000000000000000000000050
:10C0F0000000000000000000000000000000000040
:10C10000000000000000000000000000000000002F
:10C11000000000000000000000000000000000001F
:10C120000000000000000000000000003838381057
:10C1300000383800EEEE4400000000002828FE28F9
:10C14000FE2828007C92907C12927C00E2A4E810E9
:10C150002E4A8E00304830708A847A003838102099
:10C16000000000001820404040201800300804045F
:10C1700004083000004428EE284400000010107C21
:10C180001010000000000038381020000000007C73
:10C1900000000000000000003838380002040810D9
:10C1A000204080003844A2928A4438001030501059
:10C1B00010107C007C82027C8080FE007C82027CED
:10C1C00002827C00808484FE04040400FE80807C63
:10C1D00002827C007C8280FC82827C00FE840810CB
:10C1E000202020007C82827C82827C007C82827E75
:10C1F00002827C0010281000102810003838003807
:10C2000038102000081020402010080000007C009A
:10C210007C00000020100804081020007C82020C22
:10C22000100010007C82BAAABC827C0010284482D4
:10C23000FE828200FC8282FC8282FC007C82808002
:10C2400080827C00FC8282828282FC00FE8080F8F8
:10C250008080FE00FE8080F8808080007C82809E4E
:10C2600082827C00828282FE8282820038101010DC
:10C27000101038000202020282827C00848890E062
:10C2800090888400808080808080FE0082C6AA9290
:10C290008282820082C2A2928A8682007C8282820C
:10C2A00082827C00FC8282FC808080007C82828290
:10C2B0008A847A00FC8282FC888482007C82807C72
:10C2C00002827C00FE101010101010008282828208
:10C2D00082827C0082828282442810008292929222
:10C2E00092926C00824428102844820082442810D4
:10C2F00010101000FE0408102040FE007C4040405A
:10C3000040407C0080402010080402007C040404AB
:10C3100004047C001028440000000000000000001D
:10C320000000FE0038381008000000000018244209
:10C330007E424200007C427C42427C00003C424003
:10C3400040423C00007C424242427C00007E407CF5
:10C3500040407E00007E407C40404000003C424027
:10C360004E423C000042427E424242000008080821
:10C37000080808000002020202423C000042447821
:10C38000484442000040404040407E000042665A1F
:10C3900042424200004262524A464200003C42424F
:10C3A00042423C00007C42427C404000003C424211
:10C3B0004A443A00007C42427C444200003C403CFB
:10C3C00002423C00003E08080808080000424242C1
:10C3D00042423C0000424242422418000042424293
:10C3E0005A66420000422418182442000022140811
:10C3F00008080800007E040810207E00384040C075
:10C4000040403800101010001010100038040406CE
:10C410000404380060920C000000000000000000DE
:10C420000000000000000100010002000200030003
:10C4300003000400040005000500060007000800D2
:10C4400009000B000D000E00100012001400170070
:10C4500019001C001F002100240028002B002E00C2
:10C460003200360039003D00420046004A004F00CD
:10C47000540059005E00630069006E0074007A0089
:10C48000800086008C0093009900A000A700AE00F9
:10C49000B600BD00C500CD00D500DD00E500EE0012
:10C4A000F600FF00080809090A0A0B0B0C0C0D0D19
:10C4B0000E0E0F004E6F6E65000000005261696E37
:10C4C000626F77004661646500000000526F6C6C1B
:10C4D000000000004578706C6F64650052616E6406
:10C4E0006F6D0000536E616B6500000054656C65F4
:10C4F00074797065000000004375626500000000FB
:10C500004D6174726978000044726F700000000021
:10C5100053717565657A65004E6F726D616C0000D0
:10C52000436C6F636B3200000000000000000000ED
:10C53000000522000000000000152200000000009D
:10C54000000722000000000000122200000000008E
:10C550000010220000000000000C2200000000007B
:10C56000000E220000000000001322000000000066
:10C57000001122000000000000172200000000004F
:10C58000000F220000000000001622000000000042
:10C590000007172200000000001217220000000010
:10C5A0000010172200000000000B172200000000FE
:10C5B000000D1722000000000013172200000000E9
:10C5C00000111722000000000019220000000000E6
:10C5D000000418192200000000151819220000009C
:10C5E000000718192200000000121819220000008C
:10C5F0000010181922000000000C18192200000079
:10C60000000E181922000000001318192200000063
:10C610000011181922000000001B22000000000079
:10C620000004181B220000000015181B2200000047
:10C630000007181B220000000012181B2200000037
:10C640000010181B22000000000C181B2200000024
:10C65000000E181B220000000013181B220000000F
:10C660000011181B22000000001A22000000000028
:10C670000004181A220000000015181A22000000F9
:10C680000007181A220000000012181A22000000E9
:10C690000010181A22000000000C181A22000000D6
:10C6A000000E181A220000000013181A22000000C1
:10C6B0000011181A22000000001C220000000000D7
:10C6C0000004181C220000000015181C22000000A5
:10C6D0000007181C220000000012181C2200000095
:10C6E0000010181C22000000000C181C2200000082
:10C6F000000E181C220000000013181C220000006D
:10C700000011181C220000000000000000000000C2
:10C7100000091E220000000000151F22000000007A
:10C7200000071F220000000000121F22000000006E
:10C7300000101F2200000000000C1F22000000005B
:10C74000000E1F220000000000131F220000000046
:10C7500000111F220000000000171F22000000002F
:10C76000000F1F220000000000161F220000000022
:10C770000007171F220000000012171F22000000F0
:10C780000010171F22000000000B171F22000000DE
:10C79000000D171F220000000013171F22000000C9
:10C7A0000011171F2200000000191F2200000000C6
:10C7B000000418191F220000001518191F2200007C
:10C7C000000718191F220000001218191F2200006C
:10C7D000001018191F220000000C18191F22000059
:10C7E000000E18191F220000001318191F22000044
:10C7F000001118191F220000001B1F22000000005A
:10C800000004181B1F2200000015181B1F22000027
:10C810000007181B1F2200000012181B1F22000017
:10C820000010181B1F220000000C181B1F22000004
:10C83000000E181B1F2200000013181B1F220000EF
:10C840000011181B1F220000001A1F220000000008
:10C850000004181A1F2200000015181A1F220000D9
:10C860000007181A1F2200000012181A1F220000C9
:10C870000010181A1F220000000C181A1F220000B6
:10C88000000E181A1F2200000013181A1F220000A1
:10C890000011181A1F220000001C1F2200000000B7
:10C8A0000004181C1F2200000015181C1F22000085
:10C8B0000007181C1F2200000012181C1F22000075
:10C8C0000010181C1F220000000C181C1F22000062
:10C8D000000E181C1F2200000013181C1F2200004D
:10C8E0000011181C1F220000004100000000000081
:10C8F00000091E220000000000151F220000000099
:10C9000000071F220000000000121F22000000008C
:10C9100000101F2200000000000C1F220000000079
:10C92000000E1F220000000000131F220000000064
:10C9300000111F220000000000171F22000000004D
:10C94000000F1F220000000000161F220000000040
:10C950000007171F220000000012171F220000000E
:10C960000103000000000000000B171F2200000060
:10C97000000D171F220000000013171F22000000E7
:10C980000011171F2200000001171F2026000000C1
:10C9900001111F202600000001131F2026000000A7
:10C9A000010E1F2026000000010C1F2026000000A1
:10C9B00001101F202600000001121F202600000089
:10C9C00001071F202600000001151F20260000007F
:10C9D00001091F20260000000126000000000000C1
:10C9E00001091E222600000001151F22260000005A
:10C9F00001071F222600000001121F22260000004E
:10CA000001101F2226000000010C1F22260000003A
:10CA1000010E1F222600000001131F222600000025
:10CA200001111F222600000001171F22260000000E
:10CA3000010F1F222600000001161F222600000001
:10CA40000107171F222600000112171F22260000CF
:10CA500001240000000000000112171F2000000048
:10CA60000107171F2000000001161F200000000012
:10CA7000010F1F200000000001171F200000000010
:10CA800001111F200000000001131F200000000002
:10CA9000010E1F2000000000010C1F2000000000FC
:10CAA00001101F200000000001121F2000000000E4
:10CAB00001071F200000000001151F2000000000DA
:10CAC00001091E20000000000041000000000000DD
:10CAD00000091E220000000000151F2200000000B7
:10CAE00000071F220000000000121F2200000000AB
:10CAF00000101F2200000000000C1F220000000098
:10CB0000000E1F220000000000131F220000000082
:10CB100000111F220000000000171F22000000006B
:10CB2000000F1F220000000000161F22000000005E
:10CB30000007171F220000000012171F220000002C
:10CB40000003220000000000000B171F220000005D
:10CB5000000D171F220000000013171F2200000005
:10CB60000011171F2200000000191F220000000002
:10CB700001111F202600000001131F2026000000C5
:10CB8000010E1F2026000000010C1F2026000000BF
:10CB900001101F202600000001121F2026000000A7
:10CBA00001071F202600000001151F20260000009D
:10CBB00001091E20260000000126000000000000E0
:10CBC00001091E222600000001151F222600000078
:10CBD00001071F222600000001121F22260000006C
:10CBE00001101F2226000000010C1F222600000059
:10CBF000010E1F222600000001131F222600000044
:10CC000001111F222600000001191F200000000052
:10CC10000111171F200000000113171F2000000042
:10CC2000010D171F20000000010B171F200000003E
:10CC300001240000000000000112171F2000000066
:10CC40000107171F2000000001161F200000000030
:10CC5000010F1F200000000001171F20000000002E
:10CC600001111F200000000001131F200000000020
:10CC7000010E1F2000000000010C1F20000000001A
:10CC800001101F200000000001121F200000000002
:10CC900001071F200000000001151F2000000000F8
:10CCA00001091E20000000000041000000000000FB
:10CCB00000091E220000000000151F2200000000D5
:10CCC00000071F220000000000121F2200000000C9
:10CCD00000101F2200000000000C1F2200000000B6
:10CCE000000E1F220000000000131F2200000000A1
:10CCF00000111F220000000000171F22000000008A
:10CD0000000F1F220000000000161F22000000007C
:10CD10000007171F220000000012171F220000004A
:10CD20000003220000000000000B171F220000007B
:10CD3000000D171F220000000013171F2200000023
:10CD40000011171F2200000000191F220000000020
:10CD500001111F202600000001131F2026000000E3
:10CD6000010E1F2026000000010C1F2026000000DD
:10CD700001101F202600000001121F2026000000C5
:10CD800001071F202600000001151F2026000000BB
:10CD900001091E20260000000126000000000000FE
:10CDA00001091E222600000001151F222600000096
:10CDB00001071F222600000001121F22260000008A
:10CDC00001101F2226000000010C1F222600000077
:10CDD000010E1F222600000001131F222600000062
:10CDE00001111F222600000001191F200000000071
:10CDF0000111171F200000000113171F2000000061
:10CE0000010D171F20000000010B171F200000005C
:10CE100001032000000000000112171F2000000085
:10CE20000107171F2000000001161F20000000004E
:10CE3000010F1F200000000001171F20000000004C
:10CE400001111F200000000001131F20000000003E
:10CE5000010E1F2000000000010C1F200000000038
:10CE600001101F200000000001121F200000000020
:10CE700001071F200000000001151F200000000016
:10CE800001091E2000000000004100000000000019
:10CE900000091E220000000000151F2200000000F3
:10CEA00000071F220000000000121F2200000000E7
:10CEB00000101F2200000000000C1F2200000000D4
:10CEC000000E1F220000000000131F2200000000BF
:10CED00000111F220000000000171F2200000000A8
:10CEE000000F1F220000000000161F22000000009B
:10CEF0000007171F220000000012171F2200000069
:10CF00000103000000000000000B171F22000000BA
:10CF1000000D171F220000000013171F2200000041
:10CF20000011171F2200000000191F22000000003E
:10CF300001111F202600000001131F202600000001
:10CF4000010E1F2026000000010C1F2026000000FB
:10CF500001101F202600000001121F2026000000E3
:10CF600001071F202600000001151F2026000000D9
:10CF700001091E202600000001260000000000001C
:10CF800001091E222600000001151F2226000000B4
:10CF900001071F222600000001121F2226000000A8
:10CFA00001101F2226000000010C1F222600000095
:10CFB000010E1F222600000001131F222600000080
:10CFC00001111F222600000001191F20000000008F
:10CFD0000111171F200000000113171F200000007F
:10CFE000010D171F20000000010B171F200000007B
:10CFF00001240000000000000112171F20000000A3
:10D000000107171F2000000001161F20000000006C
:10D01000010F1F200000000001171F20000000006A
:10D0200001111F200000000001131F20000000005C
:10D03000010E1F2000000000010C1F200000000056
:10D0400001101F200000000001121F20000000003E
:10D0500001071F200000000001151F200000000034
:10D0600001091E2000000000004100000000000037
:10D0700000091E220000000000151F220000000011
:10D0800000071F220000000000121F220000000005
:10D0900000101F2200000000000C1F2200000000F2
:10D0A000000E1F220000000000131F2200000000DD
:10D0B00000111F220000000000171F2200000000C6
:10D0C000000F1F220000000000161F2200000000B9
:10D0D0000007171F220000000012171F2200000087
:10D0E0000003220000000000000B171F22000000B8
:10D0F000000D171F220000000013171F2200000060
:10D100000011171F2200000001171F202600000039
:10D1100001111F202600000001131F20260000001F
:10D12000010E1F2026000000010C1F202600000019
:10D1300001101F202600000001121F202600000001
:10D1400001071F202600000001151F2026000000F7
:10D1500001091E202600000001260000000000003A
:10D1600001091E222600000001151F2226000000D2
:10D1700001071F222600000001121F2226000000C6
:10D1800001101F2226000000010C1F2226000000B3
:10D19000010E1F222600000001131F22260000009E
:10D1A00001111F222600000001171F222600000087
:10D1B000010F1F222600000001161F22260000007A
:10D1C0000107171F222600000112171F2226000048
:10D1D00001032000000000000112171F20000000C2
:10D1E0000107171F2000000001161F20000000008B
:10D1F000010F1F200000000001171F200000000089
:10D2000001111F200000000001131F20000000007A
:10D21000010E1F2000000000010C1F200000000074
:10D2200001101F200000000001121F20000000005C
:10D2300001071F200000000001151F200000000052
:10D2400001091E2000000000000000000000000096
:10D250000035000000000000002B0000000000006E
:10D260000033000000000000003200000000000059
:10D27000002E000000000000003000000000000050
:10D280000028000000000000003100000000000045
:10D29000002900000000000000380000000000002D
:10D2A0000037000000000000003D0000000000000A
:10D2B0000033380000000000003238000000000099
:10D2C000002E380000000000002F38000000000091
:10D2D0000027380000000000003138000000000086
:10D2E00000293800000000000039000000000000A4
:10D2F000002C363900000000002B363900000000F9
:10D3000000333639000000000032363900000000DA
:10D31000002E3639000000000030363900000000D1
:10D3200000283639000000000031363900000000C6
:10D330000029363900000000003B0000000000001A
:10D34000002C363B00000000002B363B00000000A4
:10D350000033363B000000000032363B0000000086
:10D36000002E363B000000000030363B000000007D
:10D370000028363B000000000031363B0000000072
:10D380000029363B00000000003C000000000000C7
:10D39000002C363C00000000002B363C0000000052
:10D3A0000033363C000000000032363C0000000034
:10D3B000002E363C000000000030363C000000002B
:10D3C0000028363C000000000031363C0000000020
:10D3D0000029363C00000000003E00000000000074
:10D3E000002C363E00000000002B363E00000000FE
:10D3F0000033363E000000000032363E00000000E0
:10D40000002E363E000000000030363E00000000D6
:10D410000028363E000000000031363E00000000CB
:10D420000029363E0000000000000000000000005F
:10D4300000212D3F0000000000212B4000000000D3
:10D4400000213340000000000021324000000000B5
:10D4500000212E40000000000021304000000000AC
:10D4600000212840000000000021314000000000A1
:10D470000021294000000000002138400000000089
:10D48000002137400000000000213D400000000066
:10D4900000213338400000000021323840000000F5
:10D4A00000212E384000000000212F3840000000ED
:10D4B00000212738400000000021313840000000E2
:10D4C0000021293840000000002139400000000000
:10D4D00000212C363940000000212B363940000055
:10D4E0000021333639400000002132363940000037
:10D4F00000212E363940000000213036394000002E
:10D500000021283639400000002131363940000022
:10D51000002129363940000000213B400000000076
:10D5200000212C363B40000000212B363B40000000
:10D53000002133363B400000002132363B400000E2
:10D5400000212E363B400000002130363B400000D9
:10D55000002128363B400000002131363B400000CE
:10D56000002129363B40000000213C400000000023
:10D5700000212C363C40000000212B363C400000AE
:10D58000002133363C400000002132363C40000090
:10D5900000212E363C400000002130363C40000087
:10D5A000002128363C400000002131363C4000007C
:10D5B000002129363C40000000213E4000000000D0
:10D5C00000212C363E40000000212B363E4000005A
:10D5D000002133363E400000002132363E4000003C
:10D5E00000212E363E400000002130363E40000033
:10D5F000002128363E400000002131363E40000028
:10D60000002129363E40000000000000000000001C
:10D610000111181C1F2000000113181C1F200000FE
:10D62000010E181C1F200000010C181C1F200000F8
:10D630000110181C1F2000000112181C1F200000E0
:10D640000107181C1F2000000115181C1F200000D6
:10D650000104181C1F200000011C1F2000000000F6
:10D660000111181A1F2000000113181A1F200000B2
:10D67000010E181A1F200000010C181A1F200000AC
:10D680000110181A1F2000000112181A1F20000094
:10D690000107181A1F2000000115181A1F2000008A
:10D6A0000104181A1F20000001191F2000000000AB
:10D6B0000111181B1F2000000113181B1F20000060
:10D6C000010E181B1F200000010C181B1F2000005A
:10D6D0000110181B1F2000000112181B1F20000042
:10D6E0000107181B1F2000000115181B1F20000038
:10D6F0000104181B1F200000011B1F200000000058
:10D70000011118191F200000011318191F20000013
:10D71000010E18191F200000010C18191F2000000D
:10D72000011018191F200000011218191F200000F5
:10D73000010718191F200000011518191F200000EB
:10D74000010418191F20000001191F20000000000B
:10D750000111171F200000000113171F20000000F7
:10D76000010D171F20000000010C171F20000000F2
:10D770000110171F200000000112171F20000000D9
:10D780000107171F2000000001161F2000000000E5
:10D79000010F1F200000000001171F2000000000E3
:10D7A00001111F200000000001131F2000000000D5
:10D7B000010E1F2000000000010C1F2000000000CF
:10D7C00001101F200000000001121F2000000000B7
:10D7D00001071F200000000001151F2000000000AD
:10D7E00001091E200000000000173A0000000000A0
:10D7F000001723263A000000000F3A000000000046
:10D80000000F23263A00000000163A000000000036
:10D81000001623263A0000000007173A0000000017
:10D8200000071723263A00000012173A00000000F4
:10D8300000121723263A00000010173A00000000DB
:10D8400000101723263A0000000B173A00000000D2
:10D85000000B1723263A0000000D173A00000000C5
:10D86000000D1723263A00000013173A00000000AD
:10D8700000131723263A00000011173A0000000099
:10D8800000111723263A000000193A00000000009A
:10D89000001923263A000000000418193A0000007D
:10D8A0000004181923263A00001518193A490000F7
:10D8B0000015181923263A49000718193A4900009B
:10D8C0000007181923263A49001218193A4900008E
:10D8D0000012181923263A49001018193A49000075
:10D8E0000010181923263A49000C18193A4900006B
:10D8F000000C181923263A49000E18193A4900005D
:10D90000000E181923263A49001318193A49000045
:10D910000013181923263A49001118193A49000032
:10D920000011181923263A49001B3A49000000004B
:10D93000001B23263A4900000004181B3A49000046
:10D940000004181B23263A490015181B3A49000009
:10D950000015181B23263A490007181B3A490000F6
:10D960000007181B23263A490012181B3A490000E9
:10D970000012181B23263A490010181B3A490000D0
:10D980000010181B23263A49000C181B3A490000C6
:10D99000000C181B23263A49000E181B3A490000B8
:10D9A000000E181B23263A490013181B3A490000A1
:10D9B0000013181B23263A490011181B3A4900008E
:10D9C0000011181B23263A49000000000000000047
:10D9D0000000000000000000000000000000000047
:10D9E0000000000000000000000000000000000037
:10D9F0000000000000000000000000000000000027
:10DA00000000000000000000000000000000000016
:10DA10000000000000000000000000000000000006
:10DA20000000000000000000000000003D000000B9
:10DA3000350000002B000000330000003200000021
:10DA40002E0000003000000028000000310000001F
:10DA50002900000038000000370000003D000000F1
:10DA6000350000002B0000003300000032000000F1
:10DA70002E000000300000002800000031000000EF
:10DA80002900000038000000370000003D000000C1
:10DA90003D4100002C4100002B41000033410000BB
:10DAA000324100002E4100003041000028410000BA
:10DAB0003141000029410000384100003741000099
:10DAC0003D4100002C4100002B410000334100008B
:10DAD000324100002E41000030410000284100008A
:10DAE0003141000029410000384100003741000069
:10DAF0003D4100003D4147002C4147002B4147007C
:10DB000033414700324142482E41424830414800AB
:10DB10002841480031414800294148003841434AE2
:10DB20003741434A3D414A002C414A002B41464A75
:10DB30003341464A3241464A2E41464A304144002A
:10DB40002841440031414400294144003841440007
:10DB5000374147003D4147002A4100002C41000069
:10DB60002B41000033410000324100002E410000F3
:10DB700030410000284100003141000029410000EF
:10DB800038410000374100003D410000333841007A
:10DB9000323841002E3841002F38410027384100EB
:10DBA0003138410029384100394100002C363941D3
:10DBB0002B3639413336394132363941141D000094
:10DBC000041D0000151D0000071D0000121D0000AF
:10DBD000101D00000C1D00000E1D0000131D000094
:10DBE000111D0000171D00000F1D0000161D000074
:10DBF000041D0000151D0000071D0000121D00007F
:10DC0000101D00000C1D00000E1D0000131D000063
:10DC1000111D0000171D00000F1D0000161D000043
:10DC2000141D0000041D0000151D0000071D00004C
:10DC3000121D0000101D00000C1D00000E1D000034
:10DC4000131D0000111D0000171D00000F1D000016
:10DC5000161D000007171D0012171D0010171D00CC
:10DC60000B171D000D171D0013171D0011171D00A8
:10DC7000191D00000418191D1518191D0718191D64
:10DC80001218191D450000000000000000000000EF
:10DC90000000000000000000000000000000000084
:10DCA0000000000000000000000000000000000074
:10DCB0000000000000000000000000000000000064
:10DCC0000000000000000000000000000000000054
:10DCD0000000000000000000000000000000000044
:10DCE00000000000450000006868206D6D202831AC
:10DCF000322900006868206D6D2028323429000028
:10DD0000686820756E64206D6D202831322900000E
:10DD1000686820756E64206D6D20283234290000FB
:10DD20006D6D206E616368206868202831322B2970
:10DD3000000000006D6D206E616368206868202817
:10DD4000323429004F7373692F4265726C696E20FB
:10DD500028313229000000004F7373692F42657229
:10DD60006C696E202831322B290000004F657369E1
:10DD700020283132290000004F6573692028313294
:10DD80002B290000526865696E2F52756872202831
:10DD900031322900526865696E2F527568722028E9
:10DDA00031322B2900000000536368776162656E91
:10DDB0002028313229000000536368776162656E64
:10DDC000202831322B2900005765737369202831D0
:10DDD000322900005765737369202831322B2900DE
:10DDE000436F756E74646F776E00000054656D70DC
:10DDF000657261747572000000000000000200038B
:10DE000003000707000E03000E04000F02010004C8
:10DE100001020301020401020501070401070501D3
:10DE20000B04010B06020003020204020604020AAC
:10DE300004020E04030004030404030905030E0492
:10DE4000040003040407040B070500080508070580
:10DE50000F03060006060007060803060B03060E5E
:10DE60000407000307030B070707070E0408000455
:10DE7000080006080504080804080C04080E030836
:10DE80000E04090004090404090405090A04090E22
:10DE9000040A00040A02030A02040A06030A0A0327
:10DEA0000A0E040B00070B07040B0A080C00070CF2
:10DEB00007050C0B070D00060D00070D07030D0BE2
:10DEC000040D0F030E00060E060B0E0C040E0C06BE
:10DED0000F00070F07040F0B0700000007050000E5
:10DEE000E8DC000807060000F4DC00080805000074
:10DEF00000DD00080806000010DD00080103000036
:10DF000020DD00080104000034DD000802010000EB
:10DF100044DD00080203000058DD00080301000092
:10DF20006CDD00080303000078DD00080401000038
:10DF300084DD00080403000094DD000805020000F1
:10DF4000A8DD000805030000B8DD00080601000098
:10DF5000C8DD000806030000D4DD00080907000042
:10DF6000E0DD00080A000000ECDD000828000000E9
:10DF700054696D656F757400290D0A004F4B0000E0
:10DF80004552524F520000002D200000495041449C
:10DF90004452455353200000415020004D4F44450A
:10DFA000200000006170000054494D452000000031
:10DFB0004649524D5741524520000000434D4420F0
:10DFC00000000000485454502047455420000000F1
:10DFD0002D2D3E20000000003C30643E3C30613E70
:10DFE0000D0A00003C253032783E0000636170204D
:10DFF000222573222C22257322000000617020222A
:10E000002573222C222573220000000074696D659F
:10E010002022257322000000455350383236362026
:10E020004C4F474745520D0A00000000DCED000848
:10E03000E4ED0008ECED0008F4ED0008F8ED000850
:10E04000FCED000800EE000804EE000814E70008EC
:10E050001CE7000824E70008CCF9000828E70008BE
:10E0600034E1000834E1000834E1000834E100083C
:10E0700034E100080400000002000000020000007B
:10E0800002000000020000000CEE000818EE00087C
:10E09000DCED0008E4ED000804EE000810EB0008D9
:10E0A00014EB00081CEB000878EA00081CEE0008DE
:10E0B00020EE0008CCEB0008CCEB0008CCEB00080D
:10E0C00024EE000824EE000824EE0008DCED000831
:10E0D00028EE0008B8E4000838EE000804EE000856
:10E0E000DCED000828EE0008B8E4000804EE0008A3
:10E0F00044EE00084CEE000854EE000858EE00080C
:10E1000060EE000864EE00087CEA000804EE0008F7
:10E110006163746976650000257325640000000062
:10E12000485454502F312E3020323030204F4B0085
:10E130000D0A0D0A000000003C68746D6C3E0D0A6B
:10E14000000000003C686561643E0D0A00000000AC
:10E150003C7469746C653E003C2F7469746C653E58
:10E160000D0A00003C2F686561643E0D0A00000046
:10E170003C626F64793E0D0A000000003C48313E6D
:10E180000D0A00003C2F48313E0D0A003C6120681A
:10E190007265663D222F0000223E00003C2F613E4A
:10E1A000266E6273703B266E6273703B0D0A000030
:10E1B0004D61696E000000006E6574776F726B00D0
:10E1C0004E6574776F726B0054656D706572617423
:10E1D000757265006C6472004C445200446973703F
:10E1E0006C617900616E696D6174696F6E730000B6
:10E1F000416E696D6174696F6E730000616D626973
:10E200006C69676874000000416D62696C696768D9
:10E210007400000074696D657273000054696D6567
:10E22000727300003C503E003C7472206267636F62
:10E230006C6F723D236630663066303E0D0A00001A
:10E240003C74723E0D0A00003C74643E0000000005
:10E250003C2F74643E0000003C696E70757420743D
:10E260007970653D2274657874222069643D2200CE
:10E2700022206E616D653D22000000002220766143
:10E280006C75653D2200000022206D61786C656E22
:10E290006774683D22000000222073697A653D2280
:10E2A000000000003C74643E3C627574746F6E2024
:10E2B000747970653D227375626D697422206E6198
:10E2C0006D653D22616374696F6E222076616C75A5
:10E2D000653D227361766500223E5365743C2F6272
:10E2E0007574746F6E3E00003C2F74643E0D0A001E
:10E2F0003C7461626C6520626F726465723D303E91
:10E300000D0A00003C2F74723E0D0A003C74683EFA
:10E310003C666F6E7420636F6C6F723D626C7565E6
:10E320003E0000003C2F666F6E743E3C2F74683ECA
:10E330000D0A00003C2F7461626C653E3C503E0D3E
:10E340000A0000003C627574746F6E207479706509
:10E350003D227375626D697422206E616D653D2288
:10E36000616374696F6E222076616C75653D220071
:10E370003C2F627574746F6E3E266E6273703B0044
:10E380003C2F626F64793E0D0A0000003C2F6874D8
:10E390006D6C3E0D0A0000003C73656C6563742073
:10E3A00069643D2200000000223E0D0A00000000CA
:10E3B0003C2F73656C6563743E0D0A003C6F70748E
:10E3C000696F6E2076616C75653D22002073656C07
:10E3D00065637465640000003C2F6F7074696F6E34
:10E3E0003E0D0A00266E6273703B3C696E70757458
:10E3F00020747970653D22636865636B626F782273
:10E40000206E616D653D2200222076616C75653D50
:10E410002261637469766522200000006368656389
:10E420006B6564003C696E70757420747970653D2D
:10E430002272616E6765222069643D22000000003F
:10E4400022206D696E3D220022206D61783D220000
:10E4500022207374796C653D2277696474683A0090
:10E4600070783B0022206F6E696E7075743D2200DB
:10E470005F6F75747075742E76616C75653D000004
:10E480002E76616C7565223E000000003C6F75744D
:10E49000707574206E616D653D2200005F6F75744C
:10E4A000707574223E0000003C2F6F757470757497
:10E4B0003E0000002E0D0A0044656661756C740014
:10E4C000313500003C666F726D206D6574686F6455
:10E4D0003D224745542220616374696F6E3D222FAF
:10E4E000000000003C2F666F726D3E0D0A000000B8
:10E4F000436F6C6F727300003C74643E0D0A000041
:10E5000036340000266E6273703B266E6273703B79
:10E51000266E6273703B0D0A000000004C6561724C
:10E520006E696E672049522072656D6F7465206355
:10E530006F6E74726F6C2E2E2E000000537769740C
:10E540006368696E6720706F776572206F6E2E2E1C
:10E550002E000000537769746368696E6720706FDE
:10E56000776572206F66662E2E2E00006F66666CD1
:10E57000696E65004D696E696D756D206C656E67BD
:10E580007468206F66206B657920697320313021B3
:10E590000000000054696D657365727665722073C2
:10E5A00075636365737366756C6C79206368616EFF
:10E5B0006765642E0000000053657474696E6720FF
:10E5C0006F66206E65772074696D65736572766518
:10E5D00072206661696C65642E00000054696D6587
:10E5E0007A6F6E65207375636365737366756C6CA3
:10E5F00079206368616E6765642E000053657474EA
:10E60000696E67206F66206E65772074696D657A24
:10E610006F6E65206661696C65642E004765747471
:10E62000696E67206E65742074696D650000000076
:10E63000446973706C6179696E672074656D70658B
:10E640007261747572652E2E2E00000053746F7205
:10E650006564206D696E696D756D2076616C756598
:10E660000000000054657374696E672064697370FC
:10E670006C61792E2E2E0000536176696E672073CF
:10E68000657474696E6773207065726D616E656E16
:10E69000746C792E2E2E0000687474702070617472
:10E6A000683A20272573270D0A00000068747470EB
:10E6B00020706172616D65746572733A20272573ED
:10E6C000270D0A002F000000253032642E2530323D
:10E6D000640000002534640025303264000000002E
:10E6E000616374696F6E00006C6561726E697200BF
:10E6F000706F7765726F6E00706F7765726F6666A8
:10E7000000000000736176656461746574696D650D
:10E710000000000079656172000000006D6F6E748A
:10E7200068000000646179006D696E007361766550
:10E730007469636B65720000576F7264436C6F633A
:10E740006B00000056657273696F6E00454550524C
:10E750004F4D0000454550524F4D2056657273692C
:10E760006F6E00005469636B65720000506F7765CF
:10E7700072204F6E00000000506F776572204F6668
:10E78000660000004C6561726E2049522072656D12
:10E790006F746520636F6E74726F6C006565707264
:10E7A0006F6D64756D700000454550524F4D20648B
:10E7B000756D70003C503E0D0A3C666F6E742063B0
:10E7C0006F6C6F723D677265656E3E003C505245DE
:10E7D0003E000000253034780000000020200000BA
:10E7E0003C2F5052453E0000202020002F6E6574C3
:10E7F000776F726B0000000073617665776C616EF5
:10E8000000000000776C616E6D6F646500000000B1
:10E810007373696400000000576F7264436C6F6328
:10E820006B204E6574776F726B0000003C423E4374
:10E830006F6E6E656374696E6720746F20416363E9
:10E8400065737320506F696E742C20747279206127
:10E850006761696E206C617465722E3C2F423E00C8
:10E860003C423E53746174696E672061732041635A
:10E870006365737320506F696E742C2074727920F5
:10E88000616761696E206C617465722E3C2F423E37
:10E89000000000007361766574696D65736572765A
:10E8A000657200007361766574696D657A6F6E6577
:10E8B000000000006E657474696D65004950206148
:10E8C00064647265737300004553503832363620E5
:10E8D0006669726D7761726500000000574C414EA9
:10E8E000000000005353494400000000266E62738C
:10E8F000703B266E6273703B266E6273703B000045
:10E900004B65790054696D65207365727665720098
:10E9100054696D65207A6F6E652028474D54202B11
:10E9200029000000476574206E65742074696D6568
:10E93000000000003C503E0D0A3C666F6E74206380
:10E940006F6C6F723D7265643E3C423E0000000099
:10E950003C2F423E3C2F666F6E743E0D0A00000055
:10E960002F74656D706572617475726500000000CA
:10E970007361766574636F72727274630000000075
:10E980007361766574636F7272647331387878007E
:10E99000646973706C617974656D706572617475AA
:10E9A000726500002E350000266465673B43000059
:10E9B000576F7264436C6F636B2054656D70657242
:10E9C00061747572650000005254432074656D7067
:10E9D000657261747572650044533138787800004F
:10E9E00054656D7020636F7272656374696F6E2019
:10E9F0005254432028756E697473206F6620302E40
:10EA000035B043290000000054656D7020636F72BB
:10EA100072656374696F6E204453313878782028AA
:10EA2000756E697473206F6620302E35B0432900EF
:10EA3000446973706C61792074656D70657261747E
:10EA4000757265002F6C6472000000006C64726D5A
:10EA5000696E00006C64726D6178000073617665A8
:10EA60006175746F0000000025750000576F7264B7
:10EA7000436C6F636B204C44520000004D696E0084
:10EA80004D6178004175746F6D61746963206272C5
:10EA9000696768746E6573730000000053657420C5
:10EAA0006173206D696E696D756D2076616C756539
:10EAB00000000000536574206173206D6178696DFA
:10EAC000756D2076616C7565000000002F646973B8
:10EAD000706C617900000000736176656974697318
:10EAE000000000007361766573796E63616D626921
:10EAF00000000000736176656272696768746E6514
:10EB00007373000073617665636F6C6F72730000DE
:10EB100072656400677265656E000000626C756501
:10EB20000000000073617665646973706C61796DD3
:10EB30006F6465007361766574696E746572766181
:10EB40006C00000074657374646973706C617900A3
:10EB500073617665616C6C00576F7264436C6F63B0
:10EB60006B20446973706C61790000004553204943
:10EB7000535400005065726D616E656E7420646957
:10EB800073706C6179206F6620224553204953547D
:10EB900022000000446973706C6179204D6F6465D8
:10EBA0000000000055736520646973706C61792002
:10EBB000636F6C6F727300004272696768746E6590
:10EBC00073732028312D31352900000030000000FA
:10EBD00054656D7020646973706C617920696E741E
:10EBE000657276616C00000054657374206469730B
:10EBF000706C6179000000005361766520616C6C77
:10EC0000000000002F616E696D6174696F6E7300A2
:10EC100073617665616E696D6174696F6E00000085
:10EC200073617665636F6C6F72616E696D61746933
:10EC30006F6E00006465660073617665616E00004A
:10EC40007370256400000000666176256400000092
:10EC50007361766563616E00637370256400000004
:10EC60006364656600000000576F7264436C6F63F5
:10EC70006B20416E696D6174696F6E7300000000F6
:10EC8000416E696D6174696F6E000000436F6C6F57
:10EC90007220416E696D6174696F6E00616E2564EA
:10ECA000000000006465662564000000310000007B
:10ECB00063616E256400000063646566256400007E
:10ECC0002F616D62696C69676874000073617665B5
:10ECD000616D62696D6F6465000000007361766547
:10ECE000616D62696C656473000000007361766534
:10ECF000616D62696F666673657400007361766545
:10ED000061616E0061737025640000006164656676
:10ED100000000000576F7264436C6F636B20416D9D
:10ED200062696C6967687400234C45447300000095
:10ED30004F6666736574206F66207365636F6E64DB
:10ED4000203D203000000000416D62696C696768F9
:10ED500074204D6F6465000061616E2564000000E1
:10ED600061646566256400002F74696D65727300C7
:10ED70007361766569640000610000006F00000047
:10ED80006625640074256400576F7264436C6F637A
:10ED90006B2054696D65727300000000696425641E
:10EDA00000000000612564006F2564006825640090
:10EDB0006D256400485454502F312E3020343034A7
:10EDC000204E6F7420466F756E640000343034201E
:10EDD0004E6F7420466F756E640D0A004E616D654E
:10EDE0000000000056616C756500000059595959C2
:10EDF000000000004D4D0000444400006868000021
:10EE00006D6D0000416374696F6E0000574C414E98
:10EE100020436C69656E740041500000470000009B
:10EE20004200000036330000446563656C65726122
:10EE300074696F6E000000004661766F75726974C8
:10EE400065000000536C6F7400000000416374693A
:10EE5000766500004F6E000046726F6D0000000086
:10EE6000546F0000486F7572000000000100000040
:10EE70000F00000015000000070000000B0000005C
:10EE8000070000000B000000070000000B0000005E
:10EE90000F00000014000000000000000F00000040
:10EEA000140000000000000001000000000000004D
:10EEB00005000000020000000B0000000C00000034
:10EEC0001A000000020000000B0000000200000019
:10EED0000B00000000000000100000001C000000FB
:10EEE00028000000300000000100000001000000C8
:10EEF0000000000002000000050000000C000000FF
:10EF00001100000022000000050000000C000000BD
:10EF1000050000000C0000000000000010000000D0
:10EF20001000000020000000200000000100000090
:10EF300001000000000000000200000005000000C9
:10EF40000C0000001100000022000000050000007D
:10EF50000C000000050000000C0000000000000094
:10EF600000000000000000000000000000000000A1
:10EF7000010000000100000000000000030000008C
:10EF8000050000000C0000000F0000001E00000043
:10EF9000050000000C000000040000000B00000051
:10EFA0000000000010000000150000002500000017
:10EFB000250000000100000001000000000000002A
:10EFC000322E302E370000000D0A57656C636F6DCE
:10EFD0006520746F20576F7264436C6F636B204CB5
:10EFE0006F676765722100002D2D2D2D2D2D2D2D84
:10EFF0002D2D2D2D2D2D2D2D2D2D2D2D2D2D2D2D41
:10F000002D2D2D2D0000000056657273696F6E3A2C
:10F0100020000000727463206973206F6E6C696E4B
:10F0200065000000727463206973206F66666C6906
:10F030006E650000656570726F6D206973206F6E7C
:10F040006C696E650000000063757272656E7420F5
:10F05000656570726F6D2076657273696F6E3A20A8
:10F060003078253038780D0A000000007265616440
:10F07000696E6720697220636F6465732066726FC2
:10F080006D20656570726F6D0000000072656164CF
:10F09000696E6720646973706C617920636F6E6656
:10F0A000696775726174696F6E2066726F6D206535
:10F0B0006570726F6D00000072656164696E672033
:10F0C00074696D6573657276657220646174612020
:10F0D00066726F6D20656570726F6D007265616438
:10F0E000696E67206E696768742074696D657273F4
:10F0F0002066726F6D20656570726F6D0000000094
:10F1000072656164696E672074656D7020636F6EEF
:10F1100066696775726174696F6E2066726F6D20C3
:10F12000656570726F6D0000656570726F6D206946
:10F1300073206F66666C696E6500000075706461AF
:10F1400074696E6720454550524F4D20746F20768C
:10F15000657273696F6E203078253038780D0A003B
:10F1600077726974696E672076657273696F6E2055
:10F17000746F20454550524F4D206661696C65643F
:10F180000000000077726974696E6720495220633D
:10F190006F64657320746F20454550524F4D206653
:10F1A00061696C656400000077726974696E67203C
:10F1B000636F6E66696720746F20454550524F4DEE
:10F1C000206661696C65640077726974696E672096
:10F1D00074696D657365727665722064617461200F
:10F1E000746F20454550524F4D206661696C6564CF
:10F1F0000000000077726974696E67206E69676845
:10F20000742074696D65206461746120746F204599
:10F210004550524F4D206661696C656400000000E6
:10F2200063616C6C696E67204952206C6561726E17
:10F230002066756E6374696F6E0000007573657289
:10F2400020627574746F6E20707265737365643AB2
:10F2500020636F6E6669677572696E67206573708B
:10F2600038323636206173206163636573732070B2
:10F270006F696E7400000000776F7264636C6F6377
:10F280006B00000031323334353637383930000006
:10F29000636F6D6D616E643A207365742064697389
:10F2A000706C617920636F6C6F727320746F2025AE
:10F2B000642025642025640D0A000000636F6D6DD5
:10F2C000616E643A2073657420616D62696C696770
:10F2D000687420636F6C6F727320746F20256420D4
:10F2E00025642025640D0A00636F6D6D616E643ABC
:10F2F0002073657420706F7765722025730000009D
:10F30000636F6D6D616E643A207365742064697318
:10F31000706C6179206D6F646520746F2025640DB9
:10F320000A000000636F6D6D616E643A207365744E
:10F3300020616D62696C69676874206D6F64652017
:10F34000746F2025640D0A00636F6D6D616E643A01
:10F350002073657420616E696D6174696F6E206DD4
:10F360006F646520746F2025640D0A00636F6D6DF6
:10F37000616E643A2073657420636F6C6F722061F4
:10F380006E696D6174696F6E206D6F646520746F56
:10F390002025640D0A000000636F6D6D616E643A94
:10F3A0002073686F772074656D7065726174757213
:10F3B00065000000636F6D6D616E643A2073657463
:10F3C00020646973706C6179206272696768746E19
:10F3D00065737320746F2025642C206469736162E7
:10F3E0006C65206175746D6F6D6174696320627204
:10F3F000696768746E65737320636F6E74726F6C87
:10F4000020706572204C44520D0A0000636F6D6DD0
:10F41000616E643A2073657420616D62696C69671E
:10F420006874206272696768746E65737320746FA4
:10F430002025640D0A000000636F6D6D616E643AF3
:10F4400020656E61626C65206175746F6D617469B1
:10F4500063206272696768746E65737320636F6E90
:10F4600074726F6C00000000636F6D6D616E643AC2
:10F470002064697361626C65206175746F6D61747D
:10F480006963206272696768746E65737320636F65
:10F490006E74726F6C000000636F6D6D616E643A24
:10F4A0002073657420646973706C617920666C6187
:10F4B000677320746F2030782530327800000000A8
:10F4C000636F6D6D616E643A207374617274206451
:10F4D0006973706C6179207465737400636F6D6D0E
:10F4E000616E643A207365742074696D6520746F71
:10F4F000202573202534642D253032642D253032AB
:10F500006420253032643A253032643A2530326442
:10F510000D0A0000636F6D6D616E643A2073746153
:10F520007274206E65742074696D652072657175E2
:10F5300065737400636F6D6D616E643A206C656114
:10F54000726E20495220636F64657300636F6D6D46
:10F55000616E643A207361766520646973706C61D2
:10F56000792073657474696E67730000636F6D6DE5
:10F57000616E643A207072696E74207469636B65A1
:10F58000723A2027257327006C64723A206F6C64EE
:10F59000206272696768746E65733A202564206E14
:10F5A0006577206272696768746E6573733A2025A7
:10F5B000640D0A0065737038323636206E6F77201E
:10F5C0007570000065737038323636206E6F7720A4
:10F5D0006F6E6C696E650000202049502025730015
:10F5E00064636637373A202573202534642D25302F
:10F5F00032642D2530326420253032643A25303291
:10F60000643A253032640D0A0000000072656164BE
:10F61000207274633A202573202534642D253032FE
:10F62000642D2530326420253032643A253032642E
:10F630003A253032640D0A00466F756E64205469B5
:10F640006D65723A20257320617420253032643A4A
:10F65000253032640D0A0000676F742074656D7088
:10F66000657261747572652066726F6D20445331E6
:10F67000387878783A20256425730D0A0000000058
:10F68000676F742074656D70657261747572652042
:10F6900066726F6D205254433A20256425730D0A1B
:10F6A000000000006E6F2074656D70657261747586
:10F6B000726520617661696C61626C6500000000B2
:10F6C00075706461746520646973706C61790000A1
:10F6D00049524D503A20504F574552206B657900A2
:10F6E00049524D503A204F4B206B65790000000085
:10F6F00049524D503A2064656372656D656E7420A1
:10F70000646973706C6179206D6F6465000000003E
:10F7100049524D503A20696E6372656D656E742072
:10F72000646973706C6179206D6F6465000000001E
:10F7300049524D503A2064656372656D656E742060
:10F74000616E696D6174696F6E206D6F6465000034
:10F7500049524D503A20696E6372656D656E742032
:10F76000616E696D6174696F6E206D6F6465000014
:10F7700049524D503A2064656372656D656E742020
:10F78000686F75720000000049524D503A20696E52
:10F790006372656D656E7420686F7572000000009D
:10F7A00049524D503A2064656372656D656E7420F0
:10F7B0006D696E757465000049524D503A20696E4E
:10F7C0006372656D656E74206D696E757465000099
:10F7D00049524D503A2064656372656D656E7420C0
:10F7E000726564206272696768746E657373000085
:10F7F00049524D503A20696E6372656D656E742092
:10F80000726564206272696768746E657373000064
:10F8100049524D503A2064656372656D656E74207F
:10F82000677265656E206272696768746E6573736E
:10F830000000000049524D503A20696E6372656DB8
:10F84000656E7420677265656E20627269676874A0
:10F850006E6573730000000049524D503A20646594
:10F860006372656D656E7420626C75652062726985
:10F870006768746E6573730049524D503A20696E23
:10F880006372656D656E7420626C75652062726965
:10F890006768746E6573730049524D503A20646511
:10F8A0006372656D656E74206272696768746E65F7
:10F8B0007373000049524D503A20696E6372656D52
:10F8C000656E74206272696768746E657373000098
:10F8D00049524D503A206765742074656D706572A9
:10F8E0006174757265000000706F7765725F696E94
:10F8F000697428292063616C6C656400737769748E
:10F900006368696E6720706F776572206F6E0000A4
:10F91000737769746368696E6720706F77657220AA
:10F920006F66660020206765742074656D7065726F
:10F9300061747572650000002020706F7765722019
:10F940006F66662F6F6E000020206F6B0000000056
:10F95000202064656372656D656E742064697370E0
:10F960006C6179206D6F6465000000002020696E75
:10F970006372656D656E7420646973706C61792063
:10F980006D6F646500000000202064656372656D22
:10F99000656E7420616E696D6174696F6E206D6F44
:10F9A000646500002020696E6372656D656E742069
:10F9B000616E696D6174696F6E206D6F64650000C2
:10F9C000202064656372656D656E7420686F757262
:10F9D000000000002020696E6372656D656E742002
:10F9E000686F757200000000202064656372656DA9
:10F9F000656E74206D696E75746500002020696EF7
:10FA00006372656D656E74206D696E757465000056
:10FA1000202064656372656D656E74207265642074
:10FA20006272696768746E65737300002020696E86
:10FA30006372656D656E74207265642062726967B9
:10FA400068746E6573730000202064656372656D71
:10FA5000656E7420677265656E206272696768748E
:10FA60006E657373000000002020696E6372656D1F
:10FA7000656E7420677265656E206272696768746E
:10FA80006E65737300000000202064656372656D0D
:10FA9000656E7420626C7565206272696768746E49
:10FAA000657373002020696E6372656D656E7420E6
:10FAB000626C7565206272696768746E6573730045
:10FAC000202064656372656D656E7420676C6F627B
:10FAD000616C206272696768746E65737300000000
:10FAE0002020696E6372656D656E7420676C6F624D
:10FAF000616C206272696768746E657373000000E0
:10FB00002020746F67676C65206175746F20627266
:10FB1000696768746E657373000000002020546884
:10FB2000616E6B20796F7521000000003139322E33
:10FB300035332E3130332E31303300004E6577208F
:10FB400074696D657A6F6E653A2025640D0A000050
:10FB500043000000F40100201F0000001C00000012
:10FB60001F0000001E0000001F0000001E0000001B
:10FB70001F0000001F0000001E0000001F0000000A
:10FB80001E0000001F0000001F0000001D000000FC
:10FB90001F0000001E0000001F0000001E000000EB
:10FBA0001F0000001F0000001E0000001F000000DA
:10FBB0001E0000001F0000006D0100006E0100002B
:10FBC000232D302B2000686C4C0065666745464746
:10FBD00000303132333435363738394142434445C9
:10FBE0004600303132333435363738396162636438
:10FBF00065660000202020202020202020282828A2
:10FC000028282020202020202020202020202020E4
:10FC1000202020208810101010101010101010102C
:10FC2000101010100404040404040404040410104C
:10FC300010101010104141414141410101010101E9
:10FC40000101010101010101010101010101011095
:10FC500010101010104242424242420202020202BE
:10FC60000202020202020202020202020202021066
:10FC70001010102000000000000000000000000034
:10FC80000000000000000000000000000000000074
:10FC90000000000000000000000000000000000064
:10FCA0000000000000000000000000000000000054
:10FCB0000000000000000000000000000000000044
:10FCC0000000000000000000000000000000000034
:10FCD0000000000000000000000000000000000024
:10FCE0000000000000000000000000000000000014
:08FCF00000000000000000000C
:08FCF800E404FF7F010000009D
:10FD000000000000010203040102030406070809C1
:10FD100068BF000850BF00086CBF000870BF000833
:10FD200074BF000860BF000864BF0008FF00000047
:10FD3000FF000000E80300000100000018C50008F3
:10FD40000000000000000000000000003CE7000888
:10FD500000000000000000000000000020C50008B6
:10FD6000000000000000000000000000BCC400080B
:10FD7000040000000400000001000000200000005A
:10FD80002000000003000000B4C40008E11D0008CA
:10FD9000020000000200000000000000C4C40008CF
:10FDA000551E0008040000000400000003000000CD
:10FDB000CCC4000811290008020000000200000065
:10FDC00003000000D4C40008C5260008020000009B
:10FDD0000200000003000000DCC40008351B00081E
:10FDE000020000000200000000000000E4C400085F
:10FDF000DD2B0008020000000200000003000000EC
:10FE0000ECC40008152600080400000004000000EF
:10FE100003000000F8C40008592400080200000094
:10FE2000020000000300000000C50008352F000894
:10FE300003000000030000000300000008C50008E4
:10FE40008122000802000000020000000300000000
:10FE500010C5000801210008040000000400000093
:10FE6000030000000F00000020000000050000005B
:10FE700001000000200000003C0000000500000020
:10FE8000B4C40008010000000100000000000000F0
:10FE9000BCC40008040000000400000001000000D1
:10FEA000010000000F00000016000000FFFF00002E
:10FEB000FFFF0000D80E0000FFFFFFFFFF00000063
:10FEC000FF000000FF000000000000000000000034
:10FED0000102030406070809007A030A0100000072
:10FEE0003139322E35332E3130332E31303300005C
:10FEF0000000000000000000000000000000000002
:10FF000000000000000000000000000000000000F1
:10FF10000000000050FB000800000000000000008E
:10FF200000000000000000000000000000000000D1
:10FF300000000000000000000000000000000000C1
:10FF400000000000000000000000000000000000B1
:10FF500000000000F4010020F3FB00080100000095
:10FF6000000000004A000000000000000000000047
:10FF70000000000000000000000000000000000081
:10FF80004A00000000000000000000000000000027
:10FF9000000000000000000000000000AD010008AB
:04FFA00089010008CB
:0400000508000000EF
:00000001FF
